 CryPhysics

 Timestamp is 5036d35c (Fri Aug 24 03:05:32 2012)

 Preferred load address is 35000000

 Start         Length     Name                   Class
 0001:00000000 001dbe6aH .text                   CODE
 0001:001dbe70 0000034dH .text$yc                CODE
 0001:001dc1c0 00000255H .text$yd                CODE
 0002:00000000 00000110H .idata$5                DATA
 0002:00000110 00000004H .CRT$XCA                DATA
 0002:00000114 0000003cH .CRT$XCU                DATA
 0002:00000150 00000004H .CRT$XCZ                DATA
 0002:00000154 00000004H .CRT$XIA                DATA
 0002:00000158 00000004H .CRT$XIAA               DATA
 0002:0000015c 00000004H .CRT$XIC                DATA
 0002:00000160 00000004H .CRT$XIZ                DATA
 0002:00000170 00003dc0H .rdata                  DATA
 0002:00003f30 0000005fH .rdata$debug            DATA
 0002:00003f90 00000004H .rdata$sxdata           DATA
 0002:00003f94 00000004H .rtc$IAA                DATA
 0002:00003f98 00000004H .rtc$IZZ                DATA
 0002:00003f9c 00000004H .rtc$TAA                DATA
 0002:00003fa0 00000004H .rtc$TZZ                DATA
 0002:00003fa8 00000064H .xdata$x                DATA
 0002:0000400c 0000003cH .idata$2                DATA
 0002:00004048 00000014H .idata$3                DATA
 0002:0000405c 00000110H .idata$4                DATA
 0002:0000416c 000004e0H .idata$6                DATA
 0002:00004650 00000092H .edata                  DATA
 0003:00000000 00000af0H .data                   DATA
 0003:00000af0 000a5544H .bss                    DATA
 0004:00000000 00000004H .tls$                   DATA
 0005:00000000 00000058H .rsrc$01                DATA
 0005:00000060 00000248H .rsrc$02                DATA

  Address         Publics by Value              Rva+Base       Lib:Object

 0000:00000000       __except_list              00000000     <absolute>
 0000:00000001       ___safe_se_handler_count   00000001     <absolute>
 0000:00009876       __ldused                   00009876     <absolute>
 0000:00009876       __fltused                  00009876     <absolute>
 0000:00000000       ___ImageBase               35000000     <linker-defined>
 0001:00000000       ??1CPhysEntityProfiler@@QAE@XZ 35001000 f i articulatedentity.obj
 0001:00000050       ?AlertNeighbourhoodND@CArticulatedEntity@@UAEXH@Z 35001050 f   articulatedentity.obj
 0001:00000090       ?GetPotentialColliders@CArticulatedEntity@@UAEHAAPAPAVCPhysicalEntity@@M@Z 35001090 f   articulatedentity.obj
 0001:000000b0       ?CheckSelfCollision@CArticulatedEntity@@UAEHHH@Z 350010b0 f   articulatedentity.obj
 0001:000000f0       ?GetRigidBody@CArticulatedEntity@@UAEPAVRigidBody@@HH@Z 350010f0 f   articulatedentity.obj
 0001:00000130       ??_H@YGXPAXIHP6EPAX0@Z@Z   35001130 f i articulatedentity.obj
 0001:00000160       ?IsAwake@CArticulatedEntity@@UBEHH@Z 35001160 f   articulatedentity.obj
 0001:000001a0       ?GetMaxTimeStep@CArticulatedEntity@@UAEMM@Z 350011a0 f   articulatedentity.obj
 0001:000001c0       ?assign_to@?$matrix_product_tpl@M@@QBEXPAM@Z 350011c0 f i articulatedentity.obj
 0001:00000380       ?JointListUpdated@CArticulatedEntity@@QAEXXZ 35001380 f   articulatedentity.obj
 0001:00000440       ?BreakableConstraintsUpdated@CArticulatedEntity@@UAEXXZ 35001440 f   articulatedentity.obj
 0001:00000480       ?OnContactResolved@CArticulatedEntity@@UAEXPAUentity_contact@@HH@Z 35001480 f   articulatedentity.obj
 0001:00000500       ?GetMemoryStatistics@CArticulatedEntity@@UBEXPAVICrySizer@@@Z 35001500 f   articulatedentity.obj
 0001:00000570       ??4?$matrix_tpl@M@@QAEAAV0@ABV0@@Z 35001570 f i articulatedentity.obj
 0001:00000650       ?zero@?$matrix_tpl@M@@QAEAAV1@XZ 35001650 f i articulatedentity.obj
 0001:000006b0       ?identity@?$matrix_tpl@M@@QAEAAV1@XZ 350016b0 f i articulatedentity.obj
 0001:00000750       ??1?$ChangeRequest@Upe_action@@@@QAE@XZ 35001750 f i articulatedentity.obj
 0001:00000750       ??1?$ChangeRequest@Upe_params@@@@QAE@XZ 35001750 f i articulatedentity.obj
 0001:00000750       ??1?$ChangeRequest@Upe_geomparams@@@@QAE@XZ 35001750 f i articulatedentity.obj
 0001:000007a0       ??0?$vectorn_tpl@M@@QAE@HPAM@Z 350017a0 f i articulatedentity.obj
 0001:00000830       ??4?$vectorn_tpl@M@@QAEAAV0@ABV?$matrix_vector_product_tpl@M@@@Z 35001830 f i articulatedentity.obj
 0001:000008b0       ??Y?$vectorn_tpl@M@@QAEAAV0@ABV?$matrix_vector_product_tpl@M@@@Z 350018b0 f i articulatedentity.obj
 0001:00000930       ??Z?$vectorn_tpl@M@@QAEAAV0@ABV?$matrix_vector_product_tpl@M@@@Z 35001930 f i articulatedentity.obj
 0001:000009b0       ?sub_assign_to@?$matrix_product_tpl@M@@QBEXPAM@Z 350019b0 f i articulatedentity.obj
 0001:00000a50       ?get_iCaller@@YAHXZ        35001a50 f i articulatedentity.obj
 0001:00000a70       ??$?YMM@@YAAAV?$matrix_tpl@M@@AAV0@ABV0@@Z 35001a70 f i articulatedentity.obj
 0001:00000b40       ??$?XM@@YAAAV?$matrix_tpl@M@@AAV0@M@Z 35001b40 f i articulatedentity.obj
 0001:00000be0       ??$?0M@?$Ang3_tpl@M@@QAE@ABU?$Matrix33_tpl@M@@@Z 35001be0 f i articulatedentity.obj
 0001:00000ca0       ?ResetCollisionArea@CBVTree@@UAEXXZ 35001ca0 f i livingentity.obj
 0001:00000ca0       ?OnStructureUpdate@CPhysicalEntity@@UAEXXZ 35001ca0 f i articulatedentity.obj
 0001:00000ca0       ?SetGeomConvex@CBVTree@@UAEXXZ 35001ca0 f i livingentity.obj
 0001:00000ca0       ?AddLabelFmt@CDummyMemReplay@@UAAXPBDZZ 35001ca0 f i articulatedentity.obj
 0001:00000ca0       ?DumpStats@CDummyMemReplay@@UAEXXZ 35001ca0 f i articulatedentity.obj
 0001:00000ca0       ?AddFrameStart@CDummyMemReplay@@UAEXXZ 35001ca0 f i articulatedentity.obj
 0001:00000ca0       ?CreateJobThreads@@YAXHH@Z 35001ca0 f i jobq.obj
 0001:00000ca0       ?RemoveContext@CDummyMemReplay@@UAEXXZ 35001ca0 f i articulatedentity.obj
 0001:00000ca0       ?CompactMemory@CGeometry@@UAEXXZ 35001ca0 f i livingentity.obj
 0001:00000ca0       ?DumpSymbols@CDummyMemReplay@@UAEXXZ 35001ca0 f i articulatedentity.obj
 0001:00000ca0       ?Stop@CDummyMemReplay@@UAEXXZ 35001ca0 f i articulatedentity.obj
 0001:00000ca0       ?ExitScope@CDummyMemReplay@@UAEXXZ 35001ca0 f i articulatedentity.obj
 0001:00000ca0       ?Flush@CDummyMemReplay@@UAEXXZ 35001ca0 f i articulatedentity.obj
 0001:00000ca0       ?sp_enable_shared_from_this@detail@boost@@YAXZZ 35001ca0 f i CryPhysics.obj
 0001:00000ca0       ?AddScreenshot@CDummyMemReplay@@UAEXXZ 35001ca0 f i articulatedentity.obj
 0001:00000cb0       ?EnterScope@CDummyMemReplay@@UAE_NW4Class@EMemReplayAllocClass@@GH@Z 35001cb0 f i articulatedentity.obj
 0001:00000cc0       ?AddTexturePoolContext@CDummyMemReplay@@UAEXPAXHHHPBDI@Z 35001cc0 f i articulatedentity.obj
 0001:00000cc0       ?GetNodeChildrenBVs@CBVTree@@UAEXPBUBV@@ABU?$Vec3_tpl@M@@MAAPAU2@2H@Z 35001cc0 f i livingentity.obj
 0001:00000cd0       ?SetNetworkAuthority@CPhysicalEntity@@UAEXHH@Z 35001cd0 f i livingentity.obj
 0001:00000cd0       ?AddAllocReference@CDummyMemReplay@@UAEXPAX0@Z 35001cd0 f i articulatedentity.obj
 0001:00000cd0       ?RecomputeMassDistribution@CPhysicalEntity@@UAEXHH@Z 35001cd0 f i livingentity.obj
 0001:00000cd0       ?BucketEnableCleanups@CDummyMemReplay@@UAEXPAX_N@Z 35001cd0 f i articulatedentity.obj
 0001:00000cd0       ?Start@CDummyMemReplay@@UAEX_NPBD@Z 35001cd0 f i articulatedentity.obj
 0001:00000cd0       ?RegisterContainer@CDummyMemReplay@@UAEXPBXH@Z 35001cd0 f i articulatedentity.obj
 0001:00000cd0       ?UnMapPage@CDummyMemReplay@@UAEXPAXI@Z 35001cd0 f i articulatedentity.obj
 0001:00000cd0       ?Load@CBVTree@@UAEXAAVCMemStream@@PAVCGeometry@@@Z 35001cd0 f i livingentity.obj
 0001:00000cd0       ?BindToContainer@CDummyMemReplay@@UAEXPBX0@Z 35001cd0 f i articulatedentity.obj
 0001:00000cd0       ?OnNeighbourSplit@CPhysicalEntity@@UAEXPAV1@0@Z 35001cd0 f i livingentity.obj
 0001:00000cd0       ?SetStateFromSnapshotTxt@CPhysicalStub@@UAEXPBDH@Z 35001cd0 f i physarea.obj
 0001:00000cd0       ?SetNetworkAuthority@CPhysicalStub@@UAEXHH@Z 35001cd0 f i physarea.obj
 0001:00000cd0       ?SwapContainers@CDummyMemReplay@@UAEXPBX0@Z 35001cd0 f i articulatedentity.obj
 0001:00000cd0       ?SpuUnfriendly@CGeometry@@UAEXPADAAI@Z 35001cd0 f i livingentity.obj
 0001:00000cd0       ?UnMarkBucket@CDummyMemReplay@@UAEXHPAX@Z 35001cd0 f i articulatedentity.obj
 0001:00000cd0       ?MapPage@CDummyMemReplay@@UAEXPAXI@Z 35001cd0 f i articulatedentity.obj
 0001:00000cd0       ?UnMarkPool@CDummyMemReplay@@UAEXHPAX@Z 35001cd0 f i articulatedentity.obj
 0001:00000cd0       ?UnbindFromContainer@CDummyMemReplay@@UAEXPBX0@Z 35001cd0 f i articulatedentity.obj
 0001:00000cd0       ?MarkUsedTriangle@CBVTree@@UAEXHPAUgeometry_under_test@@@Z 35001cd0 f i livingentity.obj
 0001:00000cd0       ?RemoveGeometry@CPhysicalStub@@UAEXHH@Z 35001cd0 f i physarea.obj
 0001:00000ce0       ??_ECDummyMemReplay@@UAEPAXI@Z 35001ce0 f i articulatedentity.obj
 0001:00000ce0       ??_GCDummyMemReplay@@UAEPAXI@Z 35001ce0 f i articulatedentity.obj
 0001:00000ce0       ??_GIMemReplay@@UAEPAXI@Z  35001ce0 f i articulatedentity.obj
 0001:00000ce0       ??_EIMemReplay@@UAEPAXI@Z  35001ce0 f i articulatedentity.obj
 0001:00000d10       ?AllocRequestsQueue@CPhysicalWorld@@QAEXH@Z 35001d10 f i articulatedentity.obj
 0001:00000db0       ?FreeEntityPart@CPhysicalWorld@@QAEXPAUgeom@@@Z 35001db0 f i articulatedentity.obj
 0001:00000e20       ?FreeEntityParts@CPhysicalWorld@@QAEXPAUgeom@@H@Z 35001e20 f i articulatedentity.obj
 0001:00000e50       ?IsPODThread@@YAHPAVCPhysicalWorld@@@Z 35001e50 f i articulatedentity.obj
 0001:00000e80       ??0ae_joint@@QAE@XZ        35001e80 f i articulatedentity.obj
 0001:00001230       ??0CArticulatedEntity@@QAE@PAVCPhysicalWorld@@@Z 35002230 f   articulatedentity.obj
 0001:00001480       ?GetForeignData@CPhysicalPlaceholder@@UBEPAXH@Z 35002480 f i articulatedentity.obj
 0001:000014a0       ?GetiForeignData@CPhysicalPlaceholder@@UBEHXZ 350024a0 f i articulatedentity.obj
 0001:000014b0       ?GetWorld@CPhysicalEntity@@UBEPAUIPhysicalWorld@@XZ 350024b0 f i articulatedentity.obj
 0001:000014c0       ?DoStep@CPhysicalPlaceholder@@UAEHMH@Z 350024c0 f i physarea.obj
 0001:000014c0       ?Update@CPhysicalEntity@@UAEHMM@Z 350024c0 f i particleentity.obj
 0001:000014c0       ?DoStep@CPhysicalEntity@@UAEHMH@Z 350024c0 f i articulatedentity.obj
 0001:000014d0       ?GetMass@CPhysicalEntity@@UAEMH@Z 350024d0 f i articulatedentity.obj
 0001:000014f0       ?GetMassInv@CRigidEntity@@UAEMXZ 350024f0 f i articulatedentity.obj
 0001:00001520       ?GetType@CPhysArea@@UBE?AW4pe_type@@XZ 35002520 f i physarea.obj
 0001:00001520       ?GetSnapshotVersion@CRigidEntity@@UAEHXZ 35002520 f i articulatedentity.obj
 0001:00001530       ?GetLastTimeStep@CRigidEntity@@UAEMM@Z 35002530 f i articulatedentity.obj
 0001:00001540       ?GetMaxFriction@CRigidEntity@@UAEMXZ 35002540 f i articulatedentity.obj
 0001:00001550       ?GetType@CArticulatedEntity@@UBE?AW4pe_type@@XZ 35002550 f i articulatedentity.obj
 0001:00001550       ?GetType@CCapsuleGeom@@UAEHXZ 35002550 f i livingentity.obj
 0001:00001560       ?GetSleepSpeedChange@CArticulatedEntity@@UAEXHAAU?$Vec3_tpl@M@@0@Z 35002560 f i articulatedentity.obj
 0001:000015d0       ??4geom@@QAEAAU0@ABU0@@Z   350025d0 f i articulatedentity.obj
 0001:000016d0       ??4ae_part_info@@QAEAAU0@ABU0@@Z 350026d0 f i articulatedentity.obj
 0001:00001770       ??0CFrameProfiler@@QAE@PAUISystem@@PBDW4EProfiledSubsystem@@@Z 35002770 f i articulatedentity.obj
 0001:00001810       ??4RigidBody@@QAEAAV0@ABV0@@Z 35002810 f i articulatedentity.obj
 0001:000019d0       ?UpdatePosition@CArticulatedEntity@@QAEXH@Z 350029d0 f   articulatedentity.obj
 0001:00001b40       ?UpdateJointDyn@CArticulatedEntity@@QAEXXZ 35002b40 f   articulatedentity.obj
 0001:00001cc0       ?GetDamping@CArticulatedEntity@@UAEMM@Z 35002cc0 f   articulatedentity.obj
 0001:00001d10       ?CalcEnergy@CArticulatedEntity@@UAEMM@Z 35002d10 f   articulatedentity.obj
 0001:00002630       ??0pe_params_pos@@QAE@XZ   35003630 f i articulatedentity.obj
 0001:00002690       ?GetContactMatrix@CArticulatedEntity@@UAEXABU?$Vec3_tpl@M@@HAAU?$Matrix33_tpl@M@@@Z 35003690 f   articulatedentity.obj
 0001:00002720       ?validate@pe_params_joint@@QAE_NPBDPAUILog@@ABU?$Vec3_tpl@M@@PAUIPhysRenderer@@PAXHH@Z 35003720 f i articulatedentity.obj
 0001:00002af0       ??0pe_params_articulated_body@@QAE@XZ 35003af0 f i articulatedentity.obj
 0001:00002bf0       ??0pe_action_impulse@@QAE@XZ 35003bf0 f i articulatedentity.obj
 0001:00002c50       ?validate@pe_action_impulse@@QAE_NPBDPAUILog@@ABU?$Vec3_tpl@M@@PAUIPhysRenderer@@PAXHH@Z 35003c50 f i articulatedentity.obj
 0001:000030f0       ??0?$ChangeRequest@Upe_geomparams@@@@QAE@PAVCPhysicalPlaceholder@@PAVCPhysicalWorld@@PAUpe_geomparams@@HPAXH@Z 350040f0 f i articulatedentity.obj
 0001:00003570       ??0pe_status_dynamics@@QAE@XZ 35004570 f i articulatedentity.obj
 0001:000035f0       ??0?$ChangeRequest@X@@QAE@PAVCPhysicalPlaceholder@@PAVCPhysicalWorld@@PAXH2H@Z 350045f0 f i articulatedentity.obj
 0001:00003900       ??0pe_geomparams@@QAE@XZ   35004900 f i articulatedentity.obj
 0001:00003990       ??0?$ChangeRequest@Upe_params@@@@QAE@PAVCPhysicalPlaceholder@@PAVCPhysicalWorld@@PAUpe_params@@HPAXH@Z 35004990 f i articulatedentity.obj
 0001:00003de0       ??0pe_articgeomparams@@QAE@AAUpe_geomparams@@@Z 35004de0 f i articulatedentity.obj
 0001:00003f20       ??0?$ChangeRequest@Upe_action@@@@QAE@PAVCPhysicalPlaceholder@@PAVCPhysicalWorld@@PAUpe_action@@HPAXH@Z 35004f20 f i articulatedentity.obj
 0001:00004300       ??0geom_world_data@@QAE@XZ 35005300 f i articulatedentity.obj
 0001:00004390       ??0intersection_params@@QAE@XZ 35005390 f i articulatedentity.obj
 0001:00004460       ??$AllocPooledObj@Ugeom@@@CPhysicalWorld@@QAEPAUgeom@@AAPAU1@AAH1ACH@Z 35005460 f i articulatedentity.obj
 0001:000045a0       ??$ReallocateList@Uae_joint@@@@YAPAUae_joint@@AAPAU0@HH_N1@Z 350055a0 f i articulatedentity.obj
 0001:000046d0       ??$ReallocateList@Uae_part_info@@@@YAPAUae_part_info@@AAPAU0@HH_N1@Z 350056d0 f i articulatedentity.obj
 0001:00004770       ?CryGetIMemReplay@@YAPAUIMemReplay@@XZ 35005770 f i articulatedentity.obj
 0001:000047d0       ?GetLocTransform@CPhysicalEntity@@UAEXHAAU?$Vec3_tpl@M@@AAU?$Quat_tpl@M@@AAM@Z 350057d0 f i articulatedentity.obj
 0001:00004a70       ?AllocEntityParts@CPhysicalWorld@@QAEPAUgeom@@H@Z 35005a70 f i articulatedentity.obj
 0001:00004ac0       ?Loc2Glob@@YA?AU?$Vec3_tpl@M@@ABUentity_contact@@ABU1@H@Z 35005ac0 f i articulatedentity.obj
 0001:00004d40       ??1CArticulatedEntity@@UAE@XZ 35005d40 f   articulatedentity.obj
 0001:00004dd0       ??0geom@@QAE@ABU0@@Z       35005dd0 f i articulatedentity.obj
 0001:00004ed0       ?RemoveGeometry@CArticulatedEntity@@UAEXHH@Z 35005ed0 f   articulatedentity.obj
 0001:00005580       ?GetParams@CArticulatedEntity@@UBEHPAUpe_params@@@Z 35006580 f   articulatedentity.obj
 0001:00005d50       ?GetStatus@CArticulatedEntity@@UBEHPAUpe_status@@@Z 35006d50 f   articulatedentity.obj
 0001:00006710       ?GetRigidBodyData@CArticulatedEntity@@UAEPAVRigidBody@@PAV2@H@Z 35007710 f   articulatedentity.obj
 0001:00006790       ?OnDelayedStep@CArticulatedEntity@@UAEXAAVCMemStreamA@@@Z 35007790 f   articulatedentity.obj
 0001:000069d0       ?UpdateJointRotationAxes@CArticulatedEntity@@QAEXH@Z 350079d0 f   articulatedentity.obj
 0001:000070a0       ?CalcBodyZa@CArticulatedEntity@@QAEHHMAAV?$vectorn_tpl@M@@@Z 350080a0 f   articulatedentity.obj
 0001:000081a0       ?CalcBodyIa@CArticulatedEntity@@QAEHHAAV?$matrix_tpl@M@@@Z 350091a0 f   articulatedentity.obj
 0001:0000ae10       ?CollectPendingImpulses@CArticulatedEntity@@QAEHHAAH@Z 3500be10 f   articulatedentity.obj
 0001:0000c090       ?PropagateImpulses@CArticulatedEntity@@QAEXABU?$Vec3_tpl@M@@H@Z 3500d090 f   articulatedentity.obj
 0001:0000c7b0       ?CalcVelocityChanges@CArticulatedEntity@@QAEXMABU?$Vec3_tpl@M@@0@Z 3500d7b0 f   articulatedentity.obj
 0001:0000ce20       ?CalcBodiesIinv@CArticulatedEntity@@QAEXH@Z 3500de20 f   articulatedentity.obj
 0001:0000ffa0       ?GetStateSnapshot@CArticulatedEntity@@UAEHV?$CSerializeWrapper@UISerialize@@@@MH@Z 35010fa0 f   articulatedentity.obj
 0001:00010350       ?CreateConstraintContact@CArticulatedEntity@@QAEPAUentity_contact@@H@Z 35011350 f   articulatedentity.obj
 0001:00010590       ?RegisterContacts@CArticulatedEntity@@UAEHMH@Z 35011590 f   articulatedentity.obj
 0001:00011c90       ??0pe_params_buoyancy@@QAE@XZ 35012c90 f i articulatedentity.obj
 0001:00011d30       ??_ECArticulatedEntity@@UAEPAXI@Z 35012d30 f i articulatedentity.obj
 0001:00011d30       ??_GCArticulatedEntity@@UAEPAXI@Z 35012d30 f i articulatedentity.obj
 0001:00011d60       ?AddGeometry@CArticulatedEntity@@UAEHPAUphys_geometry@@PAUpe_geomparams@@HH@Z 35012d60 f   articulatedentity.obj
 0001:00013e10       ?RecomputeMassDistribution@CArticulatedEntity@@UAEXHH@Z 35014e10 f   articulatedentity.obj
 0001:00015630       ?Action@CArticulatedEntity@@UAEHPAUpe_action@@H@Z 35016630 f   articulatedentity.obj
 0001:00018220       ?CheckForGimbalLock@CArticulatedEntity@@QAEXH@Z 35019220 f   articulatedentity.obj
 0001:000185d0       ?SyncBodyWithJoint@CArticulatedEntity@@QAEXHH@Z 350195d0 f   articulatedentity.obj
 0001:00019e20       ?SyncJointWithBody@CArticulatedEntity@@QAEXHH@Z 3501ae20 f   articulatedentity.obj
 0001:0001aa50       ?StepJoint@CArticulatedEntity@@QAEHHMAAHHH@Z 3501ba50 f   articulatedentity.obj
 0001:0001dc10       ?StepFeatherstone@CArticulatedEntity@@QAE?AU?$Vec3_tpl@M@@MHAAU?$Matrix33_tpl@M@@@Z 3501ec10 f   articulatedentity.obj
 0001:0001f750       ?StepBack@CArticulatedEntity@@UAEXM@Z 35020750 f   articulatedentity.obj
 0001:000205d0       ?GetStateSnapshot@CArticulatedEntity@@UAEHAAVCStream@@MH@Z 350215d0 f   articulatedentity.obj
 0001:00020b50       ?SetStateFromSnapshot@CArticulatedEntity@@UAEHV?$CSerializeWrapper@UISerialize@@@@H@Z 35021b50 f   articulatedentity.obj
 0001:00021210       ?Update@CArticulatedEntity@@UAEHMM@Z 35022210 f   articulatedentity.obj
 0001:00021f60       ?SyncWithHost@CArticulatedEntity@@QAEHHM@Z 35022f60 f   articulatedentity.obj
 0001:00022b10       ?Step@CArticulatedEntity@@UAEHM@Z 35023b10 f   articulatedentity.obj
 0001:000249a0       ?SetParams@CArticulatedEntity@@UAEHPAUpe_params@@H@Z 350259a0 f   articulatedentity.obj
 0001:000291b0       ?PrepareForIntersectionTest@CBVTree@@UAEHPAUgeometry_under_test@@PAVCGeometry@@0@Z 3502a1b0 f i livingentity.obj
 0001:000291d0       ?CalcEnergy@CPhysicalEntity@@UAEMM@Z 3502a1d0 f i particleentity.obj
 0001:000291d0       ?SplitPriority@CBVTree@@UAEMPBUBV@@@Z 3502a1d0 f i livingentity.obj
 0001:000291e0       ?CalcVolumetricPressure@CHeightfield@@UAEXPAUgeom_world_data@@ABU?$Vec3_tpl@M@@MM1AAU3@2@Z 3502a1e0 f i heightfieldgeom.obj
 0001:000291e0       ?GetNodeChildrenBVs@CBVTree@@UAEXABU?$Matrix33_tpl@M@@ABU?$Vec3_tpl@M@@MPBUBV@@AAPAU4@3H@Z 3502a1e0 f i livingentity.obj
 0001:000291e0       ?CalcVolumetricPressure@CVoxelGeom@@UAEXPAUgeom_world_data@@ABU?$Vec3_tpl@M@@MM1AAU3@2@Z 3502a1e0 f i geoman.obj
 0001:000291e0       ?CalcVolumetricPressure@CGeometry@@UAEXPAUgeom_world_data@@ABU?$Vec3_tpl@M@@MM1AAU3@2@Z 3502a1e0 f i livingentity.obj
 0001:000291f0       ?ExitScope_Realloc@CDummyMemReplay@@UAEXIIII@Z 3502a1f0 f i articulatedentity.obj
 0001:000291f0       ?DelayedIntersect@CPhysicalEntity@@UAEXPAUgeom_contact@@HPAPAV1@PAY01H@Z 3502a1f0 f i livingentity.obj
 0001:000291f0       ?GetNodeChildrenBVs@CBVTree@@UAEXPBUBV@@AAPAU2@1H@Z 3502a1f0 f i livingentity.obj
 0001:000291f0       ?MarkBucket@CDummyMemReplay@@UAEXHIPAXI@Z 3502a1f0 f i articulatedentity.obj
 0001:000291f0       ?AddContextV@CDummyMemReplay@@UAEXHIPBDPAD@Z 3502a1f0 f i articulatedentity.obj
 0001:00029200       ?GetMassInv@CPhysicalEntity@@UAEMXZ 3502a200 f i particleentity.obj
 0001:00029200       ?GetVolume@CGeometry@@UAEMXZ 3502a200 f i livingentity.obj
 0001:00029200       ?GetMaxSkipDim@CBVTree@@UAEMXZ 3502a200 f i livingentity.obj
 0001:00029210       ?GetNodeContentsIdx@CBVTree@@UAEHHAAH@Z 3502a210 f i livingentity.obj
 0001:00029230       ??_GCRayBV@@UAEPAXI@Z      3502a230 f i livingentity.obj
 0001:00029230       ??_GCSingleBoxTree@@UAEPAXI@Z 3502a230 f i livingentity.obj
 0001:00029230       ??_GCBVTree@@UAEPAXI@Z     3502a230 f i livingentity.obj
 0001:00029230       ??_GCVoxelBV@@UAEPAXI@Z    3502a230 f i geoman.obj
 0001:00029230       ??_ECVoxelBV@@UAEPAXI@Z    3502a230 f i geoman.obj
 0001:00029230       ??_ECSingleBoxTree@@UAEPAXI@Z 3502a230 f i livingentity.obj
 0001:00029230       ??_ECRayBV@@UAEPAXI@Z      3502a230 f i livingentity.obj
 0001:00029230       ??_ECBVTree@@UAEPAXI@Z     3502a230 f i livingentity.obj
 0001:00029260       ?GetType@CRayGeom@@UAEHXZ  3502a260 f i livingentity.obj
 0001:00029260       ?GetType@CRayBV@@UAEHXZ    3502a260 f i livingentity.obj
 0001:00029260       ?GetType@CWheeledVehicleEntity@@UBE?AW4pe_type@@XZ 3502a260 f i wheeledvehicleentity.obj
 0001:00029270       ?Build@CRayBV@@UAEMPAVCGeometry@@@Z 3502a270 f i livingentity.obj
 0001:00029270       ?Build@CVoxelBV@@UAEMPAVCGeometry@@@Z 3502a270 f i geoman.obj
 0001:00029280       ??1CLivingEntity@@UAE@XZ   3502a280 f   livingentity.obj
 0001:00029340       ?GetDamping@CPhysicalEntity@@UAEMM@Z 3502a340 f i livingentity.obj
 0001:00029350       ?GetMaxFriction@CPhysicalEntity@@UAEMXZ 3502a350 f i livingentity.obj
 0001:00029360       ?IgnoreCollisionsWith@CPhysicalEntity@@UBE_NPBV1@H@Z 3502a360 f i livingentity.obj
 0001:00029370       ?PreparePrimitive@CGeometry@@UAEHPAUgeom_world_data@@AAPAUprimitive@primitives@@H@Z 3502a370 f i livingentity.obj
 0001:00029370       ?RemoveContactPoint@CPhysicalEntity@@UAEHPAV1@ABU?$Vec3_tpl@M@@M@Z 3502a370 f i livingentity.obj
 0001:00029380       ?ExitScope_Free@CDummyMemReplay@@UAEXI@Z 3502a380 f i articulatedentity.obj
 0001:00029380       ?AddLabel@CDummyMemReplay@@UAEXPBD@Z 3502a380 f i articulatedentity.obj
 0001:00029380       ?GetBBox@CBVTree@@UAEXPAUbox@primitives@@@Z 3502a380 f i livingentity.obj
 0001:00029380       ?CheckAdditionalGeometry@CRigidEntity@@UAEXM@Z 3502a380 f i articulatedentity.obj
 0001:00029380       ?Save@CBVTree@@UAEXAAVCMemStream@@@Z 3502a380 f i livingentity.obj
 0001:00029380       ?StepBack@CLivingEntity@@UAEXM@Z 3502a380 f i livingentity.obj
 0001:00029380       ?GetMemoryStatistics@CGeometry@@UAEXPAVICrySizer@@@Z 3502a380 f i livingentity.obj
 0001:00029380       ?ReleaseLastSweptBVs@CBVTree@@UAEXH@Z 3502a380 f i livingentity.obj
 0001:00029380       ?PrepareForRayTest@CVoxelGeom@@UAEXM@Z 3502a380 f i geoman.obj
 0001:00029380       ?StepBack@CPhysicalStub@@UAEXM@Z 3502a380 f i physarea.obj
 0001:00029380       ?OnDelayedStep@CPhysicalEntity@@UAEXAAVCMemStreamA@@@Z 3502a380 f i livingentity.obj
 0001:00029380       ?SetData@CGeometry@@UAEXPBUprimitive@primitives@@@Z 3502a380 f i livingentity.obj
 0001:00029380       ?AddAdditionalImpulses@CRigidEntity@@UAEXM@Z 3502a380 f i articulatedentity.obj
 0001:00029380       ?PrepareForRayTest@CGeometry@@UAEXM@Z 3502a380 f i livingentity.obj
 0001:00029380       ?Load@CGeometry@@UAEXAAVCMemStream@@@Z 3502a380 f i livingentity.obj
 0001:00029380       ?CleanupAfterIntersectionTest@CGeometry@@UAEXPAUgeometry_under_test@@@Z 3502a380 f i livingentity.obj
 0001:00029380       ?GetMemoryStatistics@CPhysicalStub@@UBEXPAVICrySizer@@@Z 3502a380 f i physarea.obj
 0001:00029380       ?StepBack@CPhysicalEntity@@UAEXM@Z 3502a380 f i particleentity.obj
 0001:00029380       ?CleanupAfterIntersectionTest@CBVTree@@UAEXPAUgeometry_under_test@@@Z 3502a380 f i livingentity.obj
 0001:00029380       ?DestroyAuxilaryMeshData@CGeometry@@UAEXH@Z 3502a380 f i livingentity.obj
 0001:00029380       ?PrepareForRayTest@CHeightfield@@UAEXM@Z 3502a380 f i waterman.obj
 0001:00029380       ?RemoveAllocReference@CDummyMemReplay@@UAEXPAX@Z 3502a380 f i articulatedentity.obj
 0001:00029380       ?AddSizerTree@CDummyMemReplay@@UAEXPBD@Z 3502a380 f i articulatedentity.obj
 0001:00029380       ?Save@CGeometry@@UAEXAAVCMemStream@@@Z 3502a380 f i livingentity.obj
 0001:00029380       ?GetMemoryStatistics@CPhysicalPlaceholder@@UBEXPAVICrySizer@@@Z 3502a380 f i physarea.obj
 0001:00029380       ?StartOnCommandLine@CDummyMemReplay@@UAEXPBD@Z 3502a380 f i articulatedentity.obj
 0001:00029380       ?SetDynPoolSize@CPhysicalWorld@@UAEXH@Z 3502a380 f i physicalworld.obj
 0001:00029380       ?StartStep@CPhysicalStub@@UAEXM@Z 3502a380 f i physarea.obj
 0001:00029380       ?StartStep@CPhysicalEntity@@UAEXM@Z 3502a380 f i physicalentity.obj
 0001:00029380       ?GetMemoryStatistics@CBVTree@@UAEXPAVICrySizer@@@Z 3502a380 f i livingentity.obj
 0001:00029380       ?ReleaseLastBVs@CBVTree@@UAEXH@Z 3502a380 f i livingentity.obj
 0001:00029380       ?UnregisterContainer@CDummyMemReplay@@UAEXPBX@Z 3502a380 f i articulatedentity.obj
 0001:00029380       ?GetInfo@CDummyMemReplay@@UAEXAAUCryReplayInfo@@@Z 3502a380 f i articulatedentity.obj
 0001:00029390       ?GetRigidBodyData@CLivingEntity@@UAEPAVRigidBody@@PAV2@H@Z 3502a390 f i livingentity.obj
 0001:000293f0       ?GetMassInv@CLivingEntity@@UAEMXZ 3502a3f0 f i livingentity.obj
 0001:00029400       ?GetSpatialContactMatrix@CLivingEntity@@UAEXABU?$Vec3_tpl@M@@HQAY05M@Z 3502a400 f i livingentity.obj
 0001:00029450       ?ReleaseGroundCollider@CLivingEntity@@QAEXXZ 3502a450 f   livingentity.obj
 0001:00029470       ?GetParams@CLivingEntity@@UBEHPAUpe_params@@@Z 3502a470 f   livingentity.obj
 0001:000296f0       ?AddGeometry@CLivingEntity@@UAEHPAUphys_geometry@@PAUpe_geomparams@@HH@Z 3502a6f0 f   livingentity.obj
 0001:00029740       ?RemoveGeometry@CLivingEntity@@UAEXHH@Z 3502a740 f   livingentity.obj
 0001:00029770       ?UpdatePosition@CLivingEntity@@QAEXABU?$Vec3_tpl@M@@PBU2@H@Z 3502a770 f   livingentity.obj
 0001:000298a0       ?StartStep@CLivingEntity@@UAEXM@Z 3502a8a0 f   livingentity.obj
 0001:000298f0       ?float2int@@YAHM@Z         3502a8f0 f i livingentity.obj
 0001:00029910       ?GetMemoryStatistics@CLivingEntity@@UBEXPAVICrySizer@@@Z 3502a910 f   livingentity.obj
 0001:00029950       ??$SignalEvent@UEventPhysBBoxOverlap@@@CPhysicalWorld@@QAEHPAUEventPhysBBoxOverlap@@H@Z 3502a950 f i livingentity.obj
 0001:000299c0       ??$SignalEvent@UEventPhysCollision@@@CPhysicalWorld@@QAEHPAUEventPhysCollision@@H@Z 3502a9c0 f i livingentity.obj
 0001:00029a30       ??$SignalEvent@UEventPhysPostStep@@@CPhysicalWorld@@QAEHPAUEventPhysPostStep@@H@Z 3502aa30 f i livingentity.obj
 0001:00029aa0       ??_GIGeometry@@UAEPAXI@Z   3502aaa0 f i livingentity.obj
 0001:00029aa0       ??_EIGeometry@@UAEPAXI@Z   3502aaa0 f i livingentity.obj
 0001:00029ad0       ?AddRef@CGeometry@@UAEHXZ  3502aad0 f i livingentity.obj
 0001:00029ae0       ?GetForeignIdx@CGeometry@@UAEHH@Z 3502aae0 f i livingentity.obj
 0001:00029ae0       ?PointInsideStatus@CVoxelGeom@@UAEHABU?$Vec3_tpl@M@@@Z 3502aae0 f i geoman.obj
 0001:00029ae0       ?PointInsideStatus@CGeometry@@UAEHABU?$Vec3_tpl@M@@@Z 3502aae0 f i livingentity.obj
 0001:00029af0       ?GetPrimitiveId@CGeometry@@UAEHHH@Z 3502aaf0 f i livingentity.obj
 0001:00029b00       ?IsConvex@CGeometry@@UAEHM@Z 3502ab00 f i livingentity.obj
 0001:00029b00       ?Step@CPhysicalEntity@@UAEHM@Z 3502ab00 f i physicalentity.obj
 0001:00029b10       ?UnprojectSphere@CGeometry@@UAEHU?$Vec3_tpl@M@@MMPAUcontact@@@Z 3502ab10 f i livingentity.obj
 0001:00029b20       ?Subtract@CGeometry@@UAEHPAUIGeometry@@PAUgeom_world_data@@1H@Z 3502ab20 f i livingentity.obj
 0001:00029b30       ?GetForeignData@CGeometry@@UAEPAXH@Z 3502ab30 f i livingentity.obj
 0001:00029b50       ?GetiForeignData@CGeometry@@UAEHXZ 3502ab50 f i livingentity.obj
 0001:00029b60       ?SetForeignData@CGeometry@@UAEXPAXH@Z 3502ab60 f i livingentity.obj
 0001:00029b80       ?DrawToOcclusionCubemap@CGeometry@@UAEHPBUgeom_world_data@@HHHPAUSOcclusionCubeMap@@@Z 3502ab80 f i livingentity.obj
 0001:00029b90       ?Load@CGeometry@@UAEXAAVCMemStream@@V?$strided_pointer@$$CBU?$Vec3_tpl@M@@@@V?$strided_pointer@G@@PAD@Z 3502ab90 f i livingentity.obj
 0001:00029bb0       ?PrepareForIntersectionTest@CGeometry@@UAEHPAUgeometry_under_test@@PAV1@0_N@Z 3502abb0 f i livingentity.obj
 0001:00029bc0       ?GetPrimitiveList@CGeometry@@UAEHHHHPAUprimitive@primitives@@HPAUgeometry_under_test@@10PAD@Z 3502abc0 f i livingentity.obj
 0001:00029bd0       ?GetUnprojectionCandidates@CGeometry@@UAEHHPBUcontact@@AAPAUprimitive@primitives@@AAPAHPAUgeometry_under_test@@@Z 3502abd0 f i livingentity.obj
 0001:00029bf0       ?FindClosestPoint@CGeometry@@UAEHPAUgeom_world_data@@AAH1ABU?$Vec3_tpl@M@@2PAU3@H@Z 3502abf0 f i livingentity.obj
 0001:00029bf0       ?PreparePolygon@CGeometry@@UAEHPAUcoord_plane@primitives@@HHPAUgeometry_under_test@@AAPAU?$Vec2_tpl@M@@AAPAH3@Z 3502abf0 f i livingentity.obj
 0001:00029bf0       ?PreparePolyline@CGeometry@@UAEHPAUcoord_plane@primitives@@HHPAUgeometry_under_test@@AAPAU?$Vec2_tpl@M@@AAPAH3@Z 3502abf0 f i livingentity.obj
 0001:00029c00       ?DrawWireframe@CGeometry@@UAEXPAUIPhysRenderer@@PAUgeom_world_data@@HH@Z 3502ac00 f i livingentity.obj
 0001:00029c40       ?CalculateBuoyancy@CGeometry@@UAEMPBUplane@primitives@@PBUgeom_world_data@@AAU?$Vec3_tpl@M@@@Z 3502ac40 f i livingentity.obj
 0001:00029c60       ?CalculateMediumResistance@CGeometry@@UAEXPBUplane@primitives@@PBUgeom_world_data@@AAU?$Vec3_tpl@M@@2@Z 3502ac60 f i livingentity.obj
 0001:00029c90       ?GetNormal@CGeometry@@UAE?AU?$Vec3_tpl@M@@HABU2@@Z 3502ac90 f i livingentity.obj
 0001:00029cc0       ?GetCenter@CGeometry@@UAE?AU?$Vec3_tpl@M@@XZ 3502acc0 f i livingentity.obj
 0001:00029ce0       ?Lock@CGeometry@@UAEXH@Z   3502ace0 f i livingentity.obj
 0001:00029d50       ?Unlock@CGeometry@@UAEXH@Z 3502ad50 f i livingentity.obj
 0001:00029d90       ??_GCGeometry@@UAEPAXI@Z   3502ad90 f i livingentity.obj
 0001:00029d90       ??_ECGeometry@@UAEPAXI@Z   3502ad90 f i livingentity.obj
 0001:00029dd0       ??1CCylinderGeom@@UAE@XZ   3502add0 f i livingentity.obj
 0001:00029dd0       ??1CRayGeom@@UAE@XZ        3502add0 f i livingentity.obj
 0001:00029dd0       ??1CCapsuleGeom@@UAE@XZ    3502add0 f i livingentity.obj
 0001:00029e00       ?GetSleepSpeedChange@CPhysicalEntity@@UAEXHAAU?$Vec3_tpl@M@@0@Z 3502ae00 f i livingentity.obj
 0001:00029e30       ?GetMatId@CPhysicalEntity@@QAEHHH@Z 3502ae30 f i livingentity.obj
 0001:00029ec0       ?CheckAreas@CPhysicalWorld@@QAEHPAVCPhysicalEntity@@AAU?$Vec3_tpl@M@@PAUpe_params_buoyancy@@HABU3@H@Z 3502aec0 f i livingentity.obj
 0001:00029f60       ?AlertNeighbourhoodND@CLivingEntity@@UAEXH@Z 3502af60 f i livingentity.obj
 0001:00029fa0       ?GetContactMatrix@CLivingEntity@@UAEXABU?$Vec3_tpl@M@@HAAU?$Matrix33_tpl@M@@@Z 3502afa0 f i livingentity.obj
 0001:00029fe0       ?EncodeVec6b@@YA?AU?$Vec3_tpl@F@@ABU?$Vec3_tpl@M@@@Z 3502afe0 f i livingentity.obj
 0001:0002a0d0       ?DecodeVec6b@@YA?AU?$Vec3_tpl@M@@ABU?$Vec3_tpl@F@@@Z 3502b0d0 f i livingentity.obj
 0001:0002a120       ?EncodeVec4b@@YA?AUvec4b@@ABU?$Vec3_tpl@M@@@Z 3502b120 f i livingentity.obj
 0001:0002a230       ?DecodeVec4b@@YA?AU?$Vec3_tpl@M@@ABUvec4b@@@Z 3502b230 f i livingentity.obj
 0001:0002a2c0       ??_GCLivingEntity@@UAEPAXI@Z 3502b2c0 f i livingentity.obj
 0001:0002a2c0       ??_ECLivingEntity@@UAEPAXI@Z 3502b2c0 f i livingentity.obj
 0001:0002a2f0       ?Awake@CLivingEntity@@UAEHHH@Z 3502b2f0 f   livingentity.obj
 0001:0002a3a0       ?GetStateSnapshot@CLivingEntity@@UAEHV?$CSerializeWrapper@UISerialize@@@@MH@Z 3502b3a0 f   livingentity.obj
 0001:0002a4a0       ?GetMaxTimeStep@CLivingEntity@@UAEMM@Z 3502b4a0 f   livingentity.obj
 0001:0002a4f0       ?CalcEnergy@CLivingEntity@@UAEMM@Z 3502b4f0 f   livingentity.obj
 0001:0002a640       ?Step_HandleWasFlying@CLivingEntity@@QAEXAAU?$Vec3_tpl@M@@AAHABU2@H@Z 3502b640 f   livingentity.obj
 0001:0002ab50       ??$OnEvent@UEventPhysBBoxOverlap@@@CPhysicalWorld@@QAEHIPAUEventPhysBBoxOverlap@@PAPAU1@@Z 3502bb50 f i livingentity.obj
 0001:0002abe0       ??$OnEvent@UEventPhysCollision@@@CPhysicalWorld@@QAEHIPAUEventPhysCollision@@PAPAU1@@Z 3502bbe0 f i livingentity.obj
 0001:0002ac90       ??$OnEvent@UEventPhysPostStep@@@CPhysicalWorld@@QAEHIPAUEventPhysPostStep@@PAPAU1@@Z 3502bc90 f i livingentity.obj
 0001:0002ad60       ?validate@pe_player_dimensions@@QAE_NPBDPAUILog@@ABU?$Vec3_tpl@M@@PAUIPhysRenderer@@PAXHH@Z 3502bd60 f i livingentity.obj
 0001:0002b040       ?validate@pe_action_move@@QAE_NPBDPAUILog@@ABU?$Vec3_tpl@M@@PAUIPhysRenderer@@PAXHH@Z 3502c040 f i livingentity.obj
 0001:0002b280       ?GetType@CRigidEntity@@UBE?AW4pe_type@@XZ 3502c280 f i rigidentity.obj
 0001:0002b280       ?GetType@CSingleBoxTree@@UAEHXZ 3502c280 f i livingentity.obj
 0001:0002b280       ?GetType@CHeightfield@@UAEHXZ 3502c280 f i waterman.obj
 0001:0002b290       ?SetGeomConvex@CSingleBoxTree@@UAEXXZ 3502c290 f i livingentity.obj
 0001:0002b2a0       ?MaxPrimsInNode@CSingleBoxTree@@UAEHXZ 3502c2a0 f i livingentity.obj
 0001:0002b2b0       ?GetNodeContentsIdx@CSingleBoxTree@@UAEHHAAH@Z 3502c2b0 f i livingentity.obj
 0001:0002b2d0       ??0CCylinderGeom@@QAE@XZ   3502c2d0 f i livingentity.obj
 0001:0002b330       ?GetType@CParticleEntity@@UBE?AW4pe_type@@XZ 3502c330 f i particleentity.obj
 0001:0002b330       ?GetType@CVoxelBV@@UAEHXZ  3502c330 f i geoman.obj
 0001:0002b330       ?GetType@CCylinderGeom@@UAEHXZ 3502c330 f i livingentity.obj
 0001:0002b340       ?GetBBox@CCylinderGeom@@UAEXPAUbox@primitives@@@Z 3502c340 f i livingentity.obj
 0001:0002b350       ?GetPrimitive@CCylinderGeom@@UAEHHPAUprimitive@primitives@@@Z 3502c350 f i livingentity.obj
 0001:0002b370       ?SetData@CCylinderGeom@@UAEXPBUprimitive@primitives@@@Z 3502c370 f i livingentity.obj
 0001:0002b380       ?GetCenter@CCylinderGeom@@UAE?AU?$Vec3_tpl@M@@XZ 3502c380 f i livingentity.obj
 0001:0002b380       ?GetCenter@CSphereGeom@@UAE?AU?$Vec3_tpl@M@@XZ 3502c380 f i physicalentity.obj
 0001:0002b3a0       ?GetSizeFast@CCylinderGeom@@UAEHXZ 3502c3a0 f i livingentity.obj
 0001:0002b3b0       ?GetVolume@CCylinderGeom@@UAEMXZ 3502c3b0 f i livingentity.obj
 0001:0002b3c0       ??0CCapsuleGeom@@QAE@XZ    3502c3c0 f i livingentity.obj
 0001:0002b420       ?SetData@CCapsuleGeom@@UAEXPBUprimitive@primitives@@@Z 3502c420 f i livingentity.obj
 0001:0002b430       ?PreparePrimitive@CCapsuleGeom@@UAEHPAUgeom_world_data@@AAPAUprimitive@primitives@@H@Z 3502c430 f i livingentity.obj
 0001:0002b450       ?GetVolume@CCapsuleGeom@@UAEMXZ 3502c450 f i livingentity.obj
 0001:0002b490       ??_GCCapsuleGeom@@UAEPAXI@Z 3502c490 f i livingentity.obj
 0001:0002b490       ??_ECCylinderGeom@@UAEPAXI@Z 3502c490 f i livingentity.obj
 0001:0002b490       ??_GCCylinderGeom@@UAEPAXI@Z 3502c490 f i livingentity.obj
 0001:0002b490       ??_ECRayGeom@@UAEPAXI@Z    3502c490 f i livingentity.obj
 0001:0002b490       ??_ECCapsuleGeom@@UAEPAXI@Z 3502c490 f i livingentity.obj
 0001:0002b490       ??_GCRayGeom@@UAEPAXI@Z    3502c490 f i livingentity.obj
 0001:0002b4e0       ??0CRayGeom@@QAE@XZ        3502c4e0 f i livingentity.obj
 0001:0002b540       ?GetBVTree@CCylinderGeom@@UAEPAVCBVTree@@XZ 3502c540 f i livingentity.obj
 0001:0002b540       ?GetBVTree@CRayGeom@@UAEPAVCBVTree@@XZ 3502c540 f i livingentity.obj
 0001:0002b550       ?GetPrimitive@CRayGeom@@UAEHHPAUprimitive@primitives@@@Z 3502c550 f i livingentity.obj
 0001:0002b590       ?GetData@CSphereGeom@@UAEPBUprimitive@primitives@@XZ 3502c590 f i physicalentity.obj
 0001:0002b590       ?GetData@CRayGeom@@UAEPBUprimitive@primitives@@XZ 3502c590 f i livingentity.obj
 0001:0002b590       ?GetData@CCylinderGeom@@UAEPBUprimitive@primitives@@XZ 3502c590 f i livingentity.obj
 0001:0002b590       ?GetData@CBoxGeom@@UAEPBUprimitive@primitives@@XZ 3502c590 f i physicalentity.obj
 0001:0002b5a0       ?GetSizeFast@CRayGeom@@UAEHXZ 3502c5a0 f i livingentity.obj
 0001:0002b5b0       ?GetCenter@CRayGeom@@UAE?AU?$Vec3_tpl@M@@XZ 3502c5b0 f i livingentity.obj
 0001:0002b620       ?SetData@CRayGeom@@UAEXPBUprimitive@primitives@@@Z 3502c620 f i livingentity.obj
 0001:0002b710       ?PrepareForRayTest@CRayGeom@@UAEXM@Z 3502c710 f i livingentity.obj
 0001:0002b7d0       ??0CLivingEntity@@QAE@PAVCPhysicalWorld@@@Z 3502c7d0 f   livingentity.obj
 0001:0002bdb0       ?UnprojectionNeeded@CLivingEntity@@QBEMABU?$Vec3_tpl@M@@ABU?$Quat_tpl@M@@MM0HAAU2@H@Z 3502cdb0 f   livingentity.obj
 0001:0002ce10       ?SetParams@CLivingEntity@@UAEHPAUpe_params@@H@Z 3502de10 f   livingentity.obj
 0001:0002dd80       ?GetStatus@CLivingEntity@@UBEHPAUpe_status@@@Z 3502ed80 f   livingentity.obj
 0001:0002e720       ?Action@CLivingEntity@@UAEHPAUpe_action@@H@Z 3502f720 f   livingentity.obj
 0001:0002ed40       ?GetStateSnapshot@CLivingEntity@@UAEHAAVCStream@@MH@Z 3502fd40 f   livingentity.obj
 0001:0002f090       ?SetStateFromSnapshot@CLivingEntity@@UAEHV?$CSerializeWrapper@UISerialize@@@@H@Z 35030090 f   livingentity.obj
 0001:0002f2f0       ?AddLegsImpulse@CLivingEntity@@QAEXABU?$Vec3_tpl@M@@0_N@Z 350302f0 f   livingentity.obj
 0001:0002f7b0       ?RegisterContact@CLivingEntity@@QAEXABU?$Vec3_tpl@M@@00PAVCPhysicalEntity@@HHMHH@Z 350307b0 f   livingentity.obj
 0001:0002feb0       ?RegisterUnprojContact@CLivingEntity@@QAEXABUle_contact@@@Z 35030eb0 f   livingentity.obj
 0001:0002ff90       ?ComputeBBox@CLivingEntity@@UAEXPAU?$Vec3_tpl@M@@H@Z 35030f90 f   livingentity.obj
 0001:00030170       ?ComputeBBoxLE@CLivingEntity@@QAEXABU?$Vec3_tpl@M@@PAU2@PAUcoord_block_BBox@@@Z 35031170 f   livingentity.obj
 0001:00030250       ?RegisterContacts@CLivingEntity@@UAEHMH@Z 35031250 f   livingentity.obj
 0001:000307c0       ?GetRigidBody@CLivingEntity@@UAEPAVRigidBody@@HH@Z 350317c0 f   livingentity.obj
 0001:00030af0       ?OnContactResolved@CLivingEntity@@UAEXPAUentity_contact@@HH@Z 35031af0 f   livingentity.obj
 0001:00030d40       ?DrawHelperInformation@CLivingEntity@@UAEXPAUIPhysRenderer@@H@Z 35031d40 f   livingentity.obj
 0001:00030d70       ?Step_HandleFlying@CLivingEntity@@QAEXAAU?$Vec3_tpl@M@@ABU2@H1MM@Z 35031d70 f   livingentity.obj
 0001:000310c0       ?ShootRayDown@CLivingEntity@@QAEMPAUle_precomp_entity@@HPAUle_precomp_part@@ABU?$Vec3_tpl@M@@AAU4@M_N44@Z 350320c0 f   livingentity.obj
 0001:00032770       ?SyncWithGroundCollider@CLivingEntity@@QAE?AU?$Vec3_tpl@M@@M@Z 35033770 f   livingentity.obj
 0001:000334d0       ?Step@CLivingEntity@@UAEHM@Z 350344d0 f   livingentity.obj
 0001:0003bd90       ?Update@CLivingEntity@@UAEHMM@Z 3503cd90 f   livingentity.obj
 0001:0003c260       ??1CParticleEntity@@UAE@XZ 3503d260 f   particleentity.obj
 0001:0003c2d0       ?GetRigidBodyData@CPhysicalEntity@@UAEPAVRigidBody@@PAV2@H@Z 3503d2d0 f i particleentity.obj
 0001:0003c2f0       ?ExitScope_Alloc@CDummyMemReplay@@UAEXIII@Z 3503d2f0 f i articulatedentity.obj
 0001:0003c2f0       ?AddContext@CDummyMemReplay@@UAEXHIPBD@Z 3503d2f0 f i articulatedentity.obj
 0001:0003c2f0       ?RemapForeignIdx@CGeometry@@UAEXPAH0H@Z 3503d2f0 f i livingentity.obj
 0001:0003c2f0       ?RegisterFixedAddressRange@CDummyMemReplay@@UAEXPAXIPBD@Z 3503d2f0 f i articulatedentity.obj
 0001:0003c2f0       ?AllocUsage@CDummyMemReplay@@UAEXW4Class@EMemReplayAllocClass@@II@Z 3503d2f0 f i articulatedentity.obj
 0001:0003c2f0       ?ApplyVolumetricPressure@CPhysicalEntity@@UAEXABU?$Vec3_tpl@M@@MM@Z 3503d2f0 f i articulatedentity.obj
 0001:0003c2f0       ?AppendVertices@CGeometry@@UAEXPAU?$Vec3_tpl@M@@PAHH@Z 3503d2f0 f i livingentity.obj
 0001:0003c2f0       ?GetContactMatrix@CPhysicalEntity@@UAEXABU?$Vec3_tpl@M@@HAAU?$Matrix33_tpl@M@@@Z 3503d2f0 f i particleentity.obj
 0001:0003c2f0       ?GetSpatialContactMatrix@CPhysicalEntity@@UAEXABU?$Vec3_tpl@M@@HQAY05M@Z 3503d2f0 f i articulatedentity.obj
 0001:0003c300       ?GetMass@CParticleEntity@@UAEMH@Z 3503d300 f i particleentity.obj
 0001:0003c310       ?AlertNeighbourhoodND@CParticleEntity@@UAEXH@Z 3503d310 f i particleentity.obj
 0001:0003c340       ?StartStep@CParticleEntity@@UAEXM@Z 3503d340 f   particleentity.obj
 0001:0003c360       ?GetMemoryStatistics@CParticleEntity@@UBEXPAVICrySizer@@@Z 3503d360 f   particleentity.obj
 0001:0003c3a0       ?Init@SRWIParams@IPhysicalWorld@@QAEABU12@ABU?$Vec3_tpl@M@@0HIABUSCollisionClass@@PAUray_hit@@HPAPAUIPhysicalEntity@@HPAXHPAUray_hit_cached@@@Z 3503d3a0 f i particleentity.obj
 0001:0003c440       ?GetFriction@CPhysicalWorld@@QAEMHHH@Z 3503d440 f i particleentity.obj
 0001:0003c490       ?ComputeBBox@CParticleEntity@@UAEXPAU?$Vec3_tpl@M@@H@Z 3503d490 f i particleentity.obj
 0001:0003c530       ?Step@CParticleEntity@@UAEHM@Z 3503d530 f i particleentity.obj
 0001:0003c550       ??0CParticleEntity@@QAE@PAVCPhysicalWorld@@@Z 3503d550 f   particleentity.obj
 0001:0003c890       ??_ECParticleEntity@@UAEPAXI@Z 3503d890 f i particleentity.obj
 0001:0003c890       ??_GCParticleEntity@@UAEPAXI@Z 3503d890 f i particleentity.obj
 0001:0003c8c0       ?GetParams@CParticleEntity@@UBEHPAUpe_params@@@Z 3503d8c0 f   particleentity.obj
 0001:0003cab0       ?GetStateSnapshot@CParticleEntity@@UAEHAAVCStream@@MH@Z 3503dab0 f   particleentity.obj
 0001:0003cb30       ?Awake@CParticleEntity@@UAEHHH@Z 3503db30 f   particleentity.obj
 0001:0003cb90       ?IsAwake@CParticleEntity@@UBEHH@Z 3503db90 f   particleentity.obj
 0001:0003ccc0       ?GetMaxTimeStep@CParticleEntity@@UAEMM@Z 3503dcc0 f   particleentity.obj
 0001:0003cd10       ??0pe_params_particle@@QAE@XZ 3503dd10 f i particleentity.obj
 0001:0003ce30       ?validate@pe_params_particle@@QAE_NPBDPAUILog@@ABU?$Vec3_tpl@M@@PAUIPhysRenderer@@PAXHH@Z 3503de30 f i particleentity.obj
 0001:0003d3d0       ?GetStateSnapshot@CParticleEntity@@UAEHV?$CSerializeWrapper@UISerialize@@@@MH@Z 3503e3d0 f   particleentity.obj
 0001:0003d4b0       ?SetStateFromSnapshot@CParticleEntity@@UAEHV?$CSerializeWrapper@UISerialize@@@@H@Z 3503e4b0 f   particleentity.obj
 0001:0003d660       ?GetStatus@CParticleEntity@@UBEHPAUpe_status@@@Z 3503e660 f   particleentity.obj
 0001:0003da00       ?RayTrace@CParticleEntity@@UAEHAAUSRayTraceRes@@@Z 3503ea00 f   particleentity.obj
 0001:0003ded0       ?DrawHelperInformation@CParticleEntity@@UAEXPAUIPhysRenderer@@H@Z 3503eed0 f   particleentity.obj
 0001:0003ea30       ?SetParams@CParticleEntity@@UAEHPAUpe_params@@H@Z 3503fa30 f   particleentity.obj
 0001:0003f760       ?Action@CParticleEntity@@UAEHPAUpe_action@@H@Z 35040760 f   particleentity.obj
 0001:0003fbf0       ?DoStep@CParticleEntity@@UAEHMH@Z 35040bf0 f   particleentity.obj
 0001:000452f0       ?GetEntity@CPhysArea@@UAEPAVCPhysicalEntity@@XZ 350462f0 f   physarea.obj
 0001:00045300       ?GetParams@CPhysArea@@UBEHPAUpe_params@@@Z 35046300 f   physarea.obj
 0001:000453e0       ?GetMemoryStatistics@CPhysArea@@UBEXPAVICrySizer@@@Z 350463e0 f   physarea.obj
 0001:00045710       ?GetNextArea@CPhysicalWorld@@UAEPAUIPhysicalEntity@@PAU2@@Z 35046710 f   physarea.obj
 0001:000457a0       ??$SignalEvent@UEventPhysAreaChange@@@CPhysicalWorld@@QAEHPAUEventPhysAreaChange@@H@Z 350467a0 f i physarea.obj
 0001:00045810       ??$SignalEvent@UEventPhysArea@@@CPhysicalWorld@@QAEHPAUEventPhysArea@@H@Z 35046810 f i physarea.obj
 0001:00045880       ??_EIPhysicalEntity@@UAEPAXI@Z 35046880 f i physarea.obj
 0001:00045880       ??_GCPhysicalStub@@UAEPAXI@Z 35046880 f i physarea.obj
 0001:00045880       ??_GIPhysicalEntity@@UAEPAXI@Z 35046880 f i physarea.obj
 0001:00045880       ??_ECPhysicalStub@@UAEPAXI@Z 35046880 f i physarea.obj
 0001:000458b0       ?GetEntityFast@CPhysicalPlaceholder@@UAEPAVCPhysicalEntity@@XZ 350468b0 f i physarea.obj
 0001:000458c0       ?alloc@StandardAlloc@NAlloc@@SAPAXAAI_NH@Z 350468c0 f i physarea.obj
 0001:00045940       ?CircleRandomPoint@@YA?AU?$Vec2_tpl@M@@W4EGeomForm@@M@Z 35046940 f i physarea.obj
 0001:000459f0       ?AddGeometry@CPhysicalStub@@UAEHPAUphys_geometry@@PAUpe_geomparams@@HH@Z 350469f0 f i physarea.obj
 0001:00045a00       ?ComputeExtent@CPhysicalStub@@UAEMAAUGeomQuery@@W4EGeomForm@@@Z 35046a00 f i physarea.obj
 0001:00045a10       ?SetStateFromSnapshot@CPhysicalEntity@@UAEHAAVCStream@@H@Z 35046a10 f i physicalentity.obj
 0001:00045a10       ?DoStep@CPhysicalStub@@UAEHMH@Z 35046a10 f i physarea.obj
 0001:00045a10       ?Awake@CPhysicalEntity@@UAEHHH@Z 35046a10 f i physicalentity.obj
 0001:00045a10       ?Action@CPhysicalStub@@UAEHPAUpe_action@@H@Z 35046a10 f i physarea.obj
 0001:00045a10       ?SetStateFromSnapshot@CRopeEntity@@UAEHAAVCStream@@H@Z 35046a10 f i ropeentity.obj
 0001:00045a10       ?SetStateFromSnapshot@CLivingEntity@@UAEHAAVCStream@@H@Z 35046a10 f i livingentity.obj
 0001:00045a10       ?SetParams@CPhysicalStub@@UAEHPAUpe_params@@H@Z 35046a10 f i physarea.obj
 0001:00045a10       ?SetStateFromSnapshot@CPhysicalStub@@UAEHAAVCStream@@H@Z 35046a10 f i physarea.obj
 0001:00045a10       ?CheckSelfCollision@CRigidEntity@@UAEHHH@Z 35046a10 f i rigidentity.obj
 0001:00045a10       ?SetStateFromSnapshot@CSoftEntity@@UAEHAAVCStream@@H@Z 35046a10 f i softentity.obj
 0001:00045a10       ?SerializeGeometries@CPhysicalWorld@@UAEHPBDH@Z 35046a10 f i physicalworld.obj
 0001:00045a10       ?SetStateFromSnapshot@CParticleEntity@@UAEHAAVCStream@@H@Z 35046a10 f i particleentity.obj
 0001:00045a10       ?SetStateFromSnapshot@CPhysicalStub@@UAEHV?$CSerializeWrapper@UISerialize@@@@H@Z 35046a10 f i physarea.obj
 0001:00045a10       ?RegisterContacts@CPhysicalEntity@@UAEHMH@Z 35046a10 f i particleentity.obj
 0001:00045a10       ?HasConstraintContactsWith@CPhysicalEntity@@UBEHPBV1@H@Z 35046a10 f i livingentity.obj
 0001:00045a10       ?SerializeWorld@CPhysicalWorld@@UAEHPBDH@Z 35046a10 f i physicalworld.obj
 0001:00045a10       ?SetStateFromSnapshot@CArticulatedEntity@@UAEHAAVCStream@@H@Z 35046a10 f i articulatedentity.obj
 0001:00045a20       ?SetStateFromTypedSnapshot@CPhysicalStub@@UAEHV?$CSerializeWrapper@UISerialize@@@@HH@Z 35046a20 f i physarea.obj
 0001:00045a20       ?GetStateSnapshotTxt@CPhysicalStub@@UAEHPADHM@Z 35046a20 f i physarea.obj
 0001:00045a20       ?GetFeature@CGeometry@@UAEHHHPAU?$Vec3_tpl@M@@@Z 35046a20 f i livingentity.obj
 0001:00045a20       ?GetStateSnapshot@CPhysicalStub@@UAEHV?$CSerializeWrapper@UISerialize@@@@MH@Z 35046a20 f i physarea.obj
 0001:00045a20       ?GetStateSnapshot@CPhysicalEntity@@UAEHAAVCStream@@MH@Z 35046a20 f i physicalentity.obj
 0001:00045a20       ?GetStateSnapshot@CPhysicalStub@@UAEHAAVCStream@@MH@Z 35046a20 f i physarea.obj
 0001:00045a20       ?Boxify@CGeometry@@UAEHPAUbox@primitives@@HABUSBoxificationParams@IGeometry@@@Z 35046a20 f i livingentity.obj
 0001:00045a30       ?GetRandomPos@CPhysicalStub@@UAEXAAURandomPos@@AAUGeomQuery@@W4EGeomForm@@@Z 35046a30 f i physarea.obj
 0001:00045a60       ??1CPhysArea@@UAE@XZ       35046a60 f   physarea.obj
 0001:00045ae0       ?GetEntityFast@CPhysArea@@UAEPAVCPhysicalEntity@@XZ 35046ae0 f i physarea.obj
 0001:00045af0       ?AddRef@CPhysArea@@UAEHXZ  35046af0 f i physarea.obj
 0001:00045b10       ?Release@CPhysArea@@UAEHXZ 35046b10 f i physarea.obj
 0001:00045b30       ?GetWorld@CPhysArea@@UBEPAUIPhysicalWorld@@XZ 35046b30 f i physarea.obj
 0001:00045b40       ?IsAreaNonWater@@YAHPAVCPhysArea@@@Z 35046b40 f   physarea.obj
 0001:00045bc0       ?IsAreaGravity@@YAHPAVCPhysArea@@@Z 35046bc0 f   physarea.obj
 0001:00045c00       ?SetWaterMat@CPhysicalWorld@@UAEXH@Z 35046c00 f   physarea.obj
 0001:00045c60       ??$move_init@M@NArray@@YAXPAM0I@Z 35046c60 f i physarea.obj
 0001:00045cf0       ??0CRayGeom@@QAE@ABU?$Vec3_tpl@M@@0@Z 35046cf0 f i physarea.obj
 0001:00045e30       ?GetRandomPart@GeomQuery@@QBEHXZ 35046e30 f i physarea.obj
 0001:00045f60       ??_GCPhysArea@@UAEPAXI@Z   35046f60 f i physarea.obj
 0001:00045f60       ??_ECPhysArea@@UAEPAXI@Z   35046f60 f i physarea.obj
 0001:00045f90       ?DrawHelperInformation@CPhysArea@@UAEXPAUIPhysRenderer@@H@Z 35046f90 f   physarea.obj
 0001:00046f20       ?RepositionArea@CPhysicalWorld@@QAEXPAVCPhysArea@@@Z 35047f20 f   physarea.obj
 0001:00047030       ?RemoveArea@CPhysicalWorld@@UAEXPAUIPhysicalEntity@@@Z 35048030 f   physarea.obj
 0001:000472a0       ?resize_raw@?$SmallDynStorage@MHUStandardAlloc@NAlloc@@@NArray@@QAEXHH_N@Z 350482a0 f i physarea.obj
 0001:000473f0       ?set_size@?$SmallDynStorage@MHUStandardAlloc@NAlloc@@@NArray@@QAEXH@Z 350483f0 f i physarea.obj
 0001:00047470       ?destroy@?$DynArray@UGeomQuery@@HU?$SmallDynStorage@UGeomQuery@@HUStandardAlloc@NAlloc@@@NArray@@@@KAXU?$Array@UGeomQuery@@HU?$ArrayStorage@UGeomQuery@@H@NArray@@@@@Z 35048470 f i physarea.obj
 0001:000474a0       ?set_size@?$SmallDynStorage@UGeomQuery@@HUStandardAlloc@NAlloc@@@NArray@@QAEXH@Z 350484a0 f i physarea.obj
 0001:00047530       ?expand_raw@?$DynArray@MHU?$SmallDynStorage@MHUStandardAlloc@NAlloc@@@NArray@@@@IAEPAMPAMH@Z 35048530 f i physarea.obj
 0001:000475b0       ?findroots@?$polynomial_tpl@N$02@@QBEHNNPANHH_N@Z 350485b0 f i physarea.obj
 0001:000481c0       ??0EventPhysArea@@QAE@XZ   350491c0 f i physarea.obj
 0001:00048270       ??0CPhysArea@@QAE@PAVCPhysicalWorld@@@Z 35049270 f   physarea.obj
 0001:00048520       ?FindSplineClosestPt@CPhysArea@@QBEMABU?$Vec3_tpl@M@@AAHAAM@Z 35049520 f   physarea.obj
 0001:00049020       ?FindSplineClosestPt@CPhysArea@@QBEHABU?$Vec3_tpl@M@@0AAU2@1@Z 3504a020 f   physarea.obj
 0001:0004b1b0       ?SetParams@CPhysArea@@UAEHPAUpe_params@@H@Z 3504c1b0 f   physarea.obj
 0001:0004c790       ?AddArea@CPhysicalWorld@@UAEPAUIPhysicalEntity@@PAU?$Vec3_tpl@M@@HMMABU3@ABU?$Quat_tpl@M@@M1PAHH0@Z 3504d790 f   physarea.obj
 0001:0004e220       ?AddArea@CPhysicalWorld@@UAEPAUIPhysicalEntity@@PAUIGeometry@@ABU?$Vec3_tpl@M@@ABU?$Quat_tpl@M@@M@Z 3504f220 f   physarea.obj
 0001:0004e930       ?AddArea@CPhysicalWorld@@UAEPAUIPhysicalEntity@@PAU?$Vec3_tpl@M@@HMABU3@ABU?$Quat_tpl@M@@M@Z 3504f930 f   physarea.obj
 0001:0004f010       ?AddGlobalArea@CPhysicalWorld@@UAEPAUIPhysicalEntity@@XZ 35050010 f   physarea.obj
 0001:0004f150       ?destroy@?$DynArray@UGeomQuery@@HU?$SmallDynStorage@UGeomQuery@@HUStandardAlloc@NAlloc@@@NArray@@@@IAEXXZ 35050150 f i physarea.obj
 0001:0004f180       ?ApplyParams@CPhysArea@@QBEHABU?$Vec3_tpl@M@@AAU2@0PAUpe_params_buoyancy@@HHAAHPAUIPhysicalEntity@@@Z 35050180 f   physarea.obj
 0001:00051130       ?CheckPoint@CPhysArea@@QBEHABU?$Vec3_tpl@M@@M@Z 35052130 f   physarea.obj
 0001:000516a0       ?RayTraceInternal@CPhysArea@@QAEHABU?$Vec3_tpl@M@@0PAUray_hit@@PAUpe_params_pos@@@Z 350526a0 f   physarea.obj
 0001:000526c0       ?CheckAreas@CPhysicalWorld@@UAEHABU?$Vec3_tpl@M@@AAU2@PAUpe_params_buoyancy@@HH0PAUIPhysicalEntity@@H@Z 350536c0 f   physarea.obj
 0001:00052c20       ??1?$DynArray@MHU?$SmallDynStorage@MHUStandardAlloc@NAlloc@@@NArray@@@@QAE@XZ 35053c20 f i physarea.obj
 0001:00052c50       ??1?$DynArray@UGeomQuery@@HU?$SmallDynStorage@UGeomQuery@@HUStandardAlloc@NAlloc@@@NArray@@@@QAE@XZ 35053c50 f i physarea.obj
 0001:00052cb0       ??0?$DynArray@MHU?$SmallDynStorage@MHUStandardAlloc@NAlloc@@@NArray@@@@QAE@ABU0@@Z 35053cb0 f i physarea.obj
 0001:00052d40       ??_GGeomQuery@@QAEPAXI@Z   35053d40 f i physarea.obj
 0001:00052d90       ??0GeomQuery@@QAE@XZ       35053d90 f i physarea.obj
 0001:00052e30       ??$move_init@UGeomQuery@@@NArray@@YAXPAUGeomQuery@@0I@Z 35053e30 f i physarea.obj
 0001:00052fc0       ?resize_raw@?$SmallDynStorage@UGeomQuery@@HUStandardAlloc@NAlloc@@@NArray@@QAEXHH_N@Z 35053fc0 f i physarea.obj
 0001:00053120       ?expand_raw@?$DynArray@UGeomQuery@@HU?$SmallDynStorage@UGeomQuery@@HUStandardAlloc@NAlloc@@@NArray@@@@IAEPAUGeomQuery@@PAU2@H@Z 35054120 f i physarea.obj
 0001:000531b0       ?clear@?$DynArray@UGeomQuery@@HU?$SmallDynStorage@UGeomQuery@@HUStandardAlloc@NAlloc@@@NArray@@@@QAEXXZ 350541b0 f i physarea.obj
 0001:00053330       ?SetOwner@GeomQuery@@QAE_NPBXW4EGeomForm@@@Z 35054330 f i physarea.obj
 0001:000533b0       ??0?$DynArray@UGeomQuery@@HU?$SmallDynStorage@UGeomQuery@@HUStandardAlloc@NAlloc@@@NArray@@@@QAE@ABU0@@Z 350543b0 f i physarea.obj
 0001:00053430       ?GetRandomPos@CPhysArea@@UBEXAAURandomPos@@AAUGeomQuery@@W4EGeomForm@@@Z 35054430 f   physarea.obj
 0001:00053be0       ?GetStatus@CPhysArea@@UBEHPAUpe_status@@@Z 35054be0 f   physarea.obj
 0001:00054790       ?resize@?$DynArray@UGeomQuery@@HU?$SmallDynStorage@UGeomQuery@@HUStandardAlloc@NAlloc@@@NArray@@@@QAEXH@Z 35055790 f i physarea.obj
 0001:00054940       ??0GeomQuery@@QAE@ABU0@@Z  35055940 f i physarea.obj
 0001:00054980       ?init@?$DynArray@UGeomQuery@@HU?$SmallDynStorage@UGeomQuery@@HUStandardAlloc@NAlloc@@@NArray@@@@KAPAUGeomQuery@@U?$Array@UGeomQuery@@HU?$ArrayStorage@UGeomQuery@@H@NArray@@@@PBU2@@Z 35055980 f i physarea.obj
 0001:000549f0       ?ComputeExtent@CPhysArea@@UBEMAAUGeomQuery@@W4EGeomForm@@@Z 350559f0 f   physarea.obj
 0001:00054bb0       ?WriteBBox@CPhysicalEntity@@QAEXPAU?$Vec3_tpl@M@@@Z 35055bb0 f i physicalentity.obj
 0001:00054c10       ?CleanupGlobalState@CPhysicalEntity@@SAXXZ 35055c10 f   physicalentity.obj
 0001:00054c80       ?UpdatePartIdmatBreakable@CPhysicalEntity@@QAEXHH@Z 35055c80 f   physicalentity.obj
 0001:00054fa0       ?RemoveCollider@CPhysicalEntity@@UAEHPAV1@_N@Z 35055fa0 f   physicalentity.obj
 0001:00055030       ?GetMemoryStatistics@CPhysicalEntity@@UBEXPAVICrySizer@@@Z 35056030 f   physicalentity.obj
 0001:000552e0       ?GetStateSnapshotTxt@CPhysicalEntity@@UAEHPADHM@Z 350562e0 f   physicalentity.obj
 0001:00055310       ?SetStateFromSnapshotTxt@CPhysicalEntity@@UAEXPBDH@Z 35056310 f   physicalentity.obj
 0001:00055340       ??$ReallocateList@USStructuralJoint@@@@YAPAUSStructuralJoint@@AAPAU0@HH_N1@Z 35056340 f i physicalentity.obj
 0001:000553f0       ??$SignalEvent@UEventPhysUpdateMesh@@@CPhysicalWorld@@QAEHPAUEventPhysUpdateMesh@@H@Z 350563f0 f i physicalentity.obj
 0001:00055460       ??$SignalEvent@UEventPhysCreateEntityPart@@@CPhysicalWorld@@QAEHPAUEventPhysCreateEntityPart@@H@Z 35056460 f i physicalentity.obj
 0001:000554d0       ??$SignalEvent@UEventPhysRemoveEntityParts@@@CPhysicalWorld@@QAEHPAUEventPhysRemoveEntityParts@@H@Z 350564d0 f i physicalentity.obj
 0001:00055540       ??$SignalEvent@UEventPhysRevealEntityPart@@@CPhysicalWorld@@QAEHPAUEventPhysRevealEntityPart@@H@Z 35056540 f i physicalentity.obj
 0001:000555b0       ??$SignalEvent@UEventPhysJointBroken@@@CPhysicalWorld@@QAEHPAUEventPhysJointBroken@@H@Z 350565b0 f i physicalentity.obj
 0001:00055620       ??4box@primitives@@QAEAAU01@ABU01@@Z 35056620 f i physicalentity.obj
 0001:00055690       ??1CBoxGeom@@UAE@XZ        35056690 f i physicalentity.obj
 0001:000556c0       ??1CSphereGeom@@UAE@XZ     350566c0 f i physicalentity.obj
 0001:000556f0       ??0CPhysicalEntity@@QAE@PAVCPhysicalWorld@@@Z 350566f0 f   physicalentity.obj
 0001:000558c0       ?GetLastTimeStep@CPhysicalEntity@@UAEMM@Z 350568c0 f i livingentity.obj
 0001:000558c0       ?GetMaxTimeStep@CPhysicalEntity@@UAEMM@Z 350568c0 f i physicalentity.obj
 0001:000558d0       ?AddRef@CPhysicalEntity@@UAEHXZ 350568d0 f   physicalentity.obj
 0001:00055950       ?Release@CPhysicalEntity@@UAEHXZ 35056950 f   physicalentity.obj
 0001:000559d0       ?GetRigidBody@CPhysicalEntity@@UAEPAVRigidBody@@HH@Z 350569d0 f   physicalentity.obj
 0001:00055a40       ?IsPointInside@CPhysicalEntity@@UBEHU?$Vec3_tpl@M@@@Z 35056a40 f   physicalentity.obj
 0001:00055d50       ?AlertNeighbourhoodND@CPhysicalEntity@@UAEXH@Z 35056d50 f   physicalentity.obj
 0001:00056000       ?AddCollider@CPhysicalEntity@@UAEHPAV1@@Z 35057000 f   physicalentity.obj
 0001:00056190       ?FillGeomParams@@YAXAAUpe_geomparams@@AAUgeom@@@Z 35057190 f i physicalentity.obj
 0001:00056220       ?AABB_OBB@Overlap@@YA_NABUAABB@@ABU?$Vec3_tpl@M@@ABU?$OBB_tpl@M@@@Z 35057220 f i physicalentity.obj
 0001:00056780       ?validate@pe_params_pos@@QAE_NPBDPAUILog@@ABU?$Vec3_tpl@M@@PAUIPhysRenderer@@PAXHH@Z 35057780 f i physicalentity.obj
 0001:00056ac0       ?validate@pe_params_bbox@@QAE_NPBDPAUILog@@ABU?$Vec3_tpl@M@@PAUIPhysRenderer@@PAXHH@Z 35057ac0 f i physicalentity.obj
 0001:00056c90       ??0pe_params_part@@QAE@XZ  35057c90 f i physicalentity.obj
 0001:00056d50       ?validate@pe_params_part@@QAE_NPBDPAUILog@@ABU?$Vec3_tpl@M@@PAUIPhysRenderer@@PAXHH@Z 35057d50 f i physicalentity.obj
 0001:00057090       ??0pe_simulation_params@@QAE@XZ 35058090 f i physicalentity.obj
 0001:00057140       ??0pe_params_structural_joint@@QAE@XZ 35058140 f i physicalentity.obj
 0001:00057220       ??4pe_geomparams@@QAEAAU0@ABU0@@Z 35058220 f i physicalentity.obj
 0001:000572b0       ??0pe_params_softbody@@QAE@XZ 350582b0 f i physicalentity.obj
 0001:000573e0       ??0pe_action_add_constraint@@QAE@XZ 350583e0 f i physicalentity.obj
 0001:000574a0       ?validate@pe_geomparams@@QAE_NPBDPAUILog@@ABU?$Vec3_tpl@M@@PAUIPhysRenderer@@PAXHH@Z 350584a0 f i physicalentity.obj
 0001:000578c0       ?ReleasePartPlaceholder@CPhysicalEntity@@QAEPAVCPhysicalPlaceholder@@H@Z 350588c0 f   physicalentity.obj
 0001:000579c0       ?RepositionParts@CPhysicalEntity@@QAEXXZ 350589c0 f   physicalentity.obj
 0001:00057b30       ??0?$Matrix34_tpl@M@@QAE@ABU?$Vec3_tpl@M@@ABU?$Quat_tpl@M@@0@Z 35058b30 f i physicalentity.obj
 0001:00057ca0       ??$OnEvent@UEventPhysUpdateMesh@@@CPhysicalWorld@@QAEHIPAUEventPhysUpdateMesh@@PAPAU1@@Z 35058ca0 f i physicalentity.obj
 0001:00057d40       ??$OnEvent@UEventPhysCreateEntityPart@@@CPhysicalWorld@@QAEHIPAUEventPhysCreateEntityPart@@PAPAU1@@Z 35058d40 f i physicalentity.obj
 0001:00057df0       ??$OnEvent@UEventPhysRemoveEntityParts@@@CPhysicalWorld@@QAEHIPAUEventPhysRemoveEntityParts@@PAPAU1@@Z 35058df0 f i physicalentity.obj
 0001:00057e90       ??$OnEvent@UEventPhysRevealEntityPart@@@CPhysicalWorld@@QAEHIPAUEventPhysRevealEntityPart@@PAPAU1@@Z 35058e90 f i physicalentity.obj
 0001:00057f50       ??$OnEvent@UEventPhysJointBroken@@@CPhysicalWorld@@QAEHIPAUEventPhysJointBroken@@PAPAU1@@Z 35058f50 f i physicalentity.obj
 0001:00057ff0       ??$ReallocateList@Uplane@primitives@@@@YAPAUplane@primitives@@AAPAU01@HH_N1@Z 35058ff0 f i physicalentity.obj
 0001:000580a0       ??$ReallocateList@USPartInfo@@@@YAPAUSPartInfo@@AAPAU0@HH_N1@Z 350590a0 f i physicalentity.obj
 0001:00058140       ??$ReallocateList@Ubox@primitives@@@@YAPAUbox@primitives@@AAPAU01@HH_N1@Z 35059140 f i physicalentity.obj
 0001:00058140       ??$ReallocateList@Ubop_newtri@@@@YAPAUbop_newtri@@AAPAU0@HH_N1@Z 35059140 f i boolean3d.obj
 0001:00058140       ??$ReallocateList@USSkelInfo@@@@YAPAUSSkelInfo@@AAPAU0@HH_N1@Z 35059140 f i physicalentity.obj
 0001:000581e0       ?GetBBox@CBoxGeom@@UAEXPAUbox@primitives@@@Z 350591e0 f i physicalentity.obj
 0001:000581f0       ?GetBVTree@CBoxGeom@@UAEPAVCBVTree@@XZ 350591f0 f i physicalentity.obj
 0001:00058200       ?SetData@CBoxGeom@@UAEXPBUprimitive@primitives@@@Z 35059200 f i physicalentity.obj
 0001:00058210       ?GetCenter@CBoxGeom@@UAE?AU?$Vec3_tpl@M@@XZ 35059210 f i physicalentity.obj
 0001:00058230       ?GetSizeFast@CBoxGeom@@UAEHXZ 35059230 f i physicalentity.obj
 0001:00058240       ?GetVolume@CBoxGeom@@UAEMXZ 35059240 f i physicalentity.obj
 0001:00058250       ?GetPrimitive@CBoxGeom@@UAEHHPAUprimitive@primitives@@@Z 35059250 f i physicalentity.obj
 0001:00058270       ??_ECBoxGeom@@UAEPAXI@Z    35059270 f i physicalentity.obj
 0001:00058270       ??_GCBoxGeom@@UAEPAXI@Z    35059270 f i physicalentity.obj
 0001:000582c0       ??0CSphereGeom@@QAE@XZ     350592c0 f i physicalentity.obj
 0001:00058310       ?GetBBox@CSphereGeom@@UAEXPAUbox@primitives@@@Z 35059310 f i physicalentity.obj
 0001:00058320       ?GetBVTree@CSphereGeom@@UAEPAVCBVTree@@XZ 35059320 f i physicalentity.obj
 0001:00058330       ?GetPrimitive@CSphereGeom@@UAEHHPAUprimitive@primitives@@@Z 35059330 f i physicalentity.obj
 0001:00058360       ?SetData@CSphereGeom@@UAEXPBUprimitive@primitives@@@Z 35059360 f i physicalentity.obj
 0001:00058370       ?GetSizeFast@CSphereGeom@@UAEHXZ 35059370 f i physicalentity.obj
 0001:00058380       ?GetVolume@CSphereGeom@@UAEMXZ 35059380 f i physicalentity.obj
 0001:00058390       ??_GCSphereGeom@@UAEPAXI@Z 35059390 f i physicalentity.obj
 0001:00058390       ??_ECSphereGeom@@UAEPAXI@Z 35059390 f i physicalentity.obj
 0001:000583e0       ??1CPhysicalEntity@@UAE@XZ 350593e0 f   physicalentity.obj
 0001:00058660       ?GetParams@CPhysicalEntity@@UBEHPAUpe_params@@@Z 35059660 f   physicalentity.obj
 0001:00059080       ?AddGeometry@CPhysicalEntity@@UAEHPAUphys_geometry@@PAUpe_geomparams@@HH@Z 3505a080 f   physicalentity.obj
 0001:00059c00       ?RemoveGeometry@CPhysicalEntity@@UAEXHH@Z 3505ac00 f   physicalentity.obj
 0001:0005a2d0       ?RemoveBrokenParent@CPhysicalEntity@@QAEXHH@Z 3505b2d0 f   physicalentity.obj
 0001:0005a490       ?MapHitPointFromParent@CPhysicalEntity@@QAEHHABU?$Vec3_tpl@M@@@Z 3505b490 f   physicalentity.obj
 0001:0005aab0       ?OnContactResolved@CPhysicalEntity@@UAEXPAUentity_contact@@HH@Z 3505bab0 f   physicalentity.obj
 0001:0005bb00       ?TouchesSphere@CPhysicalEntity@@QAEHABU?$Vec3_tpl@M@@M@Z 3505cb00 f   physicalentity.obj
 0001:0005c1f0       ?UpdateDeformablePart@CPhysicalEntity@@QAEXH@Z 3505d1f0 f   physicalentity.obj
 0001:0005d170       ?AllocStructureInfo@CPhysicalEntity@@QAEXXZ 3505e170 f   physicalentity.obj
 0001:0005d230       ?_Assign@?$CryStringT@D@@IAEXPBDI@Z 3505e230 f i physicalentity.obj
 0001:0005d2e0       ??_GCPhysicalEntity@@UAEPAXI@Z 3505e2e0 f i physicalentity.obj
 0001:0005d2e0       ??_ECPhysicalEntity@@UAEPAXI@Z 3505e2e0 f i physicalentity.obj
 0001:0005d310       ?ComputeBBox@CPhysicalEntity@@UAEXPAU?$Vec3_tpl@M@@H@Z 3505e310 f   physicalentity.obj
 0001:0005e280       ?Action@CPhysicalEntity@@UAEHPAUpe_action@@H@Z 3505f280 f   physicalentity.obj
 0001:00060af0       ?OccupiesEntityGridSquare@CPhysicalEntity@@QAE_NABUAABB@@@Z 35061af0 f   physicalentity.obj
 0001:000612c0       ?DrawHelperInformation@CPhysicalEntity@@UAEXPAUIPhysRenderer@@H@Z 350622c0 f   physicalentity.obj
 0001:00063560       ?CapsulizePart@CPhysicalEntity@@QAEHH@Z 35064560 f   physicalentity.obj
 0001:00065540       ?MakeDeformable@CPhysicalEntity@@QAE_NHHM@Z 35066540 f   physicalentity.obj
 0001:00067060       ?UpdateStructure@CPhysicalEntity@@QAEHMPAUpe_explosion@@HU?$Vec3_tpl@M@@@Z 35068060 f   physicalentity.obj
 0001:00075cc0       ?GenerateJoints@CPhysicalEntity@@QAEHXZ 35076cc0 f   physicalentity.obj
 0001:00077870       ?SetSharedSerializeString@?$CSerializeWrapper@UISerialize@@@@QAEAAUSSerializeString@@ABV?$CryStringT@D@@@Z 35078870 f i physicalentity.obj
 0001:000778d0       ?SetParams@CPhysicalEntity@@UAEHPAUpe_params@@H@Z 350788d0 f   physicalentity.obj
 0001:0007a6c0       ?Value@?$CSerializeWrapper@UISerialize@@@@QAEXPBDAAV?$CryStringT@D@@H@Z 3507b6c0 f i physicalentity.obj
 0001:0007a770       ?GetStateSnapshot@CPhysicalEntity@@UAEHV?$CSerializeWrapper@UISerialize@@@@MH@Z 3507b770 f   physicalentity.obj
 0001:0007ac20       ?SetStateFromSnapshot@CPhysicalEntity@@UAEHV?$CSerializeWrapper@UISerialize@@@@H@Z 3507bc20 f   physicalentity.obj
 0001:0007b0c0       ??$GetExtent@VCPhysicalEntity@@@GeomQuery@@QAEMPAVCPhysicalEntity@@W4EGeomForm@@@Z 3507c0c0 f i physicalentity.obj
 0001:0007b100       ?GetStatus@CPhysicalEntity@@UBEHPAUpe_status@@@Z 3507c100 f   physicalentity.obj
 0001:0007bc60       ?GetRandomPos@CPhysicalEntity@@UBEXAAURandomPos@@AAUGeomQuery@@W4EGeomForm@@@Z 3507cc60 f   physicalentity.obj
 0001:0007c020       ?ComputeExtent@CPhysicalEntity@@UBEMAAUGeomQuery@@W4EGeomForm@@@Z 3507d020 f   physicalentity.obj
 0001:0007c0e0       ?IsPlaceholder@CPhysicalWorld@@QAEHPBVCPhysicalPlaceholder@@@Z 3507d0e0 f i physicalplaceholder.obj
 0001:0007c140       ?GetWorld@CPhysicalPlaceholder@@UBEPAUIPhysicalWorld@@XZ 3507d140 f   physicalplaceholder.obj
 0001:0007c1e0       ?GetEntity@CPhysicalPlaceholder@@UAEPAVCPhysicalEntity@@XZ 3507d1e0 f   physicalplaceholder.obj
 0001:0007c2d0       ?GetType@CPhysicalPlaceholder@@UBE?AW4pe_type@@XZ 3507d2d0 f   physicalplaceholder.obj
 0001:0007c310       ?GetParams@CPhysicalPlaceholder@@UBEHPAUpe_params@@@Z 3507d310 f   physicalplaceholder.obj
 0001:0007c390       ?GetStatus@CPhysicalPlaceholder@@UBEHPAUpe_status@@@Z 3507d390 f   physicalplaceholder.obj
 0001:0007c3d0       ?Action@CPhysicalPlaceholder@@UAEHPAUpe_action@@H@Z 3507d3d0 f   physicalplaceholder.obj
 0001:0007c470       ?AddGeometry@CPhysicalPlaceholder@@UAEHPAUphys_geometry@@PAUpe_geomparams@@HH@Z 3507d470 f   physicalplaceholder.obj
 0001:0007c490       ?RemoveGeometry@CPhysicalPlaceholder@@UAEXHH@Z 3507d490 f   physicalplaceholder.obj
 0001:0007c4b0       ?GetStateSnapshot@CPhysicalPlaceholder@@UAEHAAVCStream@@MH@Z 3507d4b0 f   physicalplaceholder.obj
 0001:0007c4e0       ?GetStateSnapshot@CPhysicalPlaceholder@@UAEHV?$CSerializeWrapper@UISerialize@@@@MH@Z 3507d4e0 f   physicalplaceholder.obj
 0001:0007c510       ?SetStateFromSnapshot@CPhysicalPlaceholder@@UAEHAAVCStream@@H@Z 3507d510 f   physicalplaceholder.obj
 0001:0007c530       ?SetStateFromSnapshot@CPhysicalPlaceholder@@UAEHV?$CSerializeWrapper@UISerialize@@@@H@Z 3507d530 f   physicalplaceholder.obj
 0001:0007c550       ?SetStateFromTypedSnapshot@CPhysicalPlaceholder@@UAEHV?$CSerializeWrapper@UISerialize@@@@HH@Z 3507d550 f   physicalplaceholder.obj
 0001:0007c580       ?PostSetStateFromSnapshot@CPhysicalPlaceholder@@UAEHXZ 3507d580 f   physicalplaceholder.obj
 0001:0007c590       ?GetStateSnapshotTxt@CPhysicalPlaceholder@@UAEHPADHM@Z 3507d590 f   physicalplaceholder.obj
 0001:0007c5c0       ?SetStateFromSnapshotTxt@CPhysicalPlaceholder@@UAEXPBDH@Z 3507d5c0 f   physicalplaceholder.obj
 0001:0007c5e0       ?GetStateChecksum@CPhysicalPlaceholder@@UAEIXZ 3507d5e0 f   physicalplaceholder.obj
 0001:0007c5f0       ?SetNetworkAuthority@CPhysicalPlaceholder@@UAEXHH@Z 3507d5f0 f   physicalplaceholder.obj
 0001:0007c610       ?Step@CPhysicalPlaceholder@@UAEHM@Z 3507d610 f   physicalplaceholder.obj
 0001:0007c630       ?StartStep@CPhysicalPlaceholder@@UAEXM@Z 3507d630 f   physicalplaceholder.obj
 0001:0007c650       ?StepBack@CPhysicalPlaceholder@@UAEXM@Z 3507d650 f   physicalplaceholder.obj
 0001:0007c670       ??$SignalEvent@UEventPhysStateChange@@@CPhysicalWorld@@QAEHPAUEventPhysStateChange@@H@Z 3507d670 f i physicalplaceholder.obj
 0001:0007c6e0       ??$OnEvent@UEventPhysStateChange@@@CPhysicalWorld@@QAEHIPAUEventPhysStateChange@@PAPAU1@@Z 3507d6e0 f i physicalplaceholder.obj
 0001:0007c790       ?SetParams@CPhysicalPlaceholder@@UAEHPAUpe_params@@H@Z 3507d790 f   physicalplaceholder.obj
 0001:0007ca50       ??_GIThreadTask@@UAEPAXI@Z 3507da50 f i physicalworld.obj
 0001:0007ca50       ??_EIThreadTask@@UAEPAXI@Z 3507da50 f i physicalworld.obj
 0001:0007ca80       ??Ape_entgrid@@QAEHH@Z     3507da80 f i physicalworld.obj
 0001:0007cae0       ??Ape_entgrid@@QAEAAHI@Z   3507dae0 f i physicalworld.obj
 0001:0007cb50       ?GetGridSize@@YAHAAUpe_entgrid@@ABU?$Vec2_tpl@H@@@Z 3507db50 f i physicalworld.obj
 0001:0007cc00       ?GetTmpEntList@CPhysicalWorld@@QAEHAAPAPAVCPhysicalEntity@@H@Z 3507dc00 f i physicalworld.obj
 0001:0007cc80       ??1CBlockProfiler@@QAE@XZ  3507dc80 f i physicalworld.obj
 0001:0007cca0       ?CryLog@@YAXPBDZZ          3507dca0 f i physicalworld.obj
 0001:0007ccd0       ?CryLogAlways@@YAXPBDZZ    3507dcd0 f i physicalworld.obj
 0001:0007cd00       ?IsEnd@CPhysicalEntityIt@CPhysicalWorld@@UAE_NXZ 3507dd00 f   physicalworld.obj
 0001:0007cd10       ?Next@CPhysicalEntityIt@CPhysicalWorld@@UAEPAUIPhysicalEntity@@XZ 3507dd10 f   physicalworld.obj
 0001:0007cd90       ?This@CPhysicalEntityIt@CPhysicalWorld@@UAEPAUIPhysicalEntity@@XZ 3507dd90 f   physicalworld.obj
 0001:0007cdb0       ?MoveFirst@CPhysicalEntityIt@CPhysicalWorld@@UAEXXZ 3507ddb0 f   physicalworld.obj
 0001:0007cdf0       ?GetEntityProfileType@@YAHPAVCPhysicalEntity@@@Z 3507ddf0 f   physicalworld.obj
 0001:0007ceb0       ?Cleanup@CPhysicalWorld@@UAEXXZ 3507deb0 f   physicalworld.obj
 0001:0007ced0       ?DeactivateOnDemandGrid@CPhysicalWorld@@UAEXXZ 3507ded0 f   physicalworld.obj
 0001:0007cfa0       ?SetSurfaceParameters@CPhysicalWorld@@UAEHHMMI@Z 3507dfa0 f   physicalworld.obj
 0001:0007d020       ?GetSurfaceParameters@CPhysicalWorld@@UAEHHAAM0AAI@Z 3507e020 f   physicalworld.obj
 0001:0007d060       ?SetSurfaceParameters@CPhysicalWorld@@UAEHHMMMMMMI@Z 3507e060 f   physicalworld.obj
 0001:0007d0e0       ?GetSurfaceParameters@CPhysicalWorld@@UAEHHAAM00000AAI@Z 3507e0e0 f   physicalworld.obj
 0001:0007d150       ?CleanseEventsQueue@CPhysicalWorld@@QAEXXZ 3507e150 f   physicalworld.obj
 0001:0007d200       ?PatchEventsQueue@CPhysicalWorld@@QAEXPAUIPhysicalEntity@@PAXH@Z 3507e200 f   physicalworld.obj
 0001:0007d2b0       ?GetFreeEntId@CPhysicalWorld@@QAEHXZ 3507e2b0 f   physicalworld.obj
 0001:0007d3d0       ?bitcount@@YAHH@Z          3507e3d0 f i physicalworld.obj
 0001:0007d430       ?GetPhysicalEntityId@CPhysicalWorld@@UAEHPAUIPhysicalEntity@@@Z 3507e430 f   physicalworld.obj
 0001:0007d450       ?GetPhysicalEntityById@CPhysicalWorld@@UAEPAUIPhysicalEntity@@H@Z 3507e450 f   physicalworld.obj
 0001:0007d8f0       ?GroupByOuterEntity@@YAXPAPAVCPhysicalEntity@@HH@Z 3507e8f0 f   physicalworld.obj
 0001:0007d9a0       ?ScheduleForStep@CPhysicalWorld@@QAEXPAVCPhysicalEntity@@M@Z 3507e9a0 f   physicalworld.obj
 0001:0007da30       ?Stop@SPhysTask@@UAEXXZ    3507ea30 f   physicalworld.obj
 0001:0007da50       ?ProcessNextEngagedIndependentEntity@CPhysicalWorld@@QAEXH@Z 3507ea50 f   physicalworld.obj
 0001:0007db80       ?ProcessNextIndependentEntity@CPhysicalWorld@@QAEXMHH@Z 3507eb80 f   physicalworld.obj
 0001:0007dcd0       ?FlushOldThunks@CPhysicalWorld@@QAEXXZ 3507ecd0 f   physicalworld.obj
 0001:0007dd70       ?ChangeEntitySimClass@CPhysicalWorld@@QAEHPAVCPhysicalEntity@@@Z 3507ed70 f   physicalworld.obj
 0001:0007e050       ?UnmarkEntityAsDeforming@CPhysicalWorld@@QAEXPAVCPhysicalEntity@@@Z 3507f050 f   physicalworld.obj
 0001:0007e0e0       ?PurgeDeletedEntities@CPhysicalWorld@@UAEXXZ 3507f0e0 f   physicalworld.obj
 0001:0007e2c0       ?DrawEntityHelperInformation@CPhysicalWorld@@UAEXPAUIPhysRenderer@@HH@Z 3507f2c0 f   physicalworld.obj
 0001:0007e2f0       ??_GIGeomManager@@UAEPAXI@Z 3507f2f0 f i physicalworld.obj
 0001:0007e2f0       ??_EIGeomManager@@UAEPAXI@Z 3507f2f0 f i physicalworld.obj
 0001:0007e320       ?AddEntityProfileInfo@CPhysicalWorld@@QAEXPAVCPhysicalEntity@@H@Z 3507f320 f   physicalworld.obj
 0001:0007e530       ?AddEventClient@CPhysicalWorld@@UAEXHP6AHPBUEventPhys@@@ZHM@Z 3507f530 f   physicalworld.obj
 0001:0007e600       ?RemoveEventClient@CPhysicalWorld@@UAEHHP6AHPBUEventPhys@@@ZH@Z 3507f600 f   physicalworld.obj
 0001:0007e6f0       ?AllocEvent@CPhysicalWorld@@QAEPAUEventPhys@@HH@Z 3507f6f0 f   physicalworld.obj
 0001:0007e7b0       ?GetPumpLoggedEventsTicks@CPhysicalWorld@@UAEIXZ 3507f7b0 f   physicalworld.obj
 0001:0007e7d0       ??_EIPhysicalWorld@@UAEPAXI@Z 3507f7d0 f i physicalworld.obj
 0001:0007e7d0       ??_GIPhysicalWorld@@UAEPAXI@Z 3507f7d0 f i physicalworld.obj
 0001:0007e800       ?ClearLoggedEvents@CPhysicalWorld@@UAEXXZ 3507f800 f   physicalworld.obj
 0001:0007e8c0       ?RemoveExplosionShape@CPhysicalWorld@@UAEXH@Z 3507f8c0 f   physicalworld.obj
 0001:0007e9c0       ?GetExplosionShape@CPhysicalWorld@@QAEPAUIGeometry@@MHAAMAAH@Z 3507f9c0 f   physicalworld.obj
 0001:0007ec10       ?GetWaterManagerParams@CPhysicalWorld@@UAEHPAUpe_params@@@Z 3507fc10 f   physicalworld.obj
 0001:0007ec30       ?GetWatermanStatus@CPhysicalWorld@@UAEHPAUpe_status@@@Z 3507fc30 f   physicalworld.obj
 0001:0007ec50       ??$FreeObjPool@Ugeom@@@CPhysicalWorld@@QAEXAAPAUgeom@@HAAH@Z 3507fc50 f i physicalworld.obj
 0001:0007ecc0       ??$SignalEvent@UEventPhysEntityDeleted@@@CPhysicalWorld@@QAEHPAUEventPhysEntityDeleted@@H@Z 3507fcc0 f i physicalworld.obj
 0001:0007ed30       ?UnregisterAllCracks@CGeomManager@@UAEXP6AXPAUIGeometry@@@Z@Z 3507fd30 f i physicalworld.obj
 0001:0007ed90       ?ReleaseGeomsImmediately@CGeomManager@@UAEX_N@Z 3507fd90 f i physicalworld.obj
 0001:0007eda0       ?CreateMesh@CGeomManager@@UAEPAUIGeometry@@V?$strided_pointer@$$CBU?$Vec3_tpl@M@@@@V?$strided_pointer@G@@PADPAHHHMHHM@Z 3507fda0 f i physicalworld.obj
 0001:0007ee10       ??_GCGeomManager@@UAEPAXI@Z 3507fe10 f i physicalworld.obj
 0001:0007ee10       ??_ECGeomManager@@UAEPAXI@Z 3507fe10 f i physicalworld.obj
 0001:0007ee40       ?AllocateGrid@@YAXAAUpe_entgrid@@ABU?$Vec2_tpl@H@@@Z 3507fe40 f i physicalworld.obj
 0001:0007ef00       ?GetTaskInfo@SPhysTask@@UAEPAUSThreadTaskInfo@@XZ 3507ff00 f i physicalworld.obj
 0001:0007ef10       ?getPODcell@CPhysicalWorld@@QAEPAUpe_PODcell@@HH@Z 3507ff10 f i physicalworld.obj
 0001:0007efd0       ??0CPhysicalEntityIt@CPhysicalWorld@@QAE@PAV1@@Z 3507ffd0 f   physicalworld.obj
 0001:0007f030       ?AddRef@CPhysicalEntityIt@CPhysicalWorld@@UAEXXZ 35080030 f i physicalworld.obj
 0001:0007f040       ?Release@CPhysicalEntityIt@CPhysicalWorld@@UAEXXZ 35080040 f i physicalworld.obj
 0001:0007f060       ?Init@CPhysicalWorld@@UAEXXZ 35080060 f   physicalworld.obj
 0001:0007f7a0       ?GetHeightfieldData@CPhysicalWorld@@UAEPAUIPhysicalEntity@@PAUheightfield@primitives@@@Z 350807a0 f   physicalworld.obj
 0001:0007f850       ?AddRefEntInPODGrid@CPhysicalWorld@@UAEHPAUIPhysicalEntity@@PBU?$Vec3_tpl@M@@@Z 35080850 f   physicalworld.obj
 0001:0007faf0       ?GetPODGridCellBBox@CPhysicalWorld@@QAEXHHAAU?$Vec3_tpl@M@@0@Z 35080af0 f   physicalworld.obj
 0001:0007fc00       ?CreatePhysicalPlaceholder@CPhysicalWorld@@UAEPAUIPhysicalEntity@@W4pe_type@@PAUpe_params@@PAXHH@Z 35080c00 f   physicalworld.obj
 0001:0007ffc0       ??_ECPhysicalPlaceholder@@UAEPAXI@Z 35080fc0 f i physicalworld.obj
 0001:00080020       ?ReserveEntityCount@CPhysicalWorld@@UAEHH@Z 35081020 f   physicalworld.obj
 0001:00080370       ?SetPhysicalEntityId@CPhysicalWorld@@UAEHPAUIPhysicalEntity@@HHH@Z 35081370 f   physicalworld.obj
 0001:00080630       ?ReallocTmpEntList@CPhysicalWorld@@QAEHAAPAPAVCPhysicalEntity@@HH@Z 35081630 f   physicalworld.obj
 0001:00080710       ?UpdateDeformingEntities@CPhysicalWorld@@UAEXM@Z 35081710 f   physicalworld.obj
 0001:00080830       ?ProcessIslandSolverResults@CPhysicalWorld@@QAEXHHMMHMAAHPAPAUentity_contact@@HHH_J@Z 35081830 f   physicalworld.obj
 0001:00080d50       ?ProcessNextEntityIsland@CPhysicalWorld@@QAEXMHHAAHH@Z 35081d50 f   physicalworld.obj
 0001:00081470       ?ProcessNextLivingEntity@CPhysicalWorld@@QAEXMHH@Z 35082470 f   physicalworld.obj
 0001:00081a20       ?ProcessBreakingEntities@CPhysicalWorld@@QAEXM@Z 35082a20 f   physicalworld.obj
 0001:00081b00       ?ThreadProc@CPhysicalWorld@@QAEXHPAUSPhysTask@@@Z 35082b00 f   physicalworld.obj
 0001:00081ca0       ??4geom_world_data@@QAEAAU0@ABU0@@Z 35082ca0 f i physicalworld.obj
 0001:00081d40       ?DetachEntityGridThunks@CPhysicalWorld@@QAEXPAVCPhysicalPlaceholder@@@Z 35082d40 f   physicalworld.obj
 0001:00081f90       ?SortThunks@CPhysicalWorld@@QAEXXZ 35082f90 f   physicalworld.obj
 0001:000825f0       ?IsAffectedByExplosion@CPhysicalWorld@@UAEMPAUIPhysicalEntity@@PAU?$Vec3_tpl@M@@@Z 350835f0 f   physicalworld.obj
 0001:00082680       ??4phys_geometry@@QAEAAU0@ABU0@@Z 35083680 f i physicalworld.obj
 0001:000826f0       ?MarkEntityAsDeforming@CPhysicalWorld@@QAEXPAVCPhysicalEntity@@@Z 350836f0 f   physicalworld.obj
 0001:000827e0       ?ResetDynamicEntities@CPhysicalWorld@@UAEXXZ 350837e0 f   physicalworld.obj
 0001:00082860       ?DestroyDynamicEntities@CPhysicalWorld@@UAEXXZ 35083860 f   physicalworld.obj
 0001:00082c90       ?DrawPhysicsHelperInformation@CPhysicalWorld@@UAEXPAUIPhysRenderer@@H@Z 35083c90 f   physicalworld.obj
 0001:00083b50       ?GetMemoryStatistics@CPhysicalWorld@@UAEXPAVICrySizer@@@Z 35084b50 f   physicalworld.obj
 0001:00084150       ?AddFuncProfileInfo@CPhysicalWorld@@QAEXPBDH@Z 35085150 f   physicalworld.obj
 0001:00084330       ?PumpLoggedEvents@CPhysicalWorld@@UAEXXZ 35085330 f   physicalworld.obj
 0001:000848f0       ?AddExplosionShape@CPhysicalWorld@@UAEHPAUIGeometry@@MHM@Z 350858f0 f   physicalworld.obj
 0001:00084b80       ?SetWaterManagerParams@CPhysicalWorld@@UAEHPAUpe_params@@@Z 35085b80 f   physicalworld.obj
 0001:00084c20       ?DestroyWaterManager@CPhysicalWorld@@UAEXXZ 35085c20 f   physicalworld.obj
 0001:00084c50       ?GetEntityMassAndCom@CPhysicalWorld@@UAEXPAUIPhysicalEntity@@AAMAAU?$Vec3_tpl@M@@@Z 35085c50 f   physicalworld.obj
 0001:00084d40       ?SerializeGarbageTypedSnapshot@CPhysicalWorld@@UAEXV?$CSerializeWrapper@UISerialize@@@@HH@Z 35085d40 f   physicalworld.obj
 0001:00084ee0       ?GetEntitiesIterator@CPhysicalWorld@@UAEPAUIPhysicalEntityIt@@XZ 35085ee0 f   physicalworld.obj
 0001:00084f00       ??_GSThreadTaskInfo@@UAEPAXI@Z 35085f00 f i physicalworld.obj
 0001:00084f00       ??_ESThreadTaskInfo@@UAEPAXI@Z 35085f00 f i physicalworld.obj
 0001:00084f00       ??_ECMultiThreadRefCount@@UAEPAXI@Z 35085f00 f i physicalworld.obj
 0001:00084f00       ??_GCMultiThreadRefCount@@UAEPAXI@Z 35085f00 f i physicalworld.obj
 0001:00084f30       ??_GSPhysTask@@UAEPAXI@Z   35085f30 f i physicalworld.obj
 0001:00084f30       ??_ESPhysTask@@UAEPAXI@Z   35085f30 f i physicalworld.obj
 0001:00084f60       ??1CPhysFuncProfiler@@QAE@XZ 35085f60 f i physicalworld.obj
 0001:00084f90       ??0CPhysicalWorld@@QAE@PAUILog@@@Z 35085f90 f   physicalworld.obj
 0001:00085620       ?GetGeomManager@CPhysicalWorld@@UAEPAUIGeomManager@@XZ 35086620 f i physicalworld.obj
 0001:00085630       ?GetPhysUtils@CPhysicalWorld@@UAEPAUIPhysUtils@@XZ 35086630 f i physicalworld.obj
 0001:00085640       ?GetPhysVars@CPhysicalWorld@@UAEPAUPhysicsVars@@XZ 35086640 f i physicalworld.obj
 0001:00085650       ?CreatePhysicalEntity@CPhysicalWorld@@UAEPAUIPhysicalEntity@@W4pe_type@@PAUpe_params@@PAXHH@Z 35086650 f i physicalworld.obj
 0001:00085680       ?GetPhysicsTime@CPhysicalWorld@@UAEMXZ 35086680 f i physicalworld.obj
 0001:00085690       ?GetiPhysicsTime@CPhysicalWorld@@UAEHXZ 35086690 f i physicalworld.obj
 0001:000856a0       ?SetPhysicsTime@CPhysicalWorld@@UAEXM@Z 350866a0 f i physicalworld.obj
 0001:000856e0       ?SetiPhysicsTime@CPhysicalWorld@@UAEXH@Z 350866e0 f i physicalworld.obj
 0001:00085710       ?SetSnapshotTime@CPhysicalWorld@@UAEXMH@Z 35086710 f i physicalworld.obj
 0001:00085750       ?SetiSnapshotTime@CPhysicalWorld@@UAEXHH@Z 35086750 f i physicalworld.obj
 0001:00085780       ?GetEntityCount@CPhysicalWorld@@UAEHH@Z 35086780 f i physicalworld.obj
 0001:000857a0       ?DeletePointer@CPhysicalWorld@@UAEXPAX@Z 350867a0 f i physicalworld.obj
 0001:000857c0       ?SetPhysicsStreamer@CPhysicalWorld@@UAEXPAUIPhysicsStreamer@@@Z 350867c0 f i physicalworld.obj
 0001:000857d0       ?SetPhysicsEventClient@CPhysicalWorld@@UAEXPAUIPhysicsEventClient@@@Z 350867d0 f i physicalworld.obj
 0001:000857e0       ?GetLastEntityUpdateTime@CPhysicalWorld@@UAEMPAUIPhysicalEntity@@@Z 350867e0 f i physicalworld.obj
 0001:00085800       ?GetInternalLock@CPhysicalWorld@@UAEPCHH@Z 35086800 f i physicalworld.obj
 0001:00085850       ?GetEntityProfileInfo@CPhysicalWorld@@UAEHAAPAUphys_profile_info@@@Z 35086850 f i physicalworld.obj
 0001:00085870       ?GetFuncProfileInfo@CPhysicalWorld@@UAEHAAPAUphys_profile_info@@@Z 35086870 f i physicalworld.obj
 0001:00085890       ?GetGroupProfileInfo@CPhysicalWorld@@UAEHAAPAUphys_profile_info@@@Z 35086890 f i physicalworld.obj
 0001:000858b0       ?GetJobProfileInfo@CPhysicalWorld@@UAEHAAPAUphys_job_info@@@Z 350868b0 f i physicalworld.obj
 0001:000858d0       ?GetWaterMat@CPhysicalWorld@@UAEHXZ 350868d0 f i physicalworld.obj
 0001:000858e0       ?RemoveAllExplosionShapes@CPhysicalWorld@@UAEXP6AXPAUIGeometry@@@Z@Z 350868e0 f i physicalworld.obj
 0001:00085950       ?GetIWorld@CPhysicalWorld@@UAEPAUIPhysicalWorld@@XZ 35086950 f i physicalworld.obj
 0001:00085960       ??$SignalEvent@UEventPhysEnvChange@@@CPhysicalWorld@@QAEHPAUEventPhysEnvChange@@H@Z 35086960 f i physicalworld.obj
 0001:000859d0       ??$SignalEvent@UEventPhysRWIResult@@@CPhysicalWorld@@QAEHPAUEventPhysRWIResult@@H@Z 350869d0 f i physicalworld.obj
 0001:00085a40       ??$SignalEvent@UEventPhysPWIResult@@@CPhysicalWorld@@QAEHPAUEventPhysPWIResult@@H@Z 35086a40 f i physicalworld.obj
 0001:00085ab0       ??_ECPhysicalWorld@@W3AEPAXI@Z 35086ab0 f i physicalworld.obj
 0001:00085ac0       ??_ECPhysicalWorld@@W7AEPAXI@Z 35086ac0 f i physicalworld.obj
 0001:00085ad0       ?CoverPolygonWithCircles@CPhysicalWorld@@UAEHV?$strided_pointer@U?$Vec2_tpl@M@@@@H_NABU?$Vec2_tpl@M@@AAPAU3@AAPAMM@Z 35086ad0 f i physicalworld.obj
 0001:00085b10       ?qhull@CPhysicalWorld@@UAEHV?$strided_pointer@U?$Vec3_tpl@M@@@@HAAPAHP6APAXI@Z@Z 35086b10 f i physicalworld.obj
 0001:00085b40       ??$OnEvent@UEventPhysEnvChange@@@CPhysicalWorld@@QAEHIPAUEventPhysEnvChange@@PAPAU1@@Z 35086b40 f i physicalworld.obj
 0001:00085bf0       ??$OnEvent@UEventPhysRWIResult@@@CPhysicalWorld@@QAEHIPAUEventPhysRWIResult@@PAPAU1@@Z 35086bf0 f i physicalworld.obj
 0001:00085c80       ??$OnEvent@UEventPhysPWIResult@@@CPhysicalWorld@@QAEHIPAUEventPhysPWIResult@@PAPAU1@@Z 35086c80 f i physicalworld.obj
 0001:00085d10       ??$OnEvent@UEventPhysArea@@@CPhysicalWorld@@QAEHIPAUEventPhysArea@@PAPAU1@@Z 35086d10 f i physicalworld.obj
 0001:00085da0       ??$OnEvent@UEventPhysAreaChange@@@CPhysicalWorld@@QAEHIPAUEventPhysAreaChange@@PAPAU1@@Z 35086da0 f i physicalworld.obj
 0001:00085e30       ??$OnEvent@UEventPhysEntityDeleted@@@CPhysicalWorld@@QAEHIPAUEventPhysEntityDeleted@@PAPAU1@@Z 35086e30 f i physicalworld.obj
 0001:00085ee0       ?RayWorldIntersection@CPhysicalWorld@@UAEHABU?$Vec3_tpl@M@@0HIPAUray_hit@@HPAPAUIPhysicalEntity@@HPAXHPBDPAUray_hit_cached@@H@Z 35086ee0 f i physicalworld.obj
 0001:00085f80       ?AddDeferredEvent@CPhysicalWorld@@UAEPAUEventPhys@@HPAU2@@Z 35086f80 f i physicalworld.obj
 0001:00086130       ?DeallocGThunksPool@CPhysicalWorld@@QAEXXZ 35087130 f   physicalworld.obj
 0001:00086190       ??_ESPwiRequest@@QAEPAXI@Z 35087190 f i physicalworld.obj
 0001:00086230       ?SetHeightfieldData@CPhysicalWorld@@UAEPAUIPhysicalEntity@@PBUheightfield@primitives@@PAHH@Z 35087230 f   physicalworld.obj
 0001:00086770       ?RegisterBBoxInPODGrid@CPhysicalWorld@@UAEXPBU?$Vec3_tpl@M@@@Z 35087770 f   physicalworld.obj
 0001:00086e10       ?GetEntitiesAround@CPhysicalWorld@@QAEHABU?$Vec3_tpl@M@@0AAPAPAVCPhysicalEntity@@HPAV3@HH@Z 35087e10 f   physicalworld.obj
 0001:000886b0       ?OnUpdate@SPhysTask@@UAEXXZ 350896b0 f   physicalworld.obj
 0001:000886c0       ??4SBreakRequest@@QAEAAU0@ABU0@@Z 350896c0 f i physicalworld.obj
 0001:00088900       ?ClonePhysGeomInEntity@CPhysicalWorld@@QAEXPAVCPhysicalEntity@@HPAUIGeometry@@@Z 35089900 f   physicalworld.obj
 0001:00088a90       ?DeformEntityPart@CPhysicalWorld@@QAEHPAVCPhysicalEntity@@HPAUpe_explosion@@PAUgeom_world_data@@2H@Z 35089a90 f   physicalworld.obj
 0001:000890f0       ?CalculateExplosionExposure@CPhysicalWorld@@UAEMPAUpe_explosion@@PAUIPhysicalEntity@@@Z 3508a0f0 f   physicalworld.obj
 0001:00089670       ?CollideEntityWithBeam@CPhysicalWorld@@UAEHPAUIPhysicalEntity@@U?$Vec3_tpl@M@@1MPAUray_hit@@@Z 3508a670 f   physicalworld.obj
 0001:00089f60       ?CollideEntityWithPrimitive@CPhysicalWorld@@UAEHPAUIPhysicalEntity@@HPAUprimitive@primitives@@U?$Vec3_tpl@M@@PAUray_hit@@PAUintersection_params@@@Z 3508af60 f   physicalworld.obj
 0001:0008ae40       ?RayTraceEntity@CPhysicalWorld@@UAEHPAUIPhysicalEntity@@U?$Vec3_tpl@M@@1PAUray_hit@@PAUpe_params_pos@@I@Z 3508be40 f   physicalworld.obj
 0001:0008b9d0       ?SavePhysicalEntityPtr@CPhysicalWorld@@UAEXV?$CSerializeWrapper@UISerialize@@@@PAUIPhysicalEntity@@@Z 3508c9d0 f   physicalworld.obj
 0001:0008ba80       ?LoadPhysicalEntityPtr@CPhysicalWorld@@UAEPAUIPhysicalEntity@@V?$CSerializeWrapper@UISerialize@@@@@Z 3508ca80 f   physicalworld.obj
 0001:0008bd30       ?SetStateFromTypedSnapshot@CPhysicalEntity@@UAEHV?$CSerializeWrapper@UISerialize@@@@HH@Z 3508cd30 f   physicalworld.obj
 0001:0008bef0       ??$ReallocQueue@USBreakRequest@@@CPhysicalWorld@@QAEXAAPAUSBreakRequest@@HAAH11H@Z 3508cef0 f i physicalworld.obj
 0001:0008c040       ??$ReallocQueue@USPwiRequest@@@CPhysicalWorld@@QAEXAAPAUSPwiRequest@@HAAH11H@Z 3508d040 f i physicalworld.obj
 0001:0008c180       ?GetEntitiesInBox@CPhysicalWorld@@UAEHU?$Vec3_tpl@M@@0AAPAPAUIPhysicalEntity@@HH@Z 3508d180 f i physicalworld.obj
 0001:0008c1e0       ?AllocGThunksPool@CPhysicalWorld@@QAEXH@Z 3508d1e0 f   physicalworld.obj
 0001:0008c500       ?Shutdown@CPhysicalWorld@@UAEXH@Z 3508d500 f   physicalworld.obj
 0001:0008cdc0       ?RepositionEntity@CPhysicalWorld@@QAEHPAVCPhysicalPlaceholder@@HPAU?$Vec3_tpl@M@@H@Z 3508ddc0 f   physicalworld.obj
 0001:0008dc40       ?DeformPhysicalEntity@CPhysicalWorld@@UAEHPAUIPhysicalEntity@@ABU?$Vec3_tpl@M@@1MH@Z 3508ec40 f   physicalworld.obj
 0001:0008e970       ?SimulateExplosion@CPhysicalWorld@@UAEXPAUpe_explosion@@PAPAUIPhysicalEntity@@HHH@Z 3508f970 f   physicalworld.obj
 0001:00092ef0       ?PrimitiveWorldIntersection@CPhysicalWorld@@UAEMABUSPWIParams@IPhysicalWorld@@AAUWriteLockCond@@PBD@Z 35093ef0 f   physicalworld.obj
 0001:00094db0       ??1CPhysicalWorld@@UAE@XZ  35095db0 f   physicalworld.obj
 0001:00094ef0       ?SetupEntityGrid@CPhysicalWorld@@UAEXHU?$Vec3_tpl@M@@HHMMH@Z 35095ef0 f   physicalworld.obj
 0001:00095260       ?CreatePhysicalEntity@CPhysicalWorld@@UAEPAUIPhysicalEntity@@W4pe_type@@MPAUpe_params@@PAXHHPAU2@@Z 35096260 f   physicalworld.obj
 0001:00095ac0       ?DestroyPhysicalEntity@CPhysicalWorld@@UAEHPAUIPhysicalEntity@@HH@Z 35096ac0 f   physicalworld.obj
 0001:00096910       ?TimeStep@CPhysicalWorld@@UAEXMH@Z 35097910 f   physicalworld.obj
 0001:00098a60       ??_ECPhysicalWorld@@UAEPAXI@Z 35099a60 f i physicalworld.obj
 0001:00098a60       ??_GCPhysicalWorld@@UAEPAXI@Z 35099a60 f i physicalworld.obj
 0001:00098a90       ?update_followers@@YAXHHH@Z 35099a90 f   rigidbody.obj
 0001:00098b20       ?add_route_follower@@YAXHHH@Z 35099b20 f   rigidbody.obj
 0001:00098bc0       ?CleanupContactSolvers@@YAXXZ 35099bc0 f   rigidbody.obj
 0001:00098be0       ??0RigidBody@@QAE@XZ       35099be0 f   rigidbody.obj
 0001:00098d30       ?zero@RigidBody@@QAEXXZ    35099d30 f   rigidbody.obj
 0001:00098da0       ?GetRBMemStats@@YAXPAVICrySizer@@@Z 35099da0 f   rigidbody.obj
 0001:00098de0       ?trace_unproj_route@@YAXHHH@Z 35099de0 f   rigidbody.obj
 0001:00098ee0       ?RegisterContact@@YAXPAUentity_contact@@@Z 35099ee0 f   rigidbody.obj
 0001:00098f40       ?DisablePreCG@@YAXXZ       35099f40 f   rigidbody.obj
 0001:00099280       ?GetContactMatrix@RigidBody@@QAEXABU?$Vec3_tpl@M@@AAU?$Matrix33_tpl@M@@@Z 3509a280 f   rigidbody.obj
 0001:000996c0       ?ComputeRc@@YANPAVRigidBody@@PAPAUentity_contact@@HHH@Z 3509a6c0 f   rigidbody.obj
 0001:0009a560       ?InitContactSolver@@YAXM@Z 3509b560 f   rigidbody.obj
 0001:0009a5f0       ?AllocSolverTmpBuf@@YAPADH@Z 3509b5f0 f   rigidbody.obj
 0001:0009a710       ?UpdateState@RigidBody@@QAEXXZ 3509b710 f   rigidbody.obj
 0001:0009ab30       ?Create@RigidBody@@QAEXABU?$Vec3_tpl@M@@0ABU?$Quat_tpl@M@@MM10@Z 3509bb30 f   rigidbody.obj
 0001:0009aea0       ?Add@RigidBody@@QAEXABU?$Vec3_tpl@M@@U2@ABU?$Quat_tpl@M@@MM@Z 3509bea0 f   rigidbody.obj
 0001:0009c150       ?Step@RigidBody@@QAEXM@Z   3509d150 f   rigidbody.obj
 0001:0009c940       ?InvokeContactSolver@@YAHMPAUSolverSettings@@MAAPAPAUentity_contact@@AAHAAPAPAVRigidBody@@@Z 3509d940 f   rigidbody.obj
 0001:000ac860       ?CryFatalError@@YAXPBDZZ   350ad860 f i rigidentity.obj
 0001:000ac8d0       ?AttachContact@CRigidEntity@@QAEXPAUentity_contact@@HPAVCPhysicalEntity@@@Z 350ad8d0 f   rigidentity.obj
 0001:000aca10       ?DetachContact@CRigidEntity@@QAEXPAUentity_contact@@HH@Z 350ada10 f   rigidentity.obj
 0001:000acb90       ?GetParams@CRigidEntity@@UBEHPAUpe_params@@@Z 350adb90 f   rigidentity.obj
 0001:000acd10       ?HasContactsWith@CRigidEntity@@UAEHPAVCPhysicalEntity@@@Z 350add10 f   rigidentity.obj
 0001:000acd70       ?HasCollisionContactsWith@CRigidEntity@@UAEHPAVCPhysicalEntity@@@Z 350add70 f   rigidentity.obj
 0001:000acdc0       ?HasConstraintContactsWith@CRigidEntity@@UBEHPBVCPhysicalEntity@@H@Z 350addc0 f   rigidentity.obj
 0001:000acea0       ?HasPartContactsWith@CRigidEntity@@UAEHPAVCPhysicalEntity@@HH@Z 350adea0 f   rigidentity.obj
 0001:000ad0c0       ?Awake@CRigidEntity@@UAEHHH@Z 350ae0c0 f   rigidentity.obj
 0001:000ad2f0       ?AlertNeighbourhoodND@CRigidEntity@@UAEXH@Z 350ae2f0 f   rigidentity.obj
 0001:000ad3e0       ?MaskIgnoredColliders@CRigidEntity@@QAE_KH@Z 350ae3e0 f   rigidentity.obj
 0001:000ad530       ?UnmaskIgnoredColliders@CRigidEntity@@QAEX_KH@Z 350ae530 f   rigidentity.obj
 0001:000ad620       ?IgnoreCollisionsWith@CRigidEntity@@UBE_NPBVCPhysicalEntity@@H@Z 350ae620 f   rigidentity.obj
 0001:000ad7a0       ?CleanupAfterContactsCheck@CRigidEntity@@QAEXH@Z 350ae7a0 f   rigidentity.obj
 0001:000ad820       ?RemoveConstraint@CRigidEntity@@QAEHH@Z 350ae820 f   rigidentity.obj
 0001:000ad910       ?BreakableConstraintsUpdated@CRigidEntity@@UAEXXZ 350ae910 f   rigidentity.obj
 0001:000adb70       ?ComputeBBoxRE@CRigidEntity@@QAEXPAUcoord_block_BBox@@@Z 350aeb70 f   rigidentity.obj
 0001:000adc80       ?UpdatePosition@CRigidEntity@@QAEXH@Z 350aec80 f   rigidentity.obj
 0001:000adf50       ?StartStep@CRigidEntity@@UAEXM@Z 350aef50 f   rigidentity.obj
 0001:000adf70       ?GetContactCount@CRigidEntity@@UAEHH@Z 350aef70 f   rigidentity.obj
 0001:000ae000       ?GetDamping@CRigidEntity@@UAEMM@Z 350af000 f   rigidentity.obj
 0001:000ae060       ??4SRigidEntityNetSerialize@@QAEAAU0@ABU0@@Z 350af060 f i rigidentity.obj
 0001:000ae0d0       ?WriteContacts@CRigidEntity@@QAEHAAVCStream@@H@Z 350af0d0 f   rigidentity.obj
 0001:000ae200       ?GetLocalSequenceNumber@CRigidEntity@@QAEEXZ 350af200 f   rigidentity.obj
 0001:000ae260       ?GetInterpSequenceNumber@CRigidEntity@@QAEMXZ 350af260 f   rigidentity.obj
 0001:000ae320       ?GetStateChecksum@CRigidEntity@@UAEIXZ 350af320 f   rigidentity.obj
 0001:000ae660       ?ReportConstraintBreak@CRigidEntity@@QAEAAUEventPhysJointBroken@@AAU2@H@Z 350af660 f   rigidentity.obj
 0001:000ae780       ?GetMemoryStatistics@CRigidEntity@@UBEXPAVICrySizer@@@Z 350af780 f   rigidentity.obj
 0001:000ae850       ??0?$AngleAxis_tpl@M@@QAE@ABU?$Quat_tpl@M@@@Z 350af850 f i rigidentity.obj
 0001:000ae960       ??$ReallocateList@PAVCPhysicalEntity@@@@YAPAPAVCPhysicalEntity@@AAPAPAV0@HH_N1@Z 350af960 f i physicalentity.obj
 0001:000ae960       ??$ReallocateList@PAD@@YAPAPADAAPAPADHH_N1@Z 350af960 f i articulatedentity.obj
 0001:000ae960       ??$ReallocateList@H@@YAPAHAAPAHHH_N1@Z 350af960 f i physicalworld.obj
 0001:000ae960       ??$ReallocateList@PAUentity_contact@@@@YAPAPAUentity_contact@@AAPAPAU0@HH_N1@Z 350af960 f i rigidentity.obj
 0001:000aea00       ??$ReallocateList@_K@@YAPA_KAAPA_KHH_N1@Z 350afa00 f i rigidentity.obj
 0001:000aeaa0       ??$?0M@?$Ang3_tpl@M@@QAE@ABU?$Quat_tpl@M@@@Z 350afaa0 f i rigidentity.obj
 0001:000aebe0       ?FreeContact@CPhysicalWorld@@QAEXPAUentity_contact@@@Z 350afbe0 f i rigidentity.obj
 0001:000aec50       ?Glob2Loc@@YA?AU?$Vec3_tpl@M@@ABUentity_contact@@H@Z 350afc50 f i rigidentity.obj
 0001:000aeed0       ??0pe_params_rope@@QAE@XZ  350afed0 f i rigidentity.obj
 0001:000af0b0       ??0pe_action_update_constraint@@QAE@XZ 350b00b0 f i rigidentity.obj
 0001:000af100       ??0CRigidEntity@@QAE@PAVCPhysicalWorld@@@Z 350b0100 f   rigidentity.obj
 0001:000af520       ?IsAwake@CRigidEntity@@UBEHH@Z 350b0520 f i rigidentity.obj
 0001:000af530       ?GetRigidBody@CRigidEntity@@UAEPAVRigidBody@@HH@Z 350b0530 f i rigidentity.obj
 0001:000af540       ?GetSleepSpeedChange@CRigidEntity@@UAEXHAAU?$Vec3_tpl@M@@0@Z 350b0540 f i rigidentity.obj
 0001:000af590       ?GetContactMatrix@CRigidEntity@@UAEXABU?$Vec3_tpl@M@@HAAU?$Matrix33_tpl@M@@@Z 350b0590 f i rigidentity.obj
 0001:000af5f0       ??1CRigidEntity@@UAE@XZ    350b05f0 f   rigidentity.obj
 0001:000af700       ?DetachAllContacts@CRigidEntity@@QAEXXZ 350b0700 f   rigidentity.obj
 0001:000af820       ?DetachPartContacts@CRigidEntity@@UAEXHHPAVCPhysicalEntity@@HH@Z 350b0820 f   rigidentity.obj
 0001:000af900       ?_AllocData@?$CryStackStringT@D$0CAA@@@QAEXI@Z 350b0900 f i rigidentity.obj
 0001:000af970       ?RemoveCollider@CRigidEntity@@UAEHPAVCPhysicalEntity@@_N@Z 350b0970 f   rigidentity.obj
 0001:000afb00       ?AddCollider@CRigidEntity@@UAEHPAVCPhysicalEntity@@@Z 350b0b00 f   rigidentity.obj
 0001:000afc40       ?RemoveContactPoint@CRigidEntity@@UAEHPAVCPhysicalEntity@@ABU?$Vec3_tpl@M@@M@Z 350b0c40 f   rigidentity.obj
 0001:000afd60       ?RegisterConstraint@CRigidEntity@@QAEHABU?$Vec3_tpl@M@@0HPAVCPhysicalEntity@@HHH@Z 350b0d60 f   rigidentity.obj
 0001:000b0080       ?VerifyExistingContacts@CRigidEntity@@QAEXM@Z 350b1080 f   rigidentity.obj
 0001:000b0210       ?CalcEnergy@CRigidEntity@@UAEMM@Z 350b1210 f   rigidentity.obj
 0001:000b0740       ?PushReceivedState@SRigidEntityNetStateHistory@@QAEXABUSRigidEntityNetSerialize@@@Z 350b1740 f   rigidentity.obj
 0001:000b07b0       ?PushReceivedSequenceDelta@SRigidEntityNetStateHistory@@QAEXE@Z 350b17b0 f   rigidentity.obj
 0001:000b0940       ?GetStateSnapshot@CRigidEntity@@UAEHAAVCStream@@MH@Z 350b1940 f   rigidentity.obj
 0001:000b0a40       ?Serialize@SRigidEntityNetSerialize@@QAEXV?$CSerializeWrapper@UISerialize@@@@@Z 350b1a40 f   rigidentity.obj
 0001:000b0af0       ?PostSetStateFromSnapshot@CRigidEntity@@UAEHXZ 350b1af0 f   rigidentity.obj
 0001:000b0ef0       ?CompactContactBlock@CRigidEntity@@QBEHPAUentity_contact@@HMHAAHAAPAU2@AAU?$Vec3_tpl@M@@AAMABU3@5@Z 350b1ef0 f   rigidentity.obj
 0001:000b1c50       ??$AllocPooledObj@Uentity_contact@@@CPhysicalWorld@@QAEPAUentity_contact@@AAPAU1@AAH1ACH@Z 350b2c50 f i rigidentity.obj
 0001:000b1d70       ??_GCWheeledVehicleEntity@@UAEPAXI@Z 350b2d70 f i wheeledvehicleentity.obj
 0001:000b1d70       ??_ECRigidEntity@@UAEPAXI@Z 350b2d70 f i rigidentity.obj
 0001:000b1d70       ??_GCRigidEntity@@UAEPAXI@Z 350b2d70 f i rigidentity.obj
 0001:000b1d70       ??_ECWheeledVehicleEntity@@UAEPAXI@Z 350b2d70 f i wheeledvehicleentity.obj
 0001:000b1da0       ?MoveConstrainedObjects@CRigidEntity@@QAEXABU?$Vec3_tpl@M@@ABU?$Quat_tpl@M@@@Z 350b2da0 f   rigidentity.obj
 0001:000b20e0       ?RemoveGeometry@CRigidEntity@@UAEXHH@Z 350b30e0 f   rigidentity.obj
 0001:000b22e0       ?SaveConstraintFrames@CRigidEntity@@QAEXH@Z 350b32e0 f   rigidentity.obj
 0001:000b25c0       ?RecomputeMassDistribution@CRigidEntity@@UAEXHH@Z 350b35c0 f   rigidentity.obj
 0001:000b3150       ?GetStatus@CRigidEntity@@UBEHPAUpe_status@@@Z 350b4150 f   rigidentity.obj
 0001:000b3a60       ?_Assign@?$CryStackStringT@D$0CAA@@@QAEXPBDI@Z 350b4a60 f i rigidentity.obj
 0001:000b3ad0       ?FakeRayCollision@CRigidEntity@@QAEXPAVCPhysicalEntity@@M@Z 350b4ad0 f   rigidentity.obj
 0001:000b46b0       ?GetPotentialColliders@CRigidEntity@@UAEHAAPAPAVCPhysicalEntity@@M@Z 350b56b0 f   rigidentity.obj
 0001:000b4d60       ?ProcessContactEvents@CRigidEntity@@QAEXPAUgeom_contact@@HH@Z 350b5d60 f   rigidentity.obj
 0001:000b5540       ?CheckForNewContacts@CRigidEntity@@QAEHPAUgeom_world_data@@PAUintersection_params@@AAHU?$Vec3_tpl@M@@HH@Z 350b6540 f   rigidentity.obj
 0001:000b7810       ?OnContactResolved@CRigidEntity@@UAEXPAUentity_contact@@HH@Z 350b8810 f   rigidentity.obj
 0001:000b7ae0       ?UpdateConstraints@CRigidEntity@@QAEXM@Z 350b8ae0 f   rigidentity.obj
 0001:000ba350       ?CapBodyVel@CRigidEntity@@QAEXXZ 350bb350 f   rigidentity.obj
 0001:000bab90       ?CheckContactConflicts@CRigidEntity@@QAEXPAUgeom_contact@@HH@Z 350bbb90 f   rigidentity.obj
 0001:000bb7e0       ?PostStepNotify@CRigidEntity@@QAEHMPAUpe_params_buoyancy@@H@Z 350bc7e0 f   rigidentity.obj
 0001:000bbb20       ?GetMaxTimeStep@CRigidEntity@@UAEMM@Z 350bcb20 f   rigidentity.obj
 0001:000bcc90       ?ArchiveContact@CRigidEntity@@QAEXPAUentity_contact@@MHM@Z 350bdc90 f   rigidentity.obj
 0001:000bd310       ?RegisterContacts@CRigidEntity@@UAEHMH@Z 350be310 f   rigidentity.obj
 0001:000bda60       ?StepBack@CRigidEntity@@UAEXM@Z 350bea60 f   rigidentity.obj
 0001:000be410       ?Update@CRigidEntity@@UAEHMM@Z 350bf410 f   rigidentity.obj
 0001:000bf8e0       ?SetNetworkAuthority@CRigidEntity@@UAEXHH@Z 350c08e0 f   rigidentity.obj
 0001:000bfa10       ?SetStateFromSnapshot@CRigidEntity@@UAEHV?$CSerializeWrapper@UISerialize@@@@H@Z 350c0a10 f   rigidentity.obj
 0001:000c0360       ?ReadContacts@CRigidEntity@@QAEHAAVCStream@@H@Z 350c1360 f   rigidentity.obj
 0001:000c0850       ?ApplyBuoyancy@CRigidEntity@@QAEXMABU?$Vec3_tpl@M@@PAUpe_params_buoyancy@@H@Z 350c1850 f   rigidentity.obj
 0001:000c2470       ?ExtractConstraintInfo@CRigidEntity@@QAEHH_KAAUpe_action_add_constraint@@@Z 350c3470 f   rigidentity.obj
 0001:000c2990       ?OnNeighbourSplit@CRigidEntity@@UAEXPAVCPhysicalEntity@@0@Z 350c3990 f   rigidentity.obj
 0001:000c3a00       ?AddGeometry@CRigidEntity@@UAEHPAUphys_geometry@@PAUpe_geomparams@@HH@Z 350c4a00 f   rigidentity.obj
 0001:000c4210       ?SetParams@CRigidEntity@@UAEHPAUpe_params@@H@Z 350c5210 f   rigidentity.obj
 0001:000c53f0       ?Action@CRigidEntity@@UAEHPAUpe_action@@H@Z 350c63f0 f   rigidentity.obj
 0001:000c8460       ?RegisterContactPoint@CRigidEntity@@QAEPAUentity_contact@@HABU?$Vec3_tpl@M@@PBUgeom_contact@@HHHHHMH0@Z 350c9460 f   rigidentity.obj
 0001:000c9530       ?ProcessCanopyContact@CRigidEntity@@QAEXPAUgeom_contact@@HMH@Z 350ca530 f   rigidentity.obj
 0001:000ca0b0       ?DelayedIntersect@CRigidEntity@@UAEXPAUgeom_contact@@HPAPAVCPhysicalEntity@@PAY01H@Z 350cb0b0 f   rigidentity.obj
 0001:000cad30       ?GetStateSnapshot@CRigidEntity@@UAEHV?$CSerializeWrapper@UISerialize@@@@MH@Z 350cbd30 f   rigidentity.obj
 0001:000cb410       ?SetStateFromSnapshot@CRigidEntity@@UAEHAAVCStream@@H@Z 350cc410 f   rigidentity.obj
 0001:000cc040       ?GetInterpolatedState@CRigidEntity@@QAE_NMAAUSRigidEntityNetSerialize@@@Z 350cd040 f   rigidentity.obj
 0001:000cc8c0       ?Format@?$CryStackStringT@D$0CAA@@@QAAAAV1@PBDZZ 350cd8c0 f i rigidentity.obj
 0001:000cc930       ?UpdateStateFromNetwork@CRigidEntity@@QAEXXZ 350cd930 f   rigidentity.obj
 0001:000cca20       ?DrawHelperInformation@CRigidEntity@@UAEXPAUIPhysRenderer@@H@Z 350cda20 f   rigidentity.obj
 0001:000cdb40       ?Step@CRigidEntity@@UAEHM@Z 350ceb40 f   rigidentity.obj
 0001:000d02d0       ??1CRopeEntity@@UAE@XZ     350d12d0 f   ropeentity.obj
 0001:000d0390       ?GetType@CRopeEntity@@UBE?AW4pe_type@@XZ 350d1390 f i ropeentity.obj
 0001:000d0390       ?GetType@CVoxelGeom@@UAEHXZ 350d1390 f i geoman.obj
 0001:000d03a0       ?GetMass@CRopeEntity@@UAEMH@Z 350d13a0 f i ropeentity.obj
 0001:000d03b0       ?GetMassInv@CRopeEntity@@UAEMXZ 350d13b0 f i ropeentity.obj
 0001:000d03c0       ?CalcEnergy@CRopeEntity@@UAEMM@Z 350d13c0 f i ropeentity.obj
 0001:000d03f0       ?GetLastTimeStep@CRopeEntity@@UAEMM@Z 350d13f0 f i ropeentity.obj
 0001:000d0400       ?GetMemoryStatistics@CRopeEntity@@UBEXPAVICrySizer@@@Z 350d1400 f   ropeentity.obj
 0001:000d0460       ?GetCheckPart@CPhysicalEntity@@QAEHH@Z 350d1460 f i ropeentity.obj
 0001:000d0580       ?GetDamping@CRopeEntity@@UAEMM@Z 350d1580 f i ropeentity.obj
 0001:000d05b0       ??_ECRopeEntity@@UAEPAXI@Z 350d15b0 f i ropeentity.obj
 0001:000d05b0       ??_GCRopeEntity@@UAEPAXI@Z 350d15b0 f i ropeentity.obj
 0001:000d05e0       ?Awake@CRopeEntity@@UAEHHH@Z 350d15e0 f   ropeentity.obj
 0001:000d07d0       ?GetStatus@CRopeEntity@@UBEHPAUpe_status@@@Z 350d17d0 f   ropeentity.obj
 0001:000d0b20       ?StartStep@CRopeEntity@@UAEXM@Z 350d1b20 f   ropeentity.obj
 0001:000d0bf0       ?GetMaxTimeStep@CRopeEntity@@UAEMM@Z 350d1bf0 f   ropeentity.obj
 0001:000d0c60       ?ZeroLengthStraighten@CRopeEntity@@QAEXM@Z 350d1c60 f   ropeentity.obj
 0001:000d1780       ?Solver@CRopeEntity@@QAEMMM@Z 350d2780 f   ropeentity.obj
 0001:000d3ab0       ?OnDelayedStep@CRopeEntity@@UAEXAAVCMemStreamA@@@Z 350d4ab0 f   ropeentity.obj
 0001:000d3c30       ?GetStateSnapshot@CRopeEntity@@UAEHAAVCStream@@MH@Z 350d4c30 f   ropeentity.obj
 0001:000d3c80       ?ComputeExtent@CRopeEntity@@UBEMAAUGeomQuery@@W4EGeomForm@@@Z 350d4c80 f   ropeentity.obj
 0001:000d3d60       ??$ReallocateList@USPrecompPartBV@@@@YAPAUSPrecompPartBV@@AAPAU0@HH_N1@Z 350d4d60 f i ropeentity.obj
 0001:000d3e10       ??0CRopeEntity@@QAE@PAVCPhysicalWorld@@@Z 350d4e10 f   ropeentity.obj
 0001:000d4320       ?AlertNeighbourhoodND@CRopeEntity@@UAEXH@Z 350d5320 f   ropeentity.obj
 0001:000d43f0       ?RecalcBBox@CRopeEntity@@QAEXXZ 350d53f0 f   ropeentity.obj
 0001:000d45f0       ?GetParams@CRopeEntity@@UBEHPAUpe_params@@@Z 350d55f0 f   ropeentity.obj
 0001:000d4a60       ?AllocSubVtx@CRopeEntity@@QAEXXZ 350d5a60 f   ropeentity.obj
 0001:000d4ba0       ?FillVtxContactData@CRopeEntity@@QAEXPAUrope_vtx@@HAAUSRopeCheckPart@@PAUgeom_contact@@@Z 350d5ba0 f   ropeentity.obj
 0001:000d4f10       ?CheckCollisions@CRopeEntity@@QAEXHPAUSRopeCheckPart@@HMM@Z 350d5f10 f   ropeentity.obj
 0001:000d6980       ?RegisterContacts@CRopeEntity@@UAEHMH@Z 350d7980 f   ropeentity.obj
 0001:000d8480       ?Update@CRopeEntity@@UAEHMM@Z 350d9480 f   ropeentity.obj
 0001:000d92d0       ?RayTrace@CRopeEntity@@UAEHAAUSRayTraceRes@@@Z 350da2d0 f   ropeentity.obj
 0001:000d98c0       ?ApplyVolumetricPressure@CRopeEntity@@UAEXABU?$Vec3_tpl@M@@MM@Z 350da8c0 f   ropeentity.obj
 0001:000d9cc0       ?OnNeighbourSplit@CRopeEntity@@UAEXPAVCPhysicalEntity@@0@Z 350dacc0 f   ropeentity.obj
 0001:000d9e70       ?SetStateFromSnapshot@CRopeEntity@@UAEHV?$CSerializeWrapper@UISerialize@@@@H@Z 350dae70 f   ropeentity.obj
 0001:000da8a0       ?DrawHelperInformation@CRopeEntity@@UAEXPAUIPhysRenderer@@H@Z 350db8a0 f   ropeentity.obj
 0001:000dae40       ?GetRandomPos@CRopeEntity@@UBEXAAURandomPos@@AAUGeomQuery@@W4EGeomForm@@@Z 350dbe40 f   ropeentity.obj
 0001:000db1b0       ?SetParams@CRopeEntity@@UAEHPAUpe_params@@H@Z 350dc1b0 f   ropeentity.obj
 0001:000dcd40       ?EnforceConstraints@CRopeEntity@@QAEXMABU?$Quat_tpl@M@@ABU?$Vec3_tpl@M@@MH@Z 350ddd40 f   ropeentity.obj
 0001:000ddfb0       ?Action@CRopeEntity@@UAEHPAUpe_action@@H@Z 350defb0 f   ropeentity.obj
 0001:000df1f0       ?StepSubdivided@CRopeEntity@@QAEXMPAUSRopeCheckPart@@HM@Z 350e01f0 f   ropeentity.obj
 0001:000e3c90       ?ApplyStiffness@CRopeEntity@@QAEXMHABU?$Quat_tpl@M@@ABU?$Vec3_tpl@M@@M@Z 350e4c90 f   ropeentity.obj
 0001:000e4f00       ?Step@CRopeEntity@@UAEHM@Z 350e5f00 f   ropeentity.obj
 0001:000ea730       ?GetStateSnapshot@CRopeEntity@@UAEHV?$CSerializeWrapper@UISerialize@@@@MH@Z 350eb730 f   ropeentity.obj
 0001:000eac00       ?GetRigidBodyData@CRopeEntity@@UAEPAVRigidBody@@PAV2@H@Z 350ebc00 f   ropeentity.obj
 0001:000eb090       ?GetLocTransform@CRopeEntity@@UAEXHAAU?$Vec3_tpl@M@@AAU?$Quat_tpl@M@@AAM@Z 350ec090 f   ropeentity.obj
 0001:000eb370       ?RemoveCore@CSoftEntity@@QAEXXZ 350ec370 f   softentity.obj
 0001:000eb3c0       ?AlertNeighbourhoodND@CSoftEntity@@UAEXH@Z 350ec3c0 f   softentity.obj
 0001:000eb480       ?Awake@CSoftEntity@@UAEHHH@Z 350ec480 f   softentity.obj
 0001:000eb4d0       ?GetParams@CSoftEntity@@UBEHPAUpe_params@@@Z 350ec4d0 f   softentity.obj
 0001:000eb690       ?StartStep@CSoftEntity@@UAEXM@Z 350ec690 f   softentity.obj
 0001:000eb6b0       ?GetStateSnapshot@CSoftEntity@@UAEHAAVCStream@@MH@Z 350ec6b0 f   softentity.obj
 0001:000eb6b0       ?HasPartContactsWith@CPhysicalEntity@@UAEHPAV1@HH@Z 350ec6b0 f   livingentity.obj
 0001:000eb6c0       ?GetMemoryStatistics@CSoftEntity@@UBEXPAVICrySizer@@@Z 350ec6c0 f   softentity.obj
 0001:000eb760       ??0CSoftEntity@@QAE@PAVCPhysicalWorld@@@Z 350ec760 f   softentity.obj
 0001:000eba20       ?GetType@CSoftEntity@@UBE?AW4pe_type@@XZ 350eca20 f i softentity.obj
 0001:000eba30       ?IsAwake@CSoftEntity@@UBEHH@Z 350eca30 f i softentity.obj
 0001:000eba30       ?IsAwake@CRopeEntity@@UBEHH@Z 350eca30 f i ropeentity.obj
 0001:000eba40       ?GetMass@CSoftEntity@@UAEMH@Z 350eca40 f i softentity.obj
 0001:000eba60       ?GetStatus@CSoftEntity@@UBEHPAUpe_status@@@Z 350eca60 f   softentity.obj
 0001:000ebec0       ?GetMaxTimeStep@CSoftEntity@@UAEMM@Z 350ecec0 f   softentity.obj
 0001:000ebf30       ?OnDelayedStep@CSoftEntity@@UAEXAAVCMemStreamA@@@Z 350ecf30 f   softentity.obj
 0001:000ec3d0       ?RecalcTriNormal@CTriMesh@@QAEXH@Z 350ed3d0 f i softentity.obj
 0001:000ec520       ??1CSoftEntity@@UAE@XZ     350ed520 f   softentity.obj
 0001:000ec680       ?BakeCurrentPose@CSoftEntity@@QAEXXZ 350ed680 f   softentity.obj
 0001:000ecce0       ?RemoveGeometry@CSoftEntity@@UAEXHH@Z 350edce0 f   softentity.obj
 0001:000ece90       ?AttachPoints@CSoftEntity@@QAEXPAUpe_action_attach_points@@PAVCPhysicalEntity@@HMMHABU?$Vec3_tpl@M@@ABU?$Quat_tpl@M@@@Z 350ede90 f   softentity.obj
 0001:000ed1a0       ?Action@CSoftEntity@@UAEHPAUpe_action@@H@Z 350ee1a0 f   softentity.obj
 0001:000f0160       ?ApplyVolumetricPressure@CSoftEntity@@UAEXABU?$Vec3_tpl@M@@MM@Z 350f1160 f   softentity.obj
 0001:000f06e0       ?RayTrace@CSoftEntity@@UAEHAAUSRayTraceRes@@@Z 350f16e0 f   softentity.obj
 0001:000f0b00       ?GetStateSnapshot@CSoftEntity@@UAEHV?$CSerializeWrapper@UISerialize@@@@MH@Z 350f1b00 f   softentity.obj
 0001:000f0bf0       ?SetStateFromSnapshot@CSoftEntity@@UAEHV?$CSerializeWrapper@UISerialize@@@@H@Z 350f1bf0 f   softentity.obj
 0001:000f0ea0       ?DrawHelperInformation@CSoftEntity@@UAEXPAUIPhysRenderer@@H@Z 350f1ea0 f   softentity.obj
 0001:000f1340       ??_ECSoftEntity@@UAEPAXI@Z 350f2340 f i softentity.obj
 0001:000f1340       ??_GCSoftEntity@@UAEPAXI@Z 350f2340 f i softentity.obj
 0001:000f1370       ?AddGeometry@CSoftEntity@@UAEHPAUphys_geometry@@PAUpe_geomparams@@HH@Z 350f2370 f   softentity.obj
 0001:000f3790       ?SetParams@CSoftEntity@@UAEHPAUpe_params@@H@Z 350f4790 f   softentity.obj
 0001:000f47f0       ?StepInner@CSoftEntity@@QAEXMHPAUcheck_part@@HABUplane@primitives@@ABU?$Vec3_tpl@M@@M2ABU?$Quat_tpl@M@@PAUse_vertex@@@Z 350f57f0 f   softentity.obj
 0001:000fb7e0       ?Step@CSoftEntity@@UAEHM@Z 350fc7e0 f   softentity.obj
 0001:000ff380       ?GetType@CSphereGeom@@UAEHXZ 35100380 f i physicalentity.obj
 0001:000ff380       ?GetType@CLivingEntity@@UBE?AW4pe_type@@XZ 35100380 f i livingentity.obj
 0001:000ff380       ?GetType@CHeightfieldBV@@UAEHXZ 35100380 f i waterman.obj
 0001:000ff390       ?MaxPrimsInNode@CHeightfieldBV@@UAEHXZ 35100390 f i waterman.obj
 0001:000ff3a0       ?MarkPool@CDummyMemReplay@@UAEXHIPAXIPBD@Z 351003a0 f i articulatedentity.obj
 0001:000ff3a0       ?GetNodeBV@CRayBV@@UAEXAAPAUBV@@ABU?$Vec3_tpl@M@@MHH@Z 351003a0 f i livingentity.obj
 0001:000ff3a0       ?DetachPartContacts@CPhysicalEntity@@UAEXHHPAV1@HH@Z 351003a0 f i livingentity.obj
 0001:000ff3a0       ?GetNodeBV@CHeightfieldBV@@UAEXAAPAUBV@@ABU?$Vec3_tpl@M@@MHH@Z 351003a0 f i waterman.obj
 0001:000ff3b0       ??_GCHeightfieldBV@@UAEPAXI@Z 351003b0 f i waterman.obj
 0001:000ff3b0       ??_ECHeightfieldBV@@UAEPAXI@Z 351003b0 f i waterman.obj
 0001:000ff3f0       ?GetPrimitiveId@CTriMesh@@UAEHHH@Z 351003f0 f i waterman.obj
 0001:000ff410       ?GetForeignIdx@CTriMesh@@UAEHH@Z 35100410 f i waterman.obj
 0001:000ff430       ?GetNormal@CTriMesh@@UAE?AU?$Vec3_tpl@M@@HABU2@@Z 35100430 f i waterman.obj
 0001:000ff460       ?GetPrimitiveCount@CTriMesh@@UAEHXZ 35100460 f i waterman.obj
 0001:000ff470       ?GetSubtractionsCount@CTriMesh@@UAEHXZ 35100470 f i waterman.obj
 0001:000ff480       ?GetTriMesh@CTriMesh@@UAEPAUIGeometry@@H@Z 35100480 f i waterman.obj
 0001:000ff4e0       ?GetErrorCount@CTriMesh@@UAEHXZ 351004e0 f i waterman.obj
 0001:000ff4f0       ?GetForeignData@CTriMesh@@UAEPAXH@Z 351004f0 f i waterman.obj
 0001:000ff520       ?SetForeignData@CTriMesh@@UAEXPAXH@Z 35100520 f i waterman.obj
 0001:000ff560       ?DestroyAuxilaryMeshData@CTriMesh@@UAEXH@Z 35100560 f i waterman.obj
 0001:000ff5d0       ?GetBVTree@CHeightfield@@UAEPAVCBVTree@@XZ 351005d0 f i waterman.obj
 0001:000ff5e0       ?GetData@CHeightfield@@UAEPBUprimitive@primitives@@XZ 351005e0 f i waterman.obj
 0001:000ff5f0       ??_ECHeightfield@@UAEPAXI@Z 351005f0 f i waterman.obj
 0001:000ff5f0       ??_GCHeightfield@@UAEPAXI@Z 351005f0 f i waterman.obj
 0001:000ff650       ?GetParams@CWaterMan@@QAEHPAUpe_params@@@Z 35100650 f   waterman.obj
 0001:000ff6c0       ?GetBBox@CTriMesh@@UAEXPAUbox@primitives@@@Z 351006c0 f i waterman.obj
 0001:000ff720       ?GetBBox@CTriMesh@@UAEXPAUbox@primitives@@H@Z 35100720 f i waterman.obj
 0001:000ff790       ?Load@CTriMesh@@UAEXAAVCMemStream@@@Z 35100790 f i waterman.obj
 0001:000ff7d0       ?GetCenter@CHeightfield@@UAE?AU?$Vec3_tpl@M@@XZ 351007d0 f i waterman.obj
 0001:000ff8c0       ??0CWaterMan@@QAE@PAVCPhysicalWorld@@@Z 351008c0 f   waterman.obj
 0001:000ffa10       ??1CWaterMan@@QAE@XZ       35100a10 f   waterman.obj
 0001:000ffac0       ?GetStatus@CWaterMan@@QAEHPAUpe_status@@@Z 35100ac0 f   waterman.obj
 0001:000ffc20       ?TimeStep@CWaterMan@@QAEXM@Z 35100c20 f   waterman.obj
 0001:001002a0       ??4heightfield@primitives@@QAEAAU01@ABU01@@Z 351012a0 f i waterman.obj
 0001:00100310       ?check_cell@jgrid_checker@@QAEHABU?$Vec2_tpl@H@@AAH@Z 35101310 f i waterman.obj
 0001:001008e0       ?MarkCellInteriorQueue@jgrid_checker@@QAEXH@Z 351018e0 f i waterman.obj
 0001:00100a70       ?GetPrimitive@CHeightfield@@UAEHHPAUprimitive@primitives@@@Z 35101a70 f i waterman.obj
 0001:00100a90       ?OnWaterHit@CWaterMan@@QAEXABU?$Vec3_tpl@M@@0@Z 35101a90 f   waterman.obj
 0001:00100ce0       ??0CHeightfield@@QAE@XZ    35101ce0 f i waterman.obj
 0001:00100d20       ?SetViewerPos@CWaterMan@@QAEXABU?$Vec3_tpl@M@@H@Z 35101d20 f   waterman.obj
 0001:00101720       ?DrawHelpers@CWaterMan@@QAEXPAUIPhysRenderer@@@Z 35102720 f   waterman.obj
 0001:00101af0       ??$DrawRayOnGrid@Ujgrid_checker@@@@YAHPAUgrid@primitives@@AAU?$Vec3_tpl@M@@1AAUjgrid_checker@@@Z 35102af0 f i waterman.obj
 0001:00102150       ?SetParams@CWaterMan@@QAEHPAUpe_params@@@Z 35103150 f   waterman.obj
 0001:00102510       ?OnWaterInteraction@CWaterMan@@QAEXPAVCPhysicalEntity@@@Z 35103510 f   waterman.obj
 0001:00105800       ?AlertNeighbourhoodND@CWheeledVehicleEntity@@UAEXH@Z 35106800 f   wheeledvehicleentity.obj
 0001:00105860       ?OnContactResolved@CWheeledVehicleEntity@@UAEXPAUentity_contact@@HH@Z 35106860 f   wheeledvehicleentity.obj
 0001:00105890       ?GetMaxTimeStep@CWheeledVehicleEntity@@UAEMM@Z 35106890 f   wheeledvehicleentity.obj
 0001:00105900       ?GetDamping@CWheeledVehicleEntity@@UAEMM@Z 35106900 f   wheeledvehicleentity.obj
 0001:00105940       ?HasContactsWith@CWheeledVehicleEntity@@UAEHPAVCPhysicalEntity@@@Z 35106940 f   wheeledvehicleentity.obj
 0001:00105990       ?HasPartContactsWith@CWheeledVehicleEntity@@UAEHPAVCPhysicalEntity@@HH@Z 35106990 f   wheeledvehicleentity.obj
 0001:00105a30       ?RemoveCollider@CWheeledVehicleEntity@@UAEHPAVCPhysicalEntity@@_N@Z 35106a30 f   wheeledvehicleentity.obj
 0001:00105a90       ?Update@CWheeledVehicleEntity@@UAEHMM@Z 35106a90 f   wheeledvehicleentity.obj
 0001:00105c30       ?GetMemoryStatistics@CWheeledVehicleEntity@@UBEXPAVICrySizer@@@Z 35106c30 f   wheeledvehicleentity.obj
 0001:00105c70       ?GetParams@CWheeledVehicleEntity@@UBEHPAUpe_params@@@Z 35106c70 f   wheeledvehicleentity.obj
 0001:00105fa0       ?ComputeBBox@CWheeledVehicleEntity@@UAEXPAU?$Vec3_tpl@M@@H@Z 35106fa0 f   wheeledvehicleentity.obj
 0001:00106050       ?ComputeDrivingTorque@CWheeledVehicleEntity@@QAEMM@Z 35107050 f   wheeledvehicleentity.obj
 0001:00106560       ?GetStateSnapshot@CWheeledVehicleEntity@@UAEHAAVCStream@@MH@Z 35107560 f   wheeledvehicleentity.obj
 0001:00106660       ?SetStateFromSnapshot@CWheeledVehicleEntity@@UAEHAAVCStream@@H@Z 35107660 f   wheeledvehicleentity.obj
 0001:00106840       ?Serialize@SWheeledVehicleEntityNetSerialize@@QAEXV?$CSerializeWrapper@UISerialize@@@@H@Z 35107840 f   wheeledvehicleentity.obj
 0001:001068d0       ?GetStateSnapshot@CWheeledVehicleEntity@@UAEHV?$CSerializeWrapper@UISerialize@@@@MH@Z 351078d0 f   wheeledvehicleentity.obj
 0001:00106970       ?DrawHelperInformation@CWheeledVehicleEntity@@UAEXPAUIPhysRenderer@@H@Z 35107970 f   wheeledvehicleentity.obj
 0001:00106a90       ??0pe_cargeomparams@@QAE@AAUpe_geomparams@@@Z 35107a90 f i wheeledvehicleentity.obj
 0001:00106bd0       ?SetParams@CWheeledVehicleEntity@@UAEHPAUpe_params@@H@Z 35107bd0 f   wheeledvehicleentity.obj
 0001:00107790       ?RemoveGeometry@CWheeledVehicleEntity@@UAEXHH@Z 35108790 f   wheeledvehicleentity.obj
 0001:00107910       ?AddAdditionalImpulses@CWheeledVehicleEntity@@UAEXM@Z 35108910 f   wheeledvehicleentity.obj
 0001:001093f0       ?RegisterContacts@CWheeledVehicleEntity@@UAEHMH@Z 3510a3f0 f   wheeledvehicleentity.obj
 0001:00109820       ?SetStateFromSnapshot@CWheeledVehicleEntity@@UAEHV?$CSerializeWrapper@UISerialize@@@@H@Z 3510a820 f   wheeledvehicleentity.obj
 0001:00109910       ??0CWheeledVehicleEntity@@QAE@PAVCPhysicalWorld@@@Z 3510a910 f   wheeledvehicleentity.obj
 0001:00109b30       ?RecalcSuspStiffness@CWheeledVehicleEntity@@QAEXXZ 3510ab30 f   wheeledvehicleentity.obj
 0001:0010a380       ?AddGeometry@CWheeledVehicleEntity@@UAEHPAUphys_geometry@@PAUpe_geomparams@@HH@Z 3510b380 f   wheeledvehicleentity.obj
 0001:0010b100       ?Action@CWheeledVehicleEntity@@UAEHPAUpe_action@@H@Z 3510c100 f   wheeledvehicleentity.obj
 0001:0010bc10       ?GetStatus@CWheeledVehicleEntity@@UBEHPAUpe_status@@@Z 3510cc10 f   wheeledvehicleentity.obj
 0001:0010ce30       ?CheckAdditionalGeometry@CWheeledVehicleEntity@@UAEXM@Z 3510de30 f   wheeledvehicleentity.obj
 0001:001121b0       ?line_seg_inters@@YAHPBU?$Vec2_tpl@M@@0PAU1@@Z 351131b0 f i boolean2d.obj
 0001:001124a0       ?get_cell@@YAAAU?$Vec2_tpl@H@@ABU?$Vec2_tpl@M@@0AAU1@@Z 351134a0 f i boolean2d.obj
 0001:00112500       ?get_rect@@YAXABU?$Vec2_tpl@H@@0PAU1@0@Z 35113500 f i boolean2d.obj
 0001:001125b0       ?check_if_inside@@YAHHAAU?$Vec2_tpl@H@@ABU1@PBU?$Vec2_tpl@M@@ABU2@@Z 351135b0 f i boolean2d.obj
 0001:00112760       ?boolean2d@@YAHW4booltype@@PAU?$Vec2_tpl@M@@H1HHAAPAU2@AAPAH@Z 35113760 f   boolean2d.obj
 0001:00113c80       ??_Ebop_meshupdate_thunk@@UAEPAXI@Z 35114c80 f i boolean3d.obj
 0001:00113c80       ??_Gbop_meshupdate_thunk@@UAEPAXI@Z 35114c80 f i boolean3d.obj
 0001:00113cc0       ??1bop_meshupdate@@UAE@XZ  35114cc0 f   boolean3d.obj
 0001:00113da0       ?TriangulatePolyBruteforce@@YAHPAU?$Vec2_tpl@M@@HPAHH@Z 35114da0 f   boolean3d.obj
 0001:00114430       ?TriangulatePoly@@YAHPAU?$Vec2_tpl@M@@HPAHH@Z 35115430 f   boolean3d.obj
 0001:001157c0       ??$ReallocateList@U?$Vec3_tpl@M@@@@YAPAU?$Vec3_tpl@M@@AAPAU0@HH_N1@Z 351167c0 f i boolean3d.obj
 0001:001157c0       ??$ReallocateList@Utrinfo@@@@YAPAUtrinfo@@AAPAU0@HH_N1@Z 351167c0 f i boolean3d.obj
 0001:00115870       ??_Ebop_meshupdate@@UAEPAXI@Z 35116870 f i boolean3d.obj
 0001:00115870       ??_Gbop_meshupdate@@UAEPAXI@Z 35116870 f i boolean3d.obj
 0001:001158a0       ?insertBorderVtx@@YAXPAUtessvtx@@HHABU?$Vec3_tpl@M@@H@Z 351168a0 f   boolean3d.obj
 0001:00115d10       ?Subtract@CTriMesh@@UAEHPAUIGeometry@@PAUgeom_world_data@@1H@Z 35116d10 f   boolean3d.obj
 0001:0011d180       ?PIII_Mult00_6x6_6x6@@YAXPAM00@Z 3511e180 f   matrixnm.obj
 0001:0011d5b0       ?zero@?$matrix_tpl@N@@QAEAAV1@XZ 3511e5b0 f i matrixnm.obj
 0001:0011d600       ?LUdecomposition@?$matrix_tpl@M@@QBEHAAPAMAAPAH@Z 3511e600 f i matrixnm.obj
 0001:0011db10       ?solveAx_b@?$matrix_tpl@M@@QBEHPAM00PAH@Z 3511eb10 f i matrixnm.obj
 0001:0011de30       ?identity@?$matrix_tpl@N@@QAEAAV1@XZ 3511ee30 f i matrixnm.obj
 0001:0011dec0       ?T@?$matrix_tpl@M@@QBE?AV1@XZ 3511eec0 f i matrixnm.obj
 0001:0011e130       ?jacobi_transformation@?$matrix_tpl@M@@QBEHAAV1@PAMM@Z 3511f130 f i matrixnm.obj
 0001:0011ecb0       ?jacobi_transformation@?$matrix_tpl@N@@QBEHAAV1@PANN@Z 3511fcb0 f i matrixnm.obj
 0001:0011f670       ?transpose@?$matrix_tpl@M@@QAEAAV1@XZ 35120670 f i matrixnm.obj
 0001:0011f820       ?invert@?$matrix_tpl@M@@QAEAAV1@XZ 35120820 f i matrixnm.obj
 0001:0011fde0       ?qhull2d@@YAHPAUptitem2d@@HPAUedgeitem@@@Z 35120de0 f   qhull.obj
 0001:00120870       ?associate_ptlist_with_trilist@@YAXPAUptitem@@PAUqhtritem@@0V?$strided_pointer@UVec3mem@@@@@Z 35121870 f   qhull.obj
 0001:001209d0       ?qhull@@YAHV?$strided_pointer@U?$Vec3_tpl@M@@@@HAAPAHP6APAXI@Z@Z 351219d0 f   qhull.obj
 0001:001230a0       ?compute_projection_integrals@@YAXPAU?$Vec3_tpl@N@@QAN@Z 351240a0 f   utils.obj
 0001:00123360       ??0SOcclusionCubeMap@@QAE@XZ 35124360 f   utils.obj
 0001:001233a0       ?FreeTextures@SOcclusionCubeMap@@QAEXXZ 351243a0 f   utils.obj
 0001:001233e0       ?get_cubemap_cell_buddy@@YAHHHH@Z 351243e0 f i utils.obj
 0001:001234c0       ?GrowAndCompareCubemaps@@YAXPAUSOcclusionCubeMap@@0HAAH1@Z 351244c0 f   utils.obj
 0001:00123760       ?crop_polygon_with_plane@@YAHPBU?$Vec3_tpl@M@@HPAU1@ABU1@M@Z 35124760 f   utils.obj
 0001:00123b10       ?bin2ascii@@YAHPBEHPAE@Z   35124b10 f   utils.obj
 0001:00123d40       ?ascii2bin@@YAHPBEHPAE@Z   35124d40 f   utils.obj
 0001:00123f40       ?WritePacked@@YAXAAVCStream@@H@Z 35124f40 f   utils.obj
 0001:00123f70       ?ReadPacked@@YAXAAVCStream@@AAH@Z 35124f70 f   utils.obj
 0001:00123fa0       ?WriteCompressedPos@@YAXAAVCStream@@ABU?$Vec3_tpl@M@@_N@Z 35124fa0 f   utils.obj
 0001:00124070       ?Free@SOcclusionCubeMap@@QAEXXZ 35125070 f   utils.obj
 0001:00124070       ??1SOcclusionCubeMap@@QAE@XZ 35125070 f   utils.obj
 0001:001240a0       ?Allocate@SOcclusionCubeMap@@QAEXH@Z 351250a0 f   utils.obj
 0001:00124140       ?Reset@SOcclusionCubeMap@@QAEXXZ 35125140 f   utils.obj
 0001:00124180       ?ProcessRmin@SOcclusionCubeMap@@QAEXXZ 35125180 f   utils.obj
 0001:00124290       ?GetMemoryStatistics@SOcclusionCubeMap@@QAEXPAVICrySizer@@@Z 35125290 f   utils.obj
 0001:001242d0       ?DebugDrawToScreen@SOcclusionCubeMap@@QAEXMMM@Z 351252d0 f   utils.obj
 0001:00124830       ?Raster@?$Rasteriser@$02@@SAXPBU?$Vec3_tpl@M@@HPAUSOcclusionCubeMap@@@Z 35125830 f i utils.obj
 0001:00125880       ?Raster@?$Rasteriser@$03@@SAXPBU?$Vec3_tpl@M@@HPAUSOcclusionCubeMap@@@Z 35126880 f i utils.obj
 0001:00126a30       ?Raster@?$Rasteriser@$07@@SAXPBU?$Vec3_tpl@M@@HPAUSOcclusionCubeMap@@@Z 35127a30 f i utils.obj
 0001:00127f10       ?compute_face_integrals@@YAXPAU?$Vec3_tpl@N@@U1@QAN@Z 35128f10 f   utils.obj
 0001:001280e0       ?ComputeMassProperties@@YANV?$strided_pointer@$$CBU?$Vec3_tpl@M@@@@PBHHAAU?$Vec3_tpl@N@@AAU?$Matrix33_tpl@N@@@Z 351290e0 f   utils.obj
 0001:00128630       ?ChoosePrimitiveForMesh@@YAHV?$strided_pointer@$$CBU?$Vec3_tpl@M@@@@V?$strided_pointer@$$CBG@@HPBU?$Vec3_tpl@N@@ABU3@HMAAPAUprimitive@primitives@@@Z 35129630 f   utils.obj
 0001:0012c4b0       ?get_xqs_from_matrices@@YAXPAU?$Matrix34_tpl@M@@PAU?$Matrix33_tpl@M@@AAU?$Vec3_tpl@M@@AAU?$Quat_tpl@M@@AAM@Z 3512d4b0 f   utils.obj
 0001:0012ca20       ?CalcMediumResistance@@YAXPBU?$Vec3_tpl@M@@HABU1@ABUplane@primitives@@111AAU1@3@Z 3512da20 f   utils.obj
 0001:0012dbe0       ?CoverPolygonWithCircles@@YAHV?$strided_pointer@U?$Vec2_tpl@M@@@@H_NABU?$Vec2_tpl@M@@AAPAU2@AAPAMM@Z 3512ebe0 f   utils.obj
 0001:0012e600       ?RasterizePolygonIntoCubemap@@YAXPBU?$Vec3_tpl@M@@HHPAUSOcclusionCubeMap@@@Z 3512f600 f   utils.obj
 0001:0012e670       ?Init@SOcclusionCubeMap@@QAEXHMM@Z 3512f670 f   utils.obj
 0001:0012e720       ?ExtrudeBox@@YAXPBUbox@primitives@@ABU?$Vec3_tpl@M@@MPAU12@@Z 3512f720 f   utils.obj
 0001:0012ed90       ?getCompressedQuat@@YA_NABU?$Quat_tpl@M@@AAU?$Vec3_tpl@F@@@Z 3512fd90 f   utils.obj
 0001:0012f1b0       ?WriteCompressedQuat@@YAXAAVCStream@@ABU?$Quat_tpl@M@@@Z 351301b0 f   utils.obj
 0001:0012f1d0       ?ReadCompressedQuat@@YAXAAVCStream@@AAU?$Quat_tpl@M@@@Z 351301d0 f   utils.obj
 0001:0012f450       ?SetGeomConvex@CAABBTree@@UAEXXZ 35130450 f   aabbtree.obj
 0001:0012f480       ?ReleaseLastSweptBVs@CAABBTree@@UAEXH@Z 35130480 f   aabbtree.obj
 0001:0012f4a0       ?GetNodeContents@CAABBTree@@UAEHHPAUBV@@HHPAUgeometry_under_test@@1@Z 351304a0 f   aabbtree.obj
 0001:0012f500       ?GetRootNodeDim@CAABBTree@@QAEXAAU?$Vec3_tpl@M@@0@Z 35130500 f i aabbtree.obj
 0001:0012f730       ?GetBBox@CAABBTree@@UAEXPAUbox@primitives@@@Z 35130730 f   aabbtree.obj
 0001:0012f7a0       ?GetNodeBV@CAABBTree@@UAEXAAPAUBV@@HH@Z 351307a0 f   aabbtree.obj
 0001:0012f840       ?GetNodeBV@CAABBTree@@UAEXAAPAUBV@@ABU?$Vec3_tpl@M@@MHH@Z 35130840 f   aabbtree.obj
 0001:0012f8e0       ?SplitPriority@CAABBTree@@UAEMPBUBV@@@Z 351308e0 f   aabbtree.obj
 0001:0012f910       ?GetNodeChildrenBVs@CAABBTree@@UAEXABU?$Matrix33_tpl@M@@ABU?$Vec3_tpl@M@@MPBUBV@@AAPAU4@3H@Z 35130910 f   aabbtree.obj
 0001:0012fe50       ?GetNodeChildrenBVs@CAABBTree@@UAEXPBUBV@@AAPAU2@1H@Z 35130e50 f   aabbtree.obj
 0001:00130480       ?GetNodeChildrenBVs@CAABBTree@@UAEXPBUBV@@ABU?$Vec3_tpl@M@@MAAPAU2@2H@Z 35131480 f   aabbtree.obj
 0001:00130b40       ?MarkUsedTriangle@CAABBTree@@UAEXHPAUgeometry_under_test@@@Z 35131b40 f   aabbtree.obj
 0001:00130bf0       ?PrepareForIntersectionTest@CAABBTree@@UAEHPAUgeometry_under_test@@PAVCGeometry@@0@Z 35131bf0 f   aabbtree.obj
 0001:00130cf0       ?GetMemoryStatistics@CAABBTree@@UAEXPAVICrySizer@@@Z 35131cf0 f   aabbtree.obj
 0001:00130d70       ?SanityCheck@CAABBTree@@UAEHXZ 35131d70 f   aabbtree.obj
 0001:00130d80       ?SetParams@CAABBTree@@QAEXHHMABU?$Matrix33_tpl@M@@H@Z 35131d80 f   aabbtree.obj
 0001:00130e50       ?BuildNode@CAABBTree@@QAEMHHHU?$Vec3_tpl@M@@0PAY02U2@H@Z 35131e50 f   aabbtree.obj
 0001:00131fd0       ?Save@CAABBTree@@UAEXAAVCMemStream@@@Z 35132fd0 f   aabbtree.obj
 0001:001321d0       ?Load@CAABBTree@@UAEXAAVCMemStream@@PAVCGeometry@@@Z 351331d0 f   aabbtree.obj
 0001:00132540       ?Build@CAABBTree@@UAEMPAVCGeometry@@@Z 35133540 f   aabbtree.obj
 0001:00132e40       ?GetNodeBV@CAABBTree@@UAEXABU?$Matrix33_tpl@M@@ABU?$Vec3_tpl@M@@MAAPAUBV@@HH@Z 35133e40 f   aabbtree.obj
 0001:00133140       ?PrepareForIntersectionTest@CBoxGeom@@UAEHPAUgeometry_under_test@@PAVCGeometry@@0_N@Z 35134140 f   boxgeom.obj
 0001:00133200       ?GetMemoryStatistics@CBoxGeom@@UAEXPAVICrySizer@@@Z 35134200 f   boxgeom.obj
 0001:00133220       ?PointInsideStatus@CBoxGeom@@UAEHABU?$Vec3_tpl@M@@@Z 35134220 f   boxgeom.obj
 0001:00133340       ?GetFeature@CBoxGeom@@UAEHHHPAU?$Vec3_tpl@M@@@Z 35134340 f   boxgeom.obj
 0001:00133a90       ?BuildTriMesh@CBoxGeom@@QAEXAAVCTriMesh@@H@Z 35134a90 f   boxgeom.obj
 0001:00134200       ?CalcVolumetricPressure@CBoxGeom@@UAEXPAUgeom_world_data@@ABU?$Vec3_tpl@M@@MM1AAU3@2@Z 35135200 f   boxgeom.obj
 0001:00134270       ?CalculateBuoyancy@CBoxGeom@@UAEMPBUplane@primitives@@PBUgeom_world_data@@AAU?$Vec3_tpl@M@@@Z 35135270 f   boxgeom.obj
 0001:001342d0       ?DrawWireframe@CBoxGeom@@UAEXPAUIPhysRenderer@@PAUgeom_world_data@@HH@Z 351352d0 f   boxgeom.obj
 0001:001343a0       ?CreateBox@CBoxGeom@@QAEPAV1@PAUbox@primitives@@@Z 351353a0 f   boxgeom.obj
 0001:001344b0       ?FindClosestPoint@CBoxGeom@@UAEHPAUgeom_world_data@@AAH1ABU?$Vec3_tpl@M@@2PAU3@H@Z 351354b0 f   boxgeom.obj
 0001:00135af0       ?UnprojectSphere@CBoxGeom@@UAEHU?$Vec3_tpl@M@@MMPAUcontact@@@Z 35136af0 f   boxgeom.obj
 0001:00135be0       ?Save@CBoxGeom@@UAEXAAVCMemStream@@@Z 35136be0 f   boxgeom.obj
 0001:00135c40       ?Load@CBoxGeom@@UAEXAAVCMemStream@@@Z 35136c40 f   boxgeom.obj
 0001:00135ca0       ?CalcPhysicalProperties@CBoxGeom@@UAEHPAUphys_geometry@@@Z 35136ca0 f   boxgeom.obj
 0001:00135f80       ?PrepareBox@CBoxGeom@@QAEXPAUbox@primitives@@PAUgeometry_under_test@@@Z 35136f80 f   boxgeom.obj
 0001:001362c0       ?PreparePrimitive@CBoxGeom@@UAEHPAUgeom_world_data@@AAPAUprimitive@primitives@@H@Z 351372c0 f   boxgeom.obj
 0001:00136610       ?GetPrimitiveList@CBoxGeom@@UAEHHHHPAUprimitive@primitives@@HPAUgeometry_under_test@@10PAD@Z 35137610 f   boxgeom.obj
 0001:001368a0       ?GetUnprojectionCandidates@CBoxGeom@@UAEHHPBUcontact@@AAPAUprimitive@primitives@@AAPAHPAUgeometry_under_test@@@Z 351378a0 f   boxgeom.obj
 0001:00136f70       ?PreparePolygon@CBoxGeom@@UAEHPAUcoord_plane@primitives@@HHPAUgeometry_under_test@@AAPAU?$Vec2_tpl@M@@AAPAH3@Z 35137f70 f   boxgeom.obj
 0001:00137720       ?PreparePolyline@CBoxGeom@@UAEHPAUcoord_plane@primitives@@HHPAUgeometry_under_test@@AAPAU?$Vec2_tpl@M@@AAPAH3@Z 35138720 f   boxgeom.obj
 0001:00137d80       ?CalculateMediumResistance@CBoxGeom@@UAEXPBUplane@primitives@@PBUgeom_world_data@@AAU?$Vec3_tpl@M@@2@Z 35138d80 f   boxgeom.obj
 0001:00138580       ?DrawToOcclusionCubemap@CBoxGeom@@UAEHPBUgeom_world_data@@HHHPAUSOcclusionCubeMap@@@Z 35139580 f   boxgeom.obj
 0001:00138dc0       ?PrepareForIntersectionTest@CCapsuleGeom@@UAEHPAUgeometry_under_test@@PAVCGeometry@@0_N@Z 35139dc0 f   capsulegeom.obj
 0001:00138e00       ?PointInsideStatus@CCapsuleGeom@@UAEHABU?$Vec3_tpl@M@@@Z 35139e00 f   capsulegeom.obj
 0001:00138f80       ?CalculateBuoyancy@CCapsuleGeom@@UAEMPBUplane@primitives@@PBUgeom_world_data@@AAU?$Vec3_tpl@M@@@Z 35139f80 f   capsulegeom.obj
 0001:00138f90       ?CreateCapsule@CCapsuleGeom@@QAEPAV1@PAUcapsule@primitives@@@Z 35139f90 f   capsulegeom.obj
 0001:001391b0       ?GetUnprojectionCandidates@CCapsuleGeom@@UAEHHPBUcontact@@AAPAUprimitive@primitives@@AAPAHPAUgeometry_under_test@@@Z 3513a1b0 f   capsulegeom.obj
 0001:00139430       ?FindClosestPoint@CCapsuleGeom@@UAEHPAUgeom_world_data@@AAH1ABU?$Vec3_tpl@M@@2PAU3@H@Z 3513a430 f   capsulegeom.obj
 0001:00139f80       ?UnprojectSphere@CCapsuleGeom@@UAEHU?$Vec3_tpl@M@@MMPAUcontact@@@Z 3513af80 f   capsulegeom.obj
 0001:0013a3e0       ?CalculateMediumResistance@CCapsuleGeom@@UAEXPBUplane@primitives@@PBUgeom_world_data@@AAU?$Vec3_tpl@M@@2@Z 3513b3e0 f   capsulegeom.obj
 0001:0013af30       ?DrawToOcclusionCubemap@CCapsuleGeom@@UAEHPBUgeom_world_data@@HHHPAUSOcclusionCubeMap@@@Z 3513bf30 f   capsulegeom.obj
 0001:0013b0e0       ?CalcPhysicalProperties@CCapsuleGeom@@UAEHPAUphys_geometry@@@Z 3513c0e0 f   capsulegeom.obj
 0001:0013b3c0       ?PrepareForIntersectionTest@CCylinderGeom@@UAEHPAUgeometry_under_test@@PAVCGeometry@@0_N@Z 3513c3c0 f   cylindergeom.obj
 0001:0013b480       ?ComputeExtent@CCylinderGeom@@UAEMAAUGeomQuery@@W4EGeomForm@@@Z 3513c480 f   cylindergeom.obj
 0001:0013b500       ?GetMemoryStatistics@CCylinderGeom@@UAEXPAVICrySizer@@@Z 3513c500 f   cylindergeom.obj
 0001:0013b520       ?PointInsideStatus@CCylinderGeom@@UAEHABU?$Vec3_tpl@M@@@Z 3513c520 f   cylindergeom.obj
 0001:0013b600       ?PrepareCylinder@CCylinderGeom@@QAEXPAUcylinder@primitives@@PAUgeometry_under_test@@@Z 3513c600 f   cylindergeom.obj
 0001:0013b780       ?PreparePrimitive@CCylinderGeom@@UAEHPAUgeom_world_data@@AAPAUprimitive@primitives@@H@Z 3513c780 f   cylindergeom.obj
 0001:0013b930       ?GetPrimitiveList@CCylinderGeom@@UAEHHHHPAUprimitive@primitives@@HPAUgeometry_under_test@@10PAD@Z 3513c930 f   cylindergeom.obj
 0001:0013b960       ?PreparePolyline@CCylinderGeom@@UAEHPAUcoord_plane@primitives@@HHPAUgeometry_under_test@@AAPAU?$Vec2_tpl@M@@AAPAH3@Z 3513c960 f   cylindergeom.obj
 0001:0013bd00       ?DrawWireframe@CCylinderGeom@@UAEXPAUIPhysRenderer@@PAUgeom_world_data@@HH@Z 3513cd00 f   cylindergeom.obj
 0001:0013bdd0       ?CreateCylinder@CCylinderGeom@@QAEPAV1@PAUcylinder@primitives@@@Z 3513cdd0 f   cylindergeom.obj
 0001:0013bff0       ?GetRandomPos@CCylinderGeom@@UAEXAAURandomPos@@AAUGeomQuery@@W4EGeomForm@@@Z 3513cff0 f   cylindergeom.obj
 0001:0013c670       ?GetUnprojectionCandidates@CCylinderGeom@@UAEHHPBUcontact@@AAPAUprimitive@primitives@@AAPAHPAUgeometry_under_test@@@Z 3513d670 f   cylindergeom.obj
 0001:0013c9b0       ?PreparePolygon@CCylinderGeom@@UAEHPAUcoord_plane@primitives@@HHPAUgeometry_under_test@@AAPAU?$Vec2_tpl@M@@AAPAH3@Z 3513d9b0 f   cylindergeom.obj
 0001:0013d010       ?UnprojectSphere@CCylinderGeom@@UAEHU?$Vec3_tpl@M@@MMPAUcontact@@@Z 3513e010 f   cylindergeom.obj
 0001:0013d210       ?CalcVolumetricPressure@CCylinderGeom@@UAEXPAUgeom_world_data@@ABU?$Vec3_tpl@M@@MM1AAU3@2@Z 3513e210 f   cylindergeom.obj
 0001:0013d520       ?CalculateBuoyancy@CCylinderGeom@@UAEMPBUplane@primitives@@PBUgeom_world_data@@AAU?$Vec3_tpl@M@@@Z 3513e520 f   cylindergeom.obj
 0001:0013e520       ?crop_polyarc2d_with_line@@YAHPBU?$Vec2_tpl@M@@PBHHMPAU1@PAHABU1@4@Z 3513f520 f   cylindergeom.obj
 0001:0013ee10       ?CalculateMediumResistance@CCylinderGeom@@UAEXPBUplane@primitives@@PBUgeom_world_data@@AAU?$Vec3_tpl@M@@2@Z 3513fe10 f   cylindergeom.obj
 0001:00141010       ?DrawToOcclusionCubemap@CCylinderGeom@@UAEHPBUgeom_world_data@@HHHPAUSOcclusionCubeMap@@@Z 35142010 f   cylindergeom.obj
 0001:001411a0       ?Save@CCylinderGeom@@UAEXAAVCMemStream@@@Z 351421a0 f   cylindergeom.obj
 0001:00141220       ?Load@CCylinderGeom@@UAEXAAVCMemStream@@@Z 35142220 f   cylindergeom.obj
 0001:00141280       ?findroots@?$polynomial_tpl@N$03@@QBEHNNPANHH_N@Z 35142280 f i cylindergeom.obj
 0001:00141eb0       ?CalcPhysicalProperties@CCylinderGeom@@UAEHPAUphys_geometry@@@Z 35142eb0 f   cylindergeom.obj
 0001:00142130       ?FindClosestPoint@CCylinderGeom@@UAEHPAUgeom_world_data@@AAH1ABU?$Vec3_tpl@M@@2PAU3@H@Z 35143130 f   cylindergeom.obj
 0001:00143dc0       ?InitGeoman@CGeomManager@@UAEXXZ 35144dc0 f   geoman.obj
 0001:00143e00       ?ShutDownGeoman@CGeomManager@@UAEXXZ 35144e00 f   geoman.obj
 0001:00143ed0       ?DestroyGeometry@CGeomManager@@UAEXPAUIGeometry@@@Z 35144ed0 f   geoman.obj
 0001:00143ef0       ?AddRefGeometry@CGeomManager@@UAEHPAUphys_geometry@@@Z 35144ef0 f   geoman.obj
 0001:00143f10       ?UnregisterGeometry@CGeomManager@@UAEHPAUphys_geometry@@@Z 35144f10 f   geoman.obj
 0001:00143ff0       ?Release@CGeometry@@UAEXXZ 35144ff0 f   geoman.obj
 0001:00144030       ?FlushOldGeoms@CGeomManager@@QAEXXZ 35145030 f   geoman.obj
 0001:00144090       ?SetGeomMatMapping@CGeomManager@@UAEXPAUphys_geometry@@PAHH@Z 35145090 f   geoman.obj
 0001:00144100       ?CreateTetrLattice@CGeomManager@@UAEPAUITetrLattice@@PBU?$Vec3_tpl@M@@HPBHH@Z 35145100 f   geoman.obj
 0001:00144150       ?MaxPrimsInNode@CVoxelBV@@UAEHXZ 35145150 f i geoman.obj
 0001:00144160       ?GetNodeBV@CVoxelBV@@UAEXAAPAUBV@@ABU?$Vec3_tpl@M@@MHH@Z 35145160 f i geoman.obj
 0001:00144180       ?GetNodeBV@CVoxelBV@@UAEXABU?$Matrix33_tpl@M@@ABU?$Vec3_tpl@M@@MAAPAUBV@@1MHH@Z 35145180 f i geoman.obj
 0001:001441b0       ?ResetCollisionArea@CVoxelBV@@UAEXXZ 351451b0 f i geoman.obj
 0001:001441e0       ?GetGridData@CBreakableGrid2d@@UAEPAUgrid@primitives@@XZ 351451e0 f i geoman.obj
 0001:001441f0       ?IsEmpty@CBreakableGrid2d@@UAE_NXZ 351451f0 f i geoman.obj
 0001:00144200       ?GetFracture@CBreakableGrid2d@@UAEMXZ 35145200 f i geoman.obj
 0001:00144220       ?GetMemoryStatistics@CBreakableGrid2d@@UBEXPAVICrySizer@@@Z 35145220 f i geoman.obj
 0001:00144290       ??_ECBreakableGrid2d@@UAEPAXI@Z 35145290 f i geoman.obj
 0001:00144290       ??_GCBreakableGrid2d@@UAEPAXI@Z 35145290 f i geoman.obj
 0001:00144300       ?GenerateBreakableGrid@CGeomManager@@UAEPAUIBreakableGrid2d@@PAU?$Vec2_tpl@M@@HABU?$Vec2_tpl@H@@HH@Z 35145300 f   geoman.obj
 0001:00144380       ??0CRayGeom@@QAE@PBUray@primitives@@@Z 35145380 f i geoman.obj
 0001:001444b0       ?GetFreeGeomSlot@CGeomManager@@QAEPAUphys_geometry@@XZ 351454b0 f   geoman.obj
 0001:00144590       ?RegisterGeometry@CGeomManager@@UAEPAUphys_geometry@@PAUIGeometry@@HPAHH@Z 35145590 f   geoman.obj
 0001:00144700       ?SaveGeometry@CGeomManager@@UAEXAAVCMemStream@@PAUIGeometry@@@Z 35145700 f   geoman.obj
 0001:00144750       ?LoadGeometry@CGeomManager@@UAEPAUIGeometry@@AAVCMemStream@@V?$strided_pointer@$$CBU?$Vec3_tpl@M@@@@V?$strided_pointer@G@@PAD@Z 35145750 f   geoman.obj
 0001:001448d0       ?SavePhysGeometry@CGeomManager@@UAEXAAVCMemStream@@PAUphys_geometry@@@Z 351458d0 f   geoman.obj
 0001:00144a00       ?LoadPhysGeometry@CGeomManager@@UAEPAUphys_geometry@@AAVCMemStream@@V?$strided_pointer@$$CBU?$Vec3_tpl@M@@@@V?$strided_pointer@G@@PAD@Z 35145a00 f   geoman.obj
 0001:00144bc0       ??$ComputeMeshEigenBasis@G@@YAXV?$strided_pointer@$$CBU?$Vec3_tpl@M@@@@V?$strided_pointer@G@@HPAU?$Vec3_tpl@N@@AAU2@@Z 35145bc0 f i geoman.obj
 0001:00145360       ?Prealloc@CMemStream@@UAEXXZ 35146360 f i geoman.obj
 0001:001453c0       ?GrowBuf@CMemStream@@UAEXH@Z 351463c0 f i geoman.obj
 0001:00145480       ??_ECMemStream@@UAEPAXI@Z  35146480 f i geoman.obj
 0001:00145480       ??_GCMemStream@@UAEPAXI@Z  35146480 f i geoman.obj
 0001:001454f0       ?GetData@CTriMesh@@UAEPBUprimitive@primitives@@XZ 351464f0 f i geoman.obj
 0001:00145500       ?GetBVTree@CVoxelGeom@@UAEPAVCBVTree@@XZ 35146500 f i geoman.obj
 0001:00145510       ??_ECVoxelGeom@@UAEPAXI@Z  35146510 f i geoman.obj
 0001:00145510       ??_GCVoxelGeom@@UAEPAXI@Z  35146510 f i geoman.obj
 0001:00145570       ?GetPrimitive@CTriMesh@@UAEHHPAUprimitive@primitives@@@Z 35146570 f i geoman.obj
 0001:00145610       ?CreateMesh@CGeomManager@@UAEPAUIGeometry@@V?$strided_pointer@$$CBU?$Vec3_tpl@M@@@@V?$strided_pointer@G@@PADPAHHHMPAUSMeshBVParams@@@Z 35146610 f   geoman.obj
 0001:001458a0       ?CreatePrimitive@CGeomManager@@UAEPAUIGeometry@@HPBUprimitive@primitives@@@Z 351468a0 f   geoman.obj
 0001:00145aa0       ?RegisterCrack@CGeomManager@@UAEHPAUIGeometry@@PAU?$Vec3_tpl@M@@H@Z 35146aa0 f   geoman.obj
 0001:00146530       ?UnregisterCrack@CGeomManager@@UAEXH@Z 35147530 f   geoman.obj
 0001:001465f0       ?GetCrackGeom@CGeomManager@@UAEPAUIGeometry@@PBU?$Vec3_tpl@M@@HPAUgeom_world_data@@@Z 351475f0 f   geoman.obj
 0001:00147a90       ?CloneGeometry@CGeomManager@@UAEPAUIGeometry@@PAU2@@Z 35148a90 f   geoman.obj
 0001:00147be0       ??0InitGeometryGlobals@@QAE@XZ 35148be0 f   geometry.obj
 0001:00147c60       ?RadiusCheckBVs@@YAHPAUradius_check_data@@PAUBV@@@Z 35148c60 f   geometry.obj
 0001:00147d30       ?SphereCheckBVs@@YAHPAVCBVTree@@PAUsphere@primitives@@PAUBV@@H@Z 35148d30 f   geometry.obj
 0001:00147e00       ?IntersectLocked@CGeometry@@UAEHPAUIGeometry@@PAUgeom_world_data@@1PAUintersection_params@@AAPAUgeom_contact@@AAUWriteLockCond@@H@Z 35148e00 f   geometry.obj
 0001:00147ea0       ?TestBV@@YAXPAVCBVTree@@PAUBV@@HHAA_NH@Z 35148ea0 f   geometry.obj
 0001:00147f40       ??0cylinder@primitives@@QAE@XZ 35148f40 f i livingentity.obj
 0001:00147f40       ??0ray@primitives@@QAE@XZ  35148f40 f i livingentity.obj
 0001:00147f40       ??0?$Vec3_tpl@M@@QAE@XZ    35148f40 f i articulatedentity.obj
 0001:00147f40       ??0?$Vec2_tpl@M@@QAE@XZ    35148f40 f i livingentity.obj
 0001:00147f40       ?GetEntity@CPhysicalEntity@@UAEPAV1@XZ 35148f40 f i rwi.obj
 0001:00147f40       ??0surface_desc@@QAE@XZ    35148f40 f i geometry.obj
 0001:00147f40       ??0BBoxExt@@QAE@XZ         35148f40 f i geometry.obj
 0001:00147f40       ??0BBox@@QAE@XZ            35148f40 f i geometry.obj
 0001:00147f40       ??0edge_desc@@QAE@XZ       35148f40 f i geometry.obj
 0001:00147f40       ??0sphere@primitives@@QAE@XZ 35148f40 f i livingentity.obj
 0001:00147f40       ?GetEntityFast@CPhysicalEntity@@UAEPAV1@XZ 35148f40 f i articulatedentity.obj
 0001:00147f40       ??0geom_contact_area@@QAE@XZ 35148f40 f i geometry.obj
 0001:00147f40       ??0box@primitives@@QAE@XZ  35148f40 f i articulatedentity.obj
 0001:00147f40       ??0geom_contact@@QAE@XZ    35148f40 f i particleentity.obj
 0001:00147f40       ??0indexed_triangle@primitives@@QAE@XZ 35148f40 f i physarea.obj
 0001:00147f50       ?ComputeExtent@CGeometry@@UAEMAAUGeomQuery@@W4EGeomForm@@@Z 35148f50 f   geometry.obj
 0001:00148010       ?SanityCheckTree@@YAHPAVCBVTree@@H@Z 35149010 f   geometry.obj
 0001:001480a0       ?BoxRandomPos@@YAXAAURandomPos@@W4EGeomForm@@ABU?$Vec3_tpl@M@@@Z 351490a0 f i geometry.obj
 0001:00148330       ?IntersectBVs@@YAHPAUgeometry_under_test@@PAUBV@@1@Z 35149330 f   geometry.obj
 0001:00148790       ?SweepTestBVs@@YAHPAUgeometry_under_test@@PAUBV@@1@Z 35149790 f   geometry.obj
 0001:00148d20       ?BuildOcclusionCubemap@CGeometry@@UAEMPAUgeom_world_data@@HPAUSOcclusionCubeMap@@1H@Z 35149d20 f   geometry.obj
 0001:00148fd0       ?RegisterIntersection@CGeometry@@UAEHPAUprimitive@primitives@@0PAUgeometry_under_test@@1PAUprim_inters@@@Z 35149fd0 f   geometry.obj
 0001:001496b0       ?GetRandomPos@CGeometry@@UAEXAAURandomPos@@AAUGeomQuery@@W4EGeomForm@@@Z 3514a6b0 f   geometry.obj
 0001:00149830       ?SphereCheck@CGeometry@@QAEHABU?$Vec3_tpl@M@@MH@Z 3514a830 f   geometry.obj
 0001:00149990       ?GTestPrepPartDeux@@YAXPAUgeometry_under_test@@AAU?$Vec3_tpl@N@@@Z 3514a990 f   geometry.obj
 0001:00149d30       ?Intersect@CGeometry@@UAEHPAUIGeometry@@PAUgeom_world_data@@1PAUintersection_params@@AAPAUgeom_contact@@@Z 3514ad30 f   geometry.obj
 0001:0014bb60       ?DrawBBox@@YAXPAUIPhysRenderer@@HPAUgeom_world_data@@PAVCBVTree@@PAUBBox@@HHH@Z 3514cb60 f   geometry.obj
 0001:0014bde0       ?Intersect@CPrimitive@@UAEHPAUIGeometry@@PAUgeom_world_data@@1PAUintersection_params@@AAPAUgeom_contact@@@Z 3514cde0 f   geometry.obj
 0001:0014dad0       ?Build@CHeightfieldBV@@UAEMPAVCGeometry@@@Z 3514ead0 f   heightfieldbv.obj
 0001:0014db00       ?MarkUsedTriangle@CHeightfieldBV@@UAEXHPAUgeometry_under_test@@@Z 3514eb00 f   heightfieldbv.obj
 0001:0014db30       ?GetBBox@CHeightfieldBV@@UAEXPAUbox@primitives@@@Z 3514eb30 f   heightfieldbv.obj
 0001:0014dc10       ?GetNodeBV@CHeightfieldBV@@UAEXAAPAUBV@@HH@Z 3514ec10 f   heightfieldbv.obj
 0001:0014dce0       ?project_box_on_grid@@YAXPAUbox@primitives@@PAUgrid@2@PAUgeometry_under_test@@AAH333AAM@Z 3514ece0 f   heightfieldbv.obj
 0001:0014e340       ?GetNodeContents@CHeightfieldBV@@UAEHHPAUBV@@HHPAUgeometry_under_test@@1@Z 3514f340 f   heightfieldbv.obj
 0001:0014e510       ?GetNodeBV@CHeightfieldBV@@UAEXABU?$Matrix33_tpl@M@@ABU?$Vec3_tpl@M@@MAAPAUBV@@HH@Z 3514f510 f   heightfieldbv.obj
 0001:0014e740       ?GetMemoryStatistics@CHeightfield@@UAEXPAVICrySizer@@@Z 3514f740 f   heightfieldgeom.obj
 0001:0014e770       ?PointInsideStatus@CHeightfield@@UAEHABU?$Vec3_tpl@M@@@Z 3514f770 f   heightfieldgeom.obj
 0001:0014e960       ?CreateHeightfield@CHeightfield@@QAEPAV1@PAUheightfield@primitives@@@Z 3514f960 f   heightfieldgeom.obj
 0001:0014eb40       ?check_cell@hf_cell_checker@@QAEHABU?$Vec2_tpl@H@@AAH@Z 3514fb40 f i heightfieldgeom.obj
 0001:0014ef70       ?PrepareForIntersectionTest@CHeightfield@@UAEHPAUgeometry_under_test@@PAVCGeometry@@0_N@Z 3514ff70 f   heightfieldgeom.obj
 0001:0014fa70       ?CheckPtEdgeDist@@YAXPBU?$Vec3_tpl@M@@ABU1@AAU1@AAH@Z 35150a70 f i heightfieldgeom.obj
 0001:0014fc70       ?CheckPtTriDist@@YAXABUtriangle@primitives@@ABU?$Vec3_tpl@M@@AAU3@AAH@Z 35150c70 f i heightfieldgeom.obj
 0001:00150070       ?FindClosestPoint@CHeightfield@@UAEHPAUgeom_world_data@@AAH1ABU?$Vec3_tpl@M@@2PAU3@H@Z 35151070 f   heightfieldgeom.obj
 0001:00150700       ?DrawToOcclusionCubemap@CHeightfield@@UAEHPBUgeom_world_data@@HHHPAUSOcclusionCubeMap@@@Z 35151700 f   heightfieldgeom.obj
 0001:00151000       ??$DrawRayOnGrid@Uhf_cell_checker@@@@YAHPAUgrid@primitives@@AAU?$Vec3_tpl@M@@1AAUhf_cell_checker@@@Z 35152000 f i heightfieldgeom.obj
 0001:00151660       ?Intersect@CHeightfield@@UAEHPAUIGeometry@@PAUgeom_world_data@@1PAUintersection_params@@AAPAUgeom_contact@@@Z 35152660 f   heightfieldgeom.obj
 0001:001529b0       ?GetErrorCount@CGeometry@@UAEHXZ 351539b0 f   livingentity.obj
 0001:001529b0       ?GetiForeignData@CPhysicalStub@@UBEHXZ 351539b0 f   physarea.obj
 0001:001529b0       ?AddRef@CPhysicalPlaceholder@@UAEHXZ 351539b0 f   physarea.obj
 0001:001529b0       ?GetStateChecksum@CPhysicalEntity@@UAEIXZ 351539b0 f   livingentity.obj
 0001:001529b0       ?GetType@CBoxGeom@@UAEHXZ  351539b0 f   physicalentity.obj
 0001:001529b0       ?GetIWorld@CGeomManager@@UAEPAUIPhysicalWorld@@XZ 351539b0 f   physicalworld.obj
 0001:001529b0       ?IsAPrimitive@CGeometry@@UAEHXZ 351539b0 f   livingentity.obj
 0001:001529b0       ?Release@CPhysicalStub@@UAEHXZ 351539b0 f   physarea.obj
 0001:001529b0       ?GetWorld@CPhysicalStub@@UBEPAUIPhysicalWorld@@XZ 351539b0 f   physarea.obj
 0001:001529b0       ?GetSubtractionsCount@CGeometry@@UAEHXZ 351539b0 f   livingentity.obj
 0001:001529b0       ?default_intersection@@YAHPBUprimitive@primitives@@0PAUprim_inters@@@Z 351539b0 f   intersectionchecks.obj
 0001:001529b0       ?GetStateChecksum@CPhysicalStub@@UAEIXZ 351539b0 f   physarea.obj
 0001:001529b0       ?GetSizeFast@CGeometry@@UAEHXZ 351539b0 f   livingentity.obj
 0001:001529b0       ?PostSetStateFromSnapshot@CPhysicalStub@@UAEHXZ 351539b0 f   physarea.obj
 0001:001529b0       ?GetBVTree@CGeometry@@UAEPAVCBVTree@@XZ 351539b0 f   livingentity.obj
 0001:001529b0       ?Release@CPhysicalPlaceholder@@UAEHXZ 351539b0 f   physarea.obj
 0001:001529b0       ?default_unprojection@@YAHPAUunprojection_mode@@PBUprimitive@primitives@@H1HPAUcontact@@PAUgeom_contact_area@@@Z 351539b0 f   linunprojectionchecks.obj
 0001:001529b0       ?AddRef@CPhysicalStub@@UAEHXZ 351539b0 f   physarea.obj
 0001:001529b0       ?GetType@COBBTree@@UAEHXZ  351539b0 f   trimesh.obj
 0001:001529c0       ?box_sphere_intersection@@YAHPBUbox@primitives@@PBUsphere@2@PAUprim_inters@@@Z 351539c0 f   intersectionchecks.obj
 0001:00152ca0       ?sphere_box_intersection@@YAHPBUsphere@primitives@@PBUbox@2@PAUprim_inters@@@Z 35153ca0 f   intersectionchecks.obj
 0001:00152d10       ?sphere_sphere_intersection@@YAHPBUsphere@primitives@@0PAUprim_inters@@@Z 35153d10 f   intersectionchecks.obj
 0001:00152eb0       ?tri_tri_intersection@@YAHPBUtriangle@primitives@@0PAUprim_inters@@@Z 35153eb0 f   intersectionchecks.obj
 0001:00153650       ?tri_sphere_intersection@@YAHPBUtriangle@primitives@@PBUsphere@2@PAUprim_inters@@@Z 35154650 f   intersectionchecks.obj
 0001:00153f60       ?sphere_tri_intersection@@YAHPBUsphere@primitives@@PBUtriangle@2@PAUprim_inters@@@Z 35154f60 f   intersectionchecks.obj
 0001:00153fc0       ?ray_tri_intersection@@YAHPBUray@primitives@@PBUtriangle@2@PAUprim_inters@@@Z 35154fc0 f   intersectionchecks.obj
 0001:00154530       ?tri_ray_intersection@@YAHPBUtriangle@primitives@@PBUray@2@PAUprim_inters@@@Z 35155530 f   intersectionchecks.obj
 0001:001545a0       ?box_cylinder_intersection@@YAHPBUbox@primitives@@PBUcylinder@2@PAUprim_inters@@@Z 351555a0 f   intersectionchecks.obj
 0001:00155980       ?cylinder_box_intersection@@YAHPBUcylinder@primitives@@PBUbox@2@PAUprim_inters@@@Z 35156980 f   intersectionchecks.obj
 0001:001559f0       ?box_capsule_intersection@@YAHPBUbox@primitives@@PBUcapsule@2@PAUprim_inters@@@Z 351569f0 f   intersectionchecks.obj
 0001:00156b50       ?capsule_box_intersection@@YAHPBUcapsule@primitives@@PBUbox@2@PAUprim_inters@@@Z 35157b50 f   intersectionchecks.obj
 0001:00156bc0       ?box_ray_intersection@@YAHPBUbox@primitives@@PBUray@2@PAUprim_inters@@@Z 35157bc0 f   intersectionchecks.obj
 0001:00157000       ?ray_box_intersection@@YAHPBUray@primitives@@PBUbox@2@PAUprim_inters@@@Z 35158000 f   intersectionchecks.obj
 0001:00157040       ?cylinder_cylinder_intersection@@YAHPBUcylinder@primitives@@0PAUprim_inters@@@Z 35158040 f   intersectionchecks.obj
 0001:00158c00       ?cylinder_sphere_intersection@@YAHPBUcylinder@primitives@@PBUsphere@2@PAUprim_inters@@@Z 35159c00 f   intersectionchecks.obj
 0001:00158f90       ?sphere_cylinder_intersection@@YAHPBUsphere@primitives@@PBUcylinder@2@PAUprim_inters@@@Z 35159f90 f   intersectionchecks.obj
 0001:00158fd0       ?cylinder_capsule_intersection@@YAHPBUcylinder@primitives@@PBUcapsule@2@PAUprim_inters@@@Z 35159fd0 f   intersectionchecks.obj
 0001:0015a070       ?capsule_cylinder_intersection@@YAHPBUcapsule@primitives@@PBUcylinder@2@PAUprim_inters@@@Z 3515b070 f   intersectionchecks.obj
 0001:0015a0b0       ?cylinder_ray_intersection@@YAHPBUcylinder@primitives@@PBUray@2@PAUprim_inters@@@Z 3515b0b0 f   intersectionchecks.obj
 0001:0015aaf0       ?ray_cylinder_intersection@@YAHPBUray@primitives@@PBUcylinder@2@PAUprim_inters@@@Z 3515baf0 f   intersectionchecks.obj
 0001:0015ab30       ?sphere_ray_intersection@@YAHPBUsphere@primitives@@PBUray@2@PAUprim_inters@@@Z 3515bb30 f   intersectionchecks.obj
 0001:0015ada0       ?ray_sphere_intersection@@YAHPBUray@primitives@@PBUsphere@2@PAUprim_inters@@@Z 3515bda0 f   intersectionchecks.obj
 0001:0015ade0       ?capsule_capsule_intersection@@YAHPBUcapsule@primitives@@0PAUprim_inters@@@Z 3515bde0 f   intersectionchecks.obj
 0001:0015b460       ?capsule_sphere_intersection@@YAHPBUcylinder@primitives@@PBUsphere@2@PAUprim_inters@@@Z 3515c460 f   intersectionchecks.obj
 0001:0015b6b0       ?sphere_capsule_intersection@@YAHPBUsphere@primitives@@PBUcapsule@2@PAUprim_inters@@@Z 3515c6b0 f   intersectionchecks.obj
 0001:0015b6f0       ?capsule_ray_intersection@@YAHPBUcapsule@primitives@@PBUray@2@PAUprim_inters@@@Z 3515c6f0 f   intersectionchecks.obj
 0001:0015c010       ?ray_capsule_intersection@@YAHPBUray@primitives@@PBUcapsule@2@PAUprim_inters@@@Z 3515d010 f   intersectionchecks.obj
 0001:0015c050       ?tri_box_intersection@@YAHPBUtriangle@primitives@@PBUbox@2@PAUprim_inters@@@Z 3515d050 f   intersectionchecks.obj
 0001:0015d920       ?box_tri_intersection@@YAHPBUbox@primitives@@PBUtriangle@2@PAUprim_inters@@@Z 3515e920 f   intersectionchecks.obj
 0001:0015d9b0       ?tri_cylinder_intersection@@YAHPBUtriangle@primitives@@PBUcylinder@2@PAUprim_inters@@@Z 3515e9b0 f   intersectionchecks.obj
 0001:00160e40       ?cylinder_tri_intersection@@YAHPBUcylinder@primitives@@PBUtriangle@2@PAUprim_inters@@@Z 35161e40 f   intersectionchecks.obj
 0001:00160ea0       ?tri_capsule_intersection@@YAHPBUtriangle@primitives@@PBUcapsule@2@PAUprim_inters@@@Z 35161ea0 f   intersectionchecks.obj
 0001:00163150       ?capsule_tri_intersection@@YAHPBUcapsule@primitives@@PBUtriangle@2@PAUprim_inters@@@Z 35164150 f   intersectionchecks.obj
 0001:001631b0       ?box_box_intersection@@YAHPBUbox@primitives@@0PAUprim_inters@@@Z 351641b0 f   intersectionchecks.obj
 0001:00163b70       ?WaitForJobFinish@@YAHAAHH@Z 35164b70 f   jobq.obj
 0001:00163b80       ?crop_polygon_with_bound@@YAHPBU?$Vec2_tpl@M@@PBHHABU1@HHPAU1@PAH@Z 35164b80 f   linunprojectionchecks.obj
 0001:001641f0       ?crop_segment_with_bound@@YAXPAU?$Vec2_tpl@M@@MHPAH1HH@Z 351651f0 f   linunprojectionchecks.obj
 0001:00164350       ?flip_contact@@YAXPBUunprojection_mode@@PAUcontact@@PAUgeom_contact_area@@@Z 35165350 f   linunprojectionchecks.obj
 0001:001645e0       ?tri_tri_lin_unprojection@@YAHPAUunprojection_mode@@PBUtriangle@primitives@@H1HPAUcontact@@PAUgeom_contact_area@@@Z 351655e0 f   linunprojectionchecks.obj
 0001:00165690       ?tri_box_lin_unprojection@@YAHPAUunprojection_mode@@PBUtriangle@primitives@@HPBUbox@3@HPAUcontact@@PAUgeom_contact_area@@@Z 35166690 f   linunprojectionchecks.obj
 0001:00166a80       ?box_tri_lin_unprojection@@YAHPAUunprojection_mode@@PBUbox@primitives@@HPBUtriangle@3@HPAUcontact@@PAUgeom_contact_area@@@Z 35167a80 f   linunprojectionchecks.obj
 0001:00166bd0       ?tri_cylinder_lin_unprojection@@YAHPAUunprojection_mode@@PBUtriangle@primitives@@HPBUcylinder@3@HPAUcontact@@PAUgeom_contact_area@@@Z 35167bd0 f   linunprojectionchecks.obj
 0001:0016a160       ?cylinder_tri_lin_unprojection@@YAHPAUunprojection_mode@@PBUcylinder@primitives@@HPBUtriangle@3@HPAUcontact@@PAUgeom_contact_area@@@Z 3516b160 f   linunprojectionchecks.obj
 0001:0016a2b0       ?tri_sphere_lin_unprojection@@YAHPAUunprojection_mode@@PBUtriangle@primitives@@HPBUsphere@3@HPAUcontact@@PAUgeom_contact_area@@@Z 3516b2b0 f   linunprojectionchecks.obj
 0001:0016b0a0       ?sphere_tri_lin_unprojection@@YAHPAUunprojection_mode@@PBUsphere@primitives@@HPBUtriangle@3@HPAUcontact@@PAUgeom_contact_area@@@Z 3516c0a0 f   linunprojectionchecks.obj
 0001:0016b1f0       ?tri_capsule_lin_unprojection@@YAHPAUunprojection_mode@@PBUtriangle@primitives@@HPBUcapsule@3@HPAUcontact@@PAUgeom_contact_area@@@Z 3516c1f0 f   linunprojectionchecks.obj
 0001:0016b380       ?capsule_tri_lin_unprojection@@YAHPAUunprojection_mode@@PBUcapsule@primitives@@HPBUtriangle@3@HPAUcontact@@PAUgeom_contact_area@@@Z 3516c380 f   linunprojectionchecks.obj
 0001:0016b4d0       ?tri_ray_lin_unprojection@@YAHPAUunprojection_mode@@PBUtriangle@primitives@@HPBUray@3@HPAUcontact@@PAUgeom_contact_area@@@Z 3516c4d0 f   linunprojectionchecks.obj
 0001:0016c2b0       ?ray_tri_lin_unprojection@@YAHPAUunprojection_mode@@PBUray@primitives@@HPBUtriangle@3@HPAUcontact@@PAUgeom_contact_area@@@Z 3516d2b0 f   linunprojectionchecks.obj
 0001:0016c400       ?box_cylinder_lin_unprojection@@YAHPAUunprojection_mode@@PBUbox@primitives@@HPBUcylinder@3@HPAUcontact@@PAUgeom_contact_area@@@Z 3516d400 f   linunprojectionchecks.obj
 0001:00171430       ?cylinder_box_lin_unprojection@@YAHPAUunprojection_mode@@PBUcylinder@primitives@@HPBUbox@3@HPAUcontact@@PAUgeom_contact_area@@@Z 35172430 f   linunprojectionchecks.obj
 0001:001714e0       ?box_sphere_lin_unprojection@@YAHPAUunprojection_mode@@PBUbox@primitives@@HPBUsphere@3@HPAUcontact@@PAUgeom_contact_area@@@Z 351724e0 f   linunprojectionchecks.obj
 0001:00172530       ?sphere_box_lin_unprojection@@YAHPAUunprojection_mode@@PBUsphere@primitives@@HPBUbox@3@HPAUcontact@@PAUgeom_contact_area@@@Z 35173530 f   linunprojectionchecks.obj
 0001:00172670       ?box_capsule_lin_unprojection@@YAHPAUunprojection_mode@@PBUbox@primitives@@HPBUcapsule@3@HPAUcontact@@PAUgeom_contact_area@@@Z 35173670 f   linunprojectionchecks.obj
 0001:00172b00       ?capsule_box_lin_unprojection@@YAHPAUunprojection_mode@@PBUcapsule@primitives@@HPBUbox@3@HPAUcontact@@PAUgeom_contact_area@@@Z 35173b00 f   linunprojectionchecks.obj
 0001:00172bb0       ?sphere_sphere_lin_unprojection@@YAHPAUunprojection_mode@@PBUsphere@primitives@@H1HPAUcontact@@PAUgeom_contact_area@@@Z 35173bb0 f   linunprojectionchecks.obj
 0001:00172f20       ?ray_box_lin_unprojection@@YAHPAUunprojection_mode@@PBUray@primitives@@HPBUbox@3@HPAUcontact@@PAUgeom_contact_area@@@Z 35173f20 f   linunprojectionchecks.obj
 0001:00173c20       ?box_ray_lin_unprojection@@YAHPAUunprojection_mode@@PBUbox@primitives@@HPBUray@3@HPAUcontact@@PAUgeom_contact_area@@@Z 35174c20 f   linunprojectionchecks.obj
 0001:00173d70       ?ray_cylinder_lin_unprojection@@YAHPAUunprojection_mode@@PBUray@primitives@@HPBUcylinder@3@HPAUcontact@@PAUgeom_contact_area@@@Z 35174d70 f   linunprojectionchecks.obj
 0001:00175e60       ?cylinder_ray_lin_unprojection@@YAHPAUunprojection_mode@@PBUcylinder@primitives@@HPBUray@3@HPAUcontact@@PAUgeom_contact_area@@@Z 35176e60 f   linunprojectionchecks.obj
 0001:00175fb0       ?ray_sphere_lin_unprojection@@YAHPAUunprojection_mode@@PBUray@primitives@@HPBUsphere@3@HPAUcontact@@PAUgeom_contact_area@@@Z 35176fb0 f   linunprojectionchecks.obj
 0001:00176850       ?sphere_ray_lin_unprojection@@YAHPAUunprojection_mode@@PBUsphere@primitives@@HPBUray@3@HPAUcontact@@PAUgeom_contact_area@@@Z 35177850 f   linunprojectionchecks.obj
 0001:001769a0       ?ray_capsule_lin_unprojection@@YAHPAUunprojection_mode@@PBUray@primitives@@HPBUcapsule@3@HPAUcontact@@PAUgeom_contact_area@@@Z 351779a0 f   linunprojectionchecks.obj
 0001:00176b30       ?capsule_ray_lin_unprojection@@YAHPAUunprojection_mode@@PBUcapsule@primitives@@HPBUray@3@HPAUcontact@@PAUgeom_contact_area@@@Z 35177b30 f   linunprojectionchecks.obj
 0001:00176c80       ?box_box_lin_unprojection@@YAHPAUunprojection_mode@@PBUbox@primitives@@H1HPAUcontact@@PAUgeom_contact_area@@@Z 35177c80 f   linunprojectionchecks.obj
 0001:00179d30       ?cylinder_sphere_lin_unprojection@@YAHPAUunprojection_mode@@PBUcylinder@primitives@@HPBUsphere@3@HPAUcontact@@PAUgeom_contact_area@@@Z 3517ad30 f   linunprojectionchecks.obj
 0001:0017b470       ?sphere_cylinder_lin_unprojection@@YAHPAUunprojection_mode@@PBUsphere@primitives@@HPBUcylinder@3@HPAUcontact@@PAUgeom_contact_area@@@Z 3517c470 f   linunprojectionchecks.obj
 0001:0017b5c0       ?cyl_cyl_lin_unprojection@@YAHPAUunprojection_mode@@PBUcylinder@primitives@@H1HPAUcontact@@PAUgeom_contact_area@@@Z 3517c5c0 f   linunprojectionchecks.obj
 0001:00182be0       ?cylinder_capsule_lin_unprojection@@YAHPAUunprojection_mode@@PBUcylinder@primitives@@HPBUcapsule@3@HPAUcontact@@PAUgeom_contact_area@@@Z 35183be0 f   linunprojectionchecks.obj
 0001:00183080       ?capsule_cylinder_lin_unprojection@@YAHPAUunprojection_mode@@PBUcapsule@primitives@@HPBUcylinder@3@HPAUcontact@@PAUgeom_contact_area@@@Z 35184080 f   linunprojectionchecks.obj
 0001:00183130       ?capsule_capsule_lin_unprojection@@YAHPAUunprojection_mode@@PBUcapsule@primitives@@H1HPAUcontact@@PAUgeom_contact_area@@@Z 35184130 f   linunprojectionchecks.obj
 0001:00183ae0       ?sphere_capsule_lin_unprojection@@YAHPAUunprojection_mode@@PBUsphere@primitives@@HPBUcapsule@3@HPAUcontact@@PAUgeom_contact_area@@@Z 35184ae0 f   linunprojectionchecks.obj
 0001:00183f60       ?capsule_sphere_lin_unprojection@@YAHPAUunprojection_mode@@PBUcapsule@primitives@@HPBUsphere@3@HPAUcontact@@PAUgeom_contact_area@@@Z 35184f60 f   linunprojectionchecks.obj
 0001:00184100       ?SetParams@COBBTree@@QAEXHHM@Z 35185100 f   obbtree.obj
 0001:00184120       ?SetGeomConvex@COBBTree@@UAEXXZ 35185120 f   obbtree.obj
 0001:00184140       ?ReleaseLastSweptBVs@COBBTree@@UAEXH@Z 35185140 f   obbtree.obj
 0001:00184140       ?ReleaseLastBVs@COBBTree@@UAEXH@Z 35185140 f   obbtree.obj
 0001:00184140       ?ReleaseLastBVs@CAABBTree@@UAEXH@Z 35185140 f   aabbtree.obj
 0001:00184160       ?GetNodeContents@COBBTree@@UAEHHPAUBV@@HHPAUgeometry_under_test@@1@Z 35185160 f   obbtree.obj
 0001:001841c0       ?CleanupAfterIntersectionTest@COBBTree@@UAEXPAUgeometry_under_test@@@Z 351851c0 f   obbtree.obj
 0001:001841c0       ?CleanupAfterIntersectionTest@CAABBTree@@UAEXPAUgeometry_under_test@@@Z 351851c0 f   aabbtree.obj
 0001:00184260       ?SanityCheck@COBBTree@@UAEHXZ 35185260 f   obbtree.obj
 0001:00184270       ?SplitPriority@COBBTree@@UAEMPBUBV@@@Z 35185270 f   obbtree.obj
 0001:001842a0       ?MarkUsedTriangle@COBBTree@@UAEXHPAUgeometry_under_test@@@Z 351852a0 f   obbtree.obj
 0001:00184390       ?PrepareForIntersectionTest@COBBTree@@UAEHPAUgeometry_under_test@@PAVCGeometry@@0@Z 35185390 f   obbtree.obj
 0001:00184480       ?GetMemoryStatistics@COBBTree@@UAEXPAVICrySizer@@@Z 35185480 f   obbtree.obj
 0001:001844f0       ?GetBBox@COBBTree@@UAEXPAUbox@primitives@@@Z 351854f0 f   obbtree.obj
 0001:001845a0       ?GetNodeBV@COBBTree@@UAEXAAPAUBV@@HH@Z 351855a0 f   obbtree.obj
 0001:001846c0       ?GetNodeBV@COBBTree@@UAEXAAPAUBV@@ABU?$Vec3_tpl@M@@MHH@Z 351856c0 f   obbtree.obj
 0001:001847f0       ?GetNodeChildrenBVs@COBBTree@@UAEXPBUBV@@AAPAU2@1H@Z 351857f0 f   obbtree.obj
 0001:001849d0       ?GetNodeChildrenBVs@COBBTree@@UAEXPBUBV@@ABU?$Vec3_tpl@M@@MAAPAU2@2H@Z 351859d0 f   obbtree.obj
 0001:00184bf0       ?Save@COBBTree@@UAEXAAVCMemStream@@@Z 35185bf0 f   obbtree.obj
 0001:00184d20       ?Load@COBBTree@@UAEXAAVCMemStream@@PAVCGeometry@@@Z 35185d20 f   obbtree.obj
 0001:00184e30       ??$ComputeMeshEigenBasis@H@@YAXV?$strided_pointer@$$CBU?$Vec3_tpl@M@@@@V?$strided_pointer@H@@HPAU?$Vec3_tpl@N@@AAU2@@Z 35185e30 f i obbtree.obj
 0001:001855c0       ?BuildNode@COBBTree@@QAEMHHHH@Z 351865c0 f   obbtree.obj
 0001:00186ac0       ?GetNodeBV@COBBTree@@UAEXABU?$Matrix33_tpl@M@@ABU?$Vec3_tpl@M@@MAAPAUBV@@HH@Z 35187ac0 f   obbtree.obj
 0001:00186e10       ?GetNodeChildrenBVs@COBBTree@@UAEXABU?$Matrix33_tpl@M@@ABU?$Vec3_tpl@M@@MPBUBV@@AAPAU4@3H@Z 35187e10 f   obbtree.obj
 0001:00187470       ?Build@COBBTree@@UAEMPAVCGeometry@@@Z 35188470 f   obbtree.obj
 0001:00187610       ?box_ray_overlap_check@@YAHPBUbox@primitives@@PBUray@2@PAVCOverlapChecker@@@Z 35188610 f   overlapchecks.obj
 0001:00187930       ?ray_box_overlap_check@@YAHPBUray@primitives@@PBUbox@2@PAVCOverlapChecker@@@Z 35188930 f   overlapchecks.obj
 0001:00187950       ?box_sphere_overlap_check@@YAHPBUbox@primitives@@PBUsphere@2@PAVCOverlapChecker@@@Z 35188950 f   overlapchecks.obj
 0001:00187ad0       ?sphere_box_overlap_check@@YAHPBUsphere@primitives@@PBUbox@2@PAVCOverlapChecker@@@Z 35188ad0 f   overlapchecks.obj
 0001:00187af0       ?sphere_sphere_overlap_check@@YAHPBUsphere@primitives@@0PAVCOverlapChecker@@@Z 35188af0 f   overlapchecks.obj
 0001:00187b50       ?heightfield_sphere_overlap_check@@YAHPBUheightfield@primitives@@PBUsphere@2@PAVCOverlapChecker@@@Z 35188b50 f   overlapchecks.obj
 0001:00187d50       ?sphere_heightfield_overlap_check@@YAHPBUsphere@primitives@@PBUheightfield@2@PAVCOverlapChecker@@@Z 35188d50 f   overlapchecks.obj
 0001:00187d70       ?box_tri_overlap_check@@YAHPBUbox@primitives@@PBUtriangle@2@PAVCOverlapChecker@@@Z 35188d70 f   overlapchecks.obj
 0001:00188400       ?tri_box_overlap_check@@YAHPBUtriangle@primitives@@PBUbox@2@PAVCOverlapChecker@@@Z 35189400 f   overlapchecks.obj
 0001:00188420       ?tri_sphere_dist2@@YA?AV?$quotient_tpl@M@@PBUtriangle@primitives@@PBUsphere@3@AAH@Z 35189420 f   overlapchecks.obj
 0001:00188970       ?tri_sphere_overlap_check@@YAHPBUtriangle@primitives@@PBUsphere@2@PAVCOverlapChecker@@@Z 35189970 f   overlapchecks.obj
 0001:001889c0       ?sphere_tri_overlap_check@@YAHPBUsphere@primitives@@PBUtriangle@2@PAVCOverlapChecker@@@Z 351899c0 f   overlapchecks.obj
 0001:00188a10       ?box_box_overlap_check@@YAHPBUbox@primitives@@0PAVCOverlapChecker@@@Z 35189a10 f   overlapchecks.obj
 0001:00189300       ?box_heightfield_overlap_check@@YAHPBUbox@primitives@@PBUheightfield@2@PAVCOverlapChecker@@@Z 3518a300 f   overlapchecks.obj
 0001:00189e60       ?heightfield_box_overlap_check@@YAHPBUheightfield@primitives@@PBUbox@2@PAVCOverlapChecker@@@Z 3518ae60 f   overlapchecks.obj
 0001:00189e80       ?box_voxgrid_overlap_check@@YAHPBUbox@primitives@@PBUvoxelgrid@2@PAVCOverlapChecker@@@Z 3518ae80 f   overlapchecks.obj
 0001:0018a9f0       ?voxgrid_box_overlap_check@@YAHPBUvoxelgrid@primitives@@PBUbox@2@PAVCOverlapChecker@@@Z 3518b9f0 f   overlapchecks.obj
 0001:0018aa10       ?GetNodeContents@CRayBV@@UAEHHPAUBV@@HHPAUgeometry_under_test@@1@Z 3518ba10 f   raybv.obj
 0001:0018aa50       ?GetNodeBV@CRayBV@@UAEXAAPAUBV@@HH@Z 3518ba50 f   raybv.obj
 0001:0018aac0       ?GetNodeBV@CRayBV@@UAEXABU?$Matrix33_tpl@M@@ABU?$Vec3_tpl@M@@MAAPAUBV@@HH@Z 3518bac0 f   raybv.obj
 0001:0018ac60       ?PreparePrimitive@CRayGeom@@UAEHPAUgeom_world_data@@AAPAUprimitive@primitives@@H@Z 3518bc60 f   raygeom.obj
 0001:0018ae10       ?PrepareRay@CRayGeom@@QAEXPAUray@primitives@@PAUgeometry_under_test@@@Z 3518be10 f   raygeom.obj
 0001:0018af90       ?GetUnprojectionCandidates@CRayGeom@@UAEHHPBUcontact@@AAPAUprimitive@primitives@@AAPAHPAUgeometry_under_test@@@Z 3518bf90 f   raygeom.obj
 0001:0018afe0       ?GetPrimitiveList@CRayGeom@@UAEHHHHPAUprimitive@primitives@@HPAUgeometry_under_test@@10PAD@Z 3518bfe0 f   raygeom.obj
 0001:0018b010       ?RegisterIntersection@CRayGeom@@UAEHPAUprimitive@primitives@@0PAUgeometry_under_test@@1PAUprim_inters@@@Z 3518c010 f   raygeom.obj
 0001:0018b220       ?GetBBox@CRayGeom@@UAEXPAUbox@primitives@@@Z 3518c220 f   raygeom.obj
 0001:0018b320       ?PrepareForIntersectionTest@CRayGeom@@UAEHPAUgeometry_under_test@@PAVCGeometry@@0_N@Z 3518c320 f   raygeom.obj
 0001:0018b3c0       ?tri_tri_rot_unprojection@@YAHPAUunprojection_mode@@PBUtriangle@primitives@@H1HPAUcontact@@PAUgeom_contact_area@@@Z 3518c3c0 f   rotunprojectionchecks.obj
 0001:0018dc50       ?ray_tri_rot_unprojection@@YAHPAUunprojection_mode@@PBUray@primitives@@HPBUtriangle@3@HPAUcontact@@PAUgeom_contact_area@@@Z 3518ec50 f   rotunprojectionchecks.obj
 0001:0018f500       ?tri_ray_rot_unprojection@@YAHPAUunprojection_mode@@PBUtriangle@primitives@@HPBUray@3@HPAUcontact@@PAUgeom_contact_area@@@Z 35190500 f   rotunprojectionchecks.obj
 0001:0018f860       ?ray_box_rot_unprojection@@YAHPAUunprojection_mode@@PBUray@primitives@@HPBUbox@3@HPAUcontact@@PAUgeom_contact_area@@@Z 35190860 f   rotunprojectionchecks.obj
 0001:00191020       ?box_ray_rot_unprojection@@YAHPAUunprojection_mode@@PBUbox@primitives@@HPBUray@3@HPAUcontact@@PAUgeom_contact_area@@@Z 35192020 f   rotunprojectionchecks.obj
 0001:00191380       ?ray_cyl_rot_unprojection@@YAHPAUunprojection_mode@@PBUray@primitives@@HPBUcylinder@3@HPAUcontact@@PAUgeom_contact_area@@@Z 35192380 f   rotunprojectionchecks.obj
 0001:001970b0       ?cyl_ray_rot_unprojection@@YAHPAUunprojection_mode@@PBUcylinder@primitives@@HPBUray@3@HPAUcontact@@PAUgeom_contact_area@@@Z 351980b0 f   rotunprojectionchecks.obj
 0001:00197410       ?ray_capsule_rot_unprojection@@YAHPAUunprojection_mode@@PBUray@primitives@@HPBUcapsule@3@HPAUcontact@@PAUgeom_contact_area@@@Z 35198410 f   rotunprojectionchecks.obj
 0001:0019cf40       ?capsule_ray_rot_unprojection@@YAHPAUunprojection_mode@@PBUcapsule@primitives@@HPBUray@3@HPAUcontact@@PAUgeom_contact_area@@@Z 3519df40 f   rotunprojectionchecks.obj
 0001:0019d2a0       ?ray_sphere_rot_unprojection@@YAHPAUunprojection_mode@@PBUray@primitives@@HPBUsphere@3@HPAUcontact@@PAUgeom_contact_area@@@Z 3519e2a0 f   rotunprojectionchecks.obj
 0001:0019f210       ?sphere_ray_rot_unprojection@@YAHPAUunprojection_mode@@PBUsphere@primitives@@HPBUray@3@HPAUcontact@@PAUgeom_contact_area@@@Z 351a0210 f   rotunprojectionchecks.obj
 0001:0019f570       ?PrepGeomExt@@YAPAUIGeometry@@PAU1@@Z 351a0570 f   rwi.obj
 0001:0019f580       ??0entity_grid_checker@@QAE@XZ 351a0580 f i rwi.obj
 0001:0019f770       ?RayWater@CPhysicalWorld@@QAEXABU?$Vec3_tpl@M@@0AAUentity_grid_checker@@HHPAUray_hit@@@Z 351a0770 f   rwi.obj
 0001:0019fbc0       ??$ReallocQueue@USRwiRequest@@@CPhysicalWorld@@QAEXAAPAUSRwiRequest@@HAAH11H@Z 351a0bc0 f i rwi.obj
 0001:0019fcd0       ?check_cell@entity_grid_checker@@QAEHABU?$Vec2_tpl@H@@AAH@Z 351a0cd0 f i rwi.obj
 0001:001a1340       ?RayHeightfield@CPhysicalWorld@@QAEXABU?$Vec3_tpl@M@@AAU2@PAUray_hit@@HH@Z 351a2340 f   rwi.obj
 0001:001a16a0       ?TracePendingRays@CPhysicalWorld@@UAEHH@Z 351a26a0 f   rwi.obj
 0001:001a1c30       ??$DrawRayOnGrid@Uentity_grid_checker@@@@YAHPAUgrid@primitives@@AAU?$Vec3_tpl@M@@1AAUentity_grid_checker@@@Z 351a2c30 f i rwi.obj
 0001:001a22a0       ?RayWorldIntersection@CPhysicalWorld@@UAEHABUSRWIParams@IPhysicalWorld@@PBDH@Z 351a32a0 f   rwi.obj
 0001:001a3640       ?GetNodeContents@CSingleBoxTree@@UAEHHPAUBV@@HHPAUgeometry_under_test@@1@Z 351a4640 f   singleboxtree.obj
 0001:001a3690       ?PrepareForIntersectionTest@CSingleBoxTree@@UAEHPAUgeometry_under_test@@PAVCGeometry@@0@Z 351a4690 f   singleboxtree.obj
 0001:001a36b0       ?Build@CSingleBoxTree@@UAEMPAVCGeometry@@@Z 351a46b0 f   singleboxtree.obj
 0001:001a36d0       ?GetNodeBV@CSingleBoxTree@@UAEXAAPAUBV@@HH@Z 351a46d0 f   singleboxtree.obj
 0001:001a3780       ?GetNodeBV@CSingleBoxTree@@UAEXAAPAUBV@@ABU?$Vec3_tpl@M@@MHH@Z 351a4780 f   singleboxtree.obj
 0001:001a3870       ?MarkUsedTriangle@CSingleBoxTree@@UAEXHPAUgeometry_under_test@@@Z 351a4870 f   singleboxtree.obj
 0001:001a3890       ?GetBBox@CSingleBoxTree@@UAEXPAUbox@primitives@@@Z 351a4890 f   singleboxtree.obj
 0001:001a3900       ?GetMemoryStatistics@CSingleBoxTree@@UAEXPAVICrySizer@@@Z 351a4900 f   singleboxtree.obj
 0001:001a3940       ?SetBox@CSingleBoxTree@@QAEXPAUbox@primitives@@@Z 351a4940 f   singleboxtree.obj
 0001:001a3a10       ?Save@CSingleBoxTree@@UAEXAAVCMemStream@@@Z 351a4a10 f   singleboxtree.obj
 0001:001a3a80       ?Load@CSingleBoxTree@@UAEXAAVCMemStream@@PAVCGeometry@@@Z 351a4a80 f   singleboxtree.obj
 0001:001a3ac0       ?GetNodeBV@CSingleBoxTree@@UAEXABU?$Matrix33_tpl@M@@ABU?$Vec3_tpl@M@@MAAPAUBV@@HH@Z 351a4ac0 f   singleboxtree.obj
 0001:001a3db0       ?GetNodeBV@CSingleBoxTree@@UAEXABU?$Matrix33_tpl@M@@ABU?$Vec3_tpl@M@@MAAPAUBV@@1MHH@Z 351a4db0 f   singleboxtree.obj
 0001:001a4130       ?PrepareForIntersectionTest@CSphereGeom@@UAEHPAUgeometry_under_test@@PAVCGeometry@@0_N@Z 351a5130 f   spheregeom.obj
 0001:001a41d0       ?GetMemoryStatistics@CSphereGeom@@UAEXPAVICrySizer@@@Z 351a51d0 f   spheregeom.obj
 0001:001a41f0       ?CreateSphere@CSphereGeom@@QAEPAV1@PAUsphere@primitives@@@Z 351a51f0 f   spheregeom.obj
 0001:001a42b0       ?CalcPhysicalProperties@CSphereGeom@@UAEHPAUphys_geometry@@@Z 351a52b0 f   spheregeom.obj
 0001:001a4330       ?PointInsideStatus@CSphereGeom@@UAEHABU?$Vec3_tpl@M@@@Z 351a5330 f   spheregeom.obj
 0001:001a4390       ?ComputeExtent@CSphereGeom@@UAEMAAUGeomQuery@@W4EGeomForm@@@Z 351a5390 f   spheregeom.obj
 0001:001a43e0       ?PreparePrimitive@CSphereGeom@@UAEHPAUgeom_world_data@@AAPAUprimitive@primitives@@H@Z 351a53e0 f   spheregeom.obj
 0001:001a4500       ?GetPrimitiveList@CSphereGeom@@UAEHHHHPAUprimitive@primitives@@HPAUgeometry_under_test@@10PAD@Z 351a5500 f   spheregeom.obj
 0001:001a4610       ?GetUnprojectionCandidates@CSphereGeom@@UAEHHPBUcontact@@AAPAUprimitive@primitives@@AAPAHPAUgeometry_under_test@@@Z 351a5610 f   spheregeom.obj
 0001:001a4730       ?CalculateBuoyancy@CSphereGeom@@UAEMPBUplane@primitives@@PBUgeom_world_data@@AAU?$Vec3_tpl@M@@@Z 351a5730 f   spheregeom.obj
 0001:001a4950       ?DrawWireframe@CSphereGeom@@UAEXPAUIPhysRenderer@@PAUgeom_world_data@@HH@Z 351a5950 f   spheregeom.obj
 0001:001a4a20       ?FindClosestPoint@CSphereGeom@@UAEHPAUgeom_world_data@@AAH1ABU?$Vec3_tpl@M@@2PAU3@H@Z 351a5a20 f   spheregeom.obj
 0001:001a4e30       ?UnprojectSphere@CSphereGeom@@UAEHU?$Vec3_tpl@M@@MMPAUcontact@@@Z 351a5e30 f   spheregeom.obj
 0001:001a4f90       ?CalculateMediumResistance@CSphereGeom@@UAEXPBUplane@primitives@@PBUgeom_world_data@@AAU?$Vec3_tpl@M@@2@Z 351a5f90 f   spheregeom.obj
 0001:001a58c0       ?CalcVolumetricPressure@CSphereGeom@@UAEXPAUgeom_world_data@@ABU?$Vec3_tpl@M@@MM1AAU3@2@Z 351a68c0 f   spheregeom.obj
 0001:001a5a30       ?DrawToOcclusionCubemap@CSphereGeom@@UAEHPBUgeom_world_data@@HHHPAUSOcclusionCubeMap@@@Z 351a6a30 f   spheregeom.obj
 0001:001a5e90       ?Save@CSphereGeom@@UAEXAAVCMemStream@@@Z 351a6e90 f   spheregeom.obj
 0001:001a5ef0       ?Load@CSphereGeom@@UAEXAAVCMemStream@@@Z 351a6ef0 f   spheregeom.obj
 0001:001a5f40       ?GetRandomPos@CSphereGeom@@UAEXAAURandomPos@@AAUGeomQuery@@W4EGeomForm@@@Z 351a6f40 f   spheregeom.obj
 0001:001a6150       ?GetParams@CTetrLattice@@UAEHPAUpe_params@@@Z 351a7150 f   tetrlattice.obj
 0001:001a61a0       ??_GITetrLattice@@UAEPAXI@Z 351a71a0 f i tetrlattice.obj
 0001:001a61a0       ??_GIPhysicalEntityIt@@UAEPAXI@Z 351a71a0 f i physicalworld.obj
 0001:001a61a0       ??_GCPhysicalEntityIt@CPhysicalWorld@@UAEPAXI@Z 351a71a0 f i physicalworld.obj
 0001:001a61a0       ??_EIBreakableGrid2d@@UAEPAXI@Z 351a71a0 f i geoman.obj
 0001:001a61a0       ??_EITetrLattice@@UAEPAXI@Z 351a71a0 f i tetrlattice.obj
 0001:001a61a0       ??_EIPhysicalEntityIt@@UAEPAXI@Z 351a71a0 f i physicalworld.obj
 0001:001a61a0       ??_GIBreakableGrid2d@@UAEPAXI@Z 351a71a0 f i geoman.obj
 0001:001a61a0       ??_ECPhysicalEntityIt@CPhysicalWorld@@UAEPAXI@Z 351a71a0 f i physicalworld.obj
 0001:001a61d0       ??0CTetrLattice@@QAE@PAUIPhysicalWorld@@@Z 351a71d0 f   tetrlattice.obj
 0001:001a6270       ?Release@CBreakableGrid2d@@UAEXXZ 351a7270 f i geoman.obj
 0001:001a6270       ?Release@CTetrLattice@@UAEXXZ 351a7270 f i tetrlattice.obj
 0001:001a6270       ?destroy@sp_counted_base@detail@boost@@UAEXXZ 351a7270 f i CryPhysics.obj
 0001:001a6270       ?Release@CPhysicalWorld@@UAEXXZ 351a7270 f i physicalworld.obj
 0001:001a6280       ??1CTetrLattice@@UAE@XZ    351a7280 f   tetrlattice.obj
 0001:001a6300       ?SetParams@CTetrLattice@@UAEHPAUpe_params@@@Z 351a7300 f   tetrlattice.obj
 0001:001a6540       ??4STetrahedron@@QAEAAU0@ABU0@@Z 351a7540 f i tetrlattice.obj
 0001:001a6650       ?DrawWireframe@CTetrLattice@@UAEXPAUIPhysRenderer@@PAUgeom_world_data@@H@Z 351a7650 f   tetrlattice.obj
 0001:001a6c10       ?CreateSkinMesh@CTetrLattice@@UAEPAUIGeometry@@H@Z 351a7c10 f   tetrlattice.obj
 0001:001a6d90       ?CropSpikes@CBreakableGrid2d@@QAEHHHPAHHHHM@Z 351a7d90 f i tetrlattice.obj
 0001:001a71a0       ?BreakIntoChunks@CBreakableGrid2d@@UAEPAHABU?$Vec2_tpl@M@@MAAPAU2@HMHMM@Z 351a81a0 f   tetrlattice.obj
 0001:001a8580       ??_GCTetrLattice@@UAEPAXI@Z 351a9580 f i tetrlattice.obj
 0001:001a8580       ??_ECTetrLattice@@UAEPAXI@Z 351a9580 f i tetrlattice.obj
 0001:001a85b0       ??0CTetrLattice@@QAE@PAV0@H@Z 351a95b0 f   tetrlattice.obj
 0001:001a88a0       ?CreateLattice@CTetrLattice@@QAEPAV1@PBU?$Vec3_tpl@M@@HPBHH@Z 351a98a0 f   tetrlattice.obj
 0001:001a9a80       ?AddImpulse@CTetrLattice@@QAEHABU?$Vec3_tpl@M@@000M@Z 351aaa80 f   tetrlattice.obj
 0001:001a9fa0       ?Defragment@CTetrLattice@@QAEHXZ 351aafa0 f   tetrlattice.obj
 0001:001aa260       ?SetGrid@CTetrLattice@@QAEXABUbox@primitives@@@Z 351ab260 f   tetrlattice.obj
 0001:001ab2c0       ?Subtract@CTetrLattice@@QAEXPAUIGeometry@@PBUgeom_world_data@@1@Z 351ac2c0 f   tetrlattice.obj
 0001:001acc40       ?CheckStructure@CTetrLattice@@QAEHMABU?$Vec3_tpl@M@@PBUplane@primitives@@HPAUpe_explosion@@HH@Z 351adc40 f   tetrlattice.obj
 0001:001b10a0       ?Split@CTetrLattice@@QAEXPAPAVCTriMesh@@HPAPAV1@@Z 351b20a0 f   tetrlattice.obj
 0001:001b2230       ?CheckPoint@CTetrLattice@@UAEHABU?$Vec3_tpl@M@@PAHPAM@Z 351b3230 f   tetrlattice.obj
 0001:001b2b40       ?SetMesh@CTetrLattice@@QAEXPAVCTriMesh@@@Z 351b3b40 f   tetrlattice.obj
 0001:001b2b80       ?Generate@CBreakableGrid2d@@QAEXPAU?$Vec2_tpl@M@@HABU?$Vec2_tpl@H@@HH@Z 351b3b80 f   tetrlattice.obj
 0001:001b3b40       ?MaxPrimsInNode@COBBTree@@UAEHXZ 351b4b40 f i trimesh.obj
 0001:001b3b50       ?GetNodeBV@CRayBV@@UAEXABU?$Matrix33_tpl@M@@ABU?$Vec3_tpl@M@@MAAPAUBV@@1MHH@Z 351b4b50 f i livingentity.obj
 0001:001b3b50       ?GetNodeBV@COBBTree@@UAEXABU?$Matrix33_tpl@M@@ABU?$Vec3_tpl@M@@MAAPAUBV@@1MHH@Z 351b4b50 f i trimesh.obj
 0001:001b3b50       ?GetNodeBV@CHeightfieldBV@@UAEXABU?$Matrix33_tpl@M@@ABU?$Vec3_tpl@M@@MAAPAUBV@@1MHH@Z 351b4b50 f i waterman.obj
 0001:001b3b50       ?GetNodeBV@CAABBTree@@UAEXABU?$Matrix33_tpl@M@@ABU?$Vec3_tpl@M@@MAAPAUBV@@1MHH@Z 351b4b50 f i trimesh.obj
 0001:001b3b60       ?GetNodeContentsIdx@COBBTree@@UAEHHAAH@Z 351b4b60 f i trimesh.obj
 0001:001b3b90       ??_GCOBBTree@@UAEPAXI@Z    351b4b90 f i trimesh.obj
 0001:001b3b90       ??_ECOBBTree@@UAEPAXI@Z    351b4b90 f i trimesh.obj
 0001:001b3bf0       ??0InitTriMeshGlobals@@QAE@XZ 351b4bf0 f   trimesh.obj
 0001:001b3c50       ?qsort@@YAXPAHHH@Z         351b4c50 f   trimesh.obj
 0001:001b3cd0       ?CleanupAfterIntersectionTest@CTriMesh@@UAEXPAUgeometry_under_test@@@Z 351b4cd0 f   trimesh.obj
 0001:001b3e30       ?GetNeighbouringEdgeId@CTriMesh@@QAEHHH@Z 351b4e30 f   trimesh.obj
 0001:001b3f00       ?CleanupGlobalLoadState@CTriMesh@@SAXXZ 351b4f00 f   trimesh.obj
 0001:001b3f40       ?GetMemoryUsage@TriMeshStaticData@@YAXPAVICrySizer@@@Z 351b4f40 f   trimesh.obj
 0001:001b3f90       ?SanityCheck@CTriMesh@@UAEHXZ 351b4f90 f   trimesh.obj
 0001:001b3fa0       ??1?$vector2_w_enforcer@M@@QAE@XZ 351b4fa0 f i trimesh.obj
 0001:001b4030       ?MaxPrimsInNode@CAABBTree@@UAEHXZ 351b5030 f i trimesh.obj
 0001:001b4040       ?GetNodeContentsIdx@CAABBTree@@UAEHHAAH@Z 351b5040 f i trimesh.obj
 0001:001b4070       ??_GCAABBTree@@UAEPAXI@Z   351b5070 f i trimesh.obj
 0001:001b4070       ??_ECAABBTree@@UAEPAXI@Z   351b5070 f i trimesh.obj
 0001:001b40d0       ?GetMaxSkipDim@CAABBTree@@UAEMXZ 351b50d0 f i trimesh.obj
 0001:001b4100       ?GetMaxSkipDim@COBBTree@@UAEMXZ 351b5100 f i trimesh.obj
 0001:001b4140       ?TriRandomPoint@@YAXQAMW4EGeomForm@@@Z 351b5140 f i trimesh.obj
 0001:001b4260       ??1CTriMesh@@UAE@XZ        351b5260 f   trimesh.obj
 0001:001b43e0       ?GetSnapshotVersion@CWheeledVehicleEntity@@UAEHXZ 351b53e0 f i wheeledvehicleentity.obj
 0001:001b43e0       ?GetType@CPhysicalEntity@@UBE?AW4pe_type@@XZ 351b53e0 f i physicalentity.obj
 0001:001b43e0       ?MaxPrimsInNode@CBVTree@@UAEHXZ 351b53e0 f i livingentity.obj
 0001:001b43e0       ?GetType@CPhysicalStub@@UBE?AW4pe_type@@XZ 351b53e0 f i physarea.obj
 0001:001b43e0       ?SanityCheck@CGeometry@@UAEHXZ 351b53e0 f i livingentity.obj
 0001:001b43e0       ?PostSetStateFromSnapshot@CPhysicalEntity@@UAEHXZ 351b53e0 f i livingentity.obj
 0001:001b43e0       ?GetType@CTriMesh@@UAEHXZ  351b53e0 f i trimesh.obj
 0001:001b43e0       ?default_overlap_check@@YAHPBUprimitive@primitives@@0PAVCOverlapChecker@@@Z 351b53e0 f i overlapchecks.obj
 0001:001b43e0       ?GetType@CAABBTree@@UAEHXZ 351b53e0 f i trimesh.obj
 0001:001b43e0       ?IsAPrimitive@CPrimitive@@UAEHXZ 351b53e0 f i livingentity.obj
 0001:001b43e0       ?IsAPrimitive@CRayGeom@@UAEHXZ 351b53e0 f i livingentity.obj
 0001:001b43e0       ?FlushDynPool@CPhysicalWorld@@UAEHXZ 351b53e0 f i physicalworld.obj
 0001:001b43e0       ?SanityCheck@CBVTree@@UAEHXZ 351b53e0 f i livingentity.obj
 0001:001b43e0       ?GetPrimitiveCount@CGeometry@@UAEHXZ 351b53e0 f i livingentity.obj
 0001:001b43f0       ?PointInsideStatus@CTriMesh@@UAEHABU?$Vec3_tpl@M@@@Z 351b53f0 f i trimesh.obj
 0001:001b4410       ?GetBVTree@CTriMesh@@UAEPAVCBVTree@@XZ 351b5410 f i trimesh.obj
 0001:001b4420       ?GetRandomPos@CTriMesh@@UAEXAAURandomPos@@AAUGeomQuery@@W4EGeomForm@@@Z 351b5420 f   trimesh.obj
 0001:001b45a0       ?GetCenter@CTriMesh@@UAE?AU?$Vec3_tpl@M@@XZ 351b55a0 f   trimesh.obj
 0001:001b47a0       ?GetFeature@CTriMesh@@UAEHHHPAU?$Vec3_tpl@M@@@Z 351b57a0 f   trimesh.obj
 0001:001b4870       ?PrepareTriangle@CTriMesh@@QAEXHPAUtriangle@primitives@@PBUgeometry_under_test@@@Z 351b5870 f   trimesh.obj
 0001:001b4b70       ?PreparePrimitive@CTriMesh@@UAEHPAUgeom_world_data@@AAPAUprimitive@primitives@@H@Z 351b5b70 f   trimesh.obj
 0001:001b4e70       ?GetPrimitiveList@CTriMesh@@UAEHHHHPAUprimitive@primitives@@HPAUgeometry_under_test@@10PAD@Z 351b5e70 f   trimesh.obj
 0001:001b54d0       ?HashTrianglesToPlane@CTriMesh@@QAEXABUcoord_plane@primitives@@ABU?$Vec2_tpl@M@@AAUgrid@3@AAPAH3M@Z 351b64d0 f   trimesh.obj
 0001:001b61c0       ?CalculateMediumResistance@CTriMesh@@UAEXPBUplane@primitives@@PBUgeom_world_data@@AAU?$Vec3_tpl@M@@2@Z 351b71c0 f   trimesh.obj
 0001:001b6300       ?DrawToOcclusionCubemap@CTriMesh@@UAEHPBUgeom_world_data@@HHHPAUSOcclusionCubeMap@@@Z 351b7300 f   trimesh.obj
 0001:001b6610       ?DrawWireframe@CTriMesh@@UAEXPAUIPhysRenderer@@PAUgeom_world_data@@HH@Z 351b7610 f   trimesh.obj
 0001:001b6960       ?GetMemoryStatistics@CTriMesh@@UAEXPAVICrySizer@@@Z 351b7960 f   trimesh.obj
 0001:001b6c80       ?Save@CTriMesh@@UAEXAAVCMemStream@@@Z 351b7c80 f   trimesh.obj
 0001:001b71a0       ?CompactMemory@CTriMesh@@UAEXXZ 351b81a0 f   trimesh.obj
 0001:001b72e0       ?ExpandVtxList@CTriMesh@@QAEHXZ 351b82e0 f   trimesh.obj
 0001:001b73f0       ?CroppedRectArea@@YAMABU?$Vec2_tpl@M@@000@Z 351b83f0 f   trimesh.obj
 0001:001b75d0       ??$qsort@M@@YAXPAHV?$strided_pointer@M@@HH@Z 351b85d0 f i trimesh.obj
 0001:001b76b0       ??0CTriMesh@@QAE@XZ        351b86b0 f   trimesh.obj
 0001:001b77e0       ??_ECTriMesh@@UAEPAXI@Z    351b87e0 f i trimesh.obj
 0001:001b77e0       ??_GCTriMesh@@UAEPAXI@Z    351b87e0 f i trimesh.obj
 0001:001b7810       ?CalculateTopology@CTriMesh@@QAEHPAHH@Z 351b8810 f   trimesh.obj
 0001:001b7eb0       ?RebuildBVTree@CTriMesh@@QAEXPAVCBVTree@@@Z 351b8eb0 f   trimesh.obj
 0001:001b8780       ?BuildIslandMap@CTriMesh@@QAEHXZ 351b9780 f   trimesh.obj
 0001:001b8d90       ?CompactTriangleList@CTriMesh@@QAEXPAH_N@Z 351b9d90 f   trimesh.obj
 0001:001b90d0       ?ComputeExtent@CTriMesh@@UAEMAAUGeomQuery@@W4EGeomForm@@@Z 351ba0d0 f   trimesh.obj
 0001:001b9520       ?IsConvex@CTriMesh@@UAEHM@Z 351ba520 f   trimesh.obj
 0001:001b9780       ?TraceTriangleInters@CTriMesh@@QAEHHQAPAUprimitive@primitives@@HHPAUprim_inters@@PAUgeometry_under_test@@PAUborder_trace@@@Z 351ba780 f   trimesh.obj
 0001:001b9c80       ?GetUnprojectionCandidates@CTriMesh@@UAEHHPBUcontact@@AAPAUprimitive@primitives@@AAPAHPAUgeometry_under_test@@@Z 351bac80 f   trimesh.obj
 0001:001ba4f0       ?update_unprojection@@YAXNPAUunprojection_mode@@PAUgeometry_under_test@@@Z 351bb4f0 f   trimesh.obj
 0001:001ba9b0       ?PreparePolygon@CTriMesh@@UAEHPAUcoord_plane@primitives@@HHPAUgeometry_under_test@@AAPAU?$Vec2_tpl@M@@AAPAH3@Z 351bb9b0 f   trimesh.obj
 0001:001bbcc0       ?PreparePolyline@CTriMesh@@UAEHPAUcoord_plane@primitives@@HHPAUgeometry_under_test@@AAPAU?$Vec2_tpl@M@@AAPAH3@Z 351bccc0 f   trimesh.obj
 0001:001bc6a0       ?FindClosestPoint@CTriMesh@@UAEHPAUgeom_world_data@@AAH1ABU?$Vec3_tpl@M@@2PAU3@H@Z 351bd6a0 f   trimesh.obj
 0001:001beb50       ?PointInsideStatusMesh@CTriMesh@@UAEHABU?$Vec3_tpl@M@@PAUindexed_triangle@primitives@@@Z 351bfb50 f   trimesh.obj
 0001:001bef30       ?PrepareForRayTest@CTriMesh@@UAEXM@Z 351bff30 f   trimesh.obj
 0001:001bf620       ?Intersect@CTriMesh@@UAEHPAUIGeometry@@PAUgeom_world_data@@1PAUintersection_params@@AAPAUgeom_contact@@@Z 351c0620 f   trimesh.obj
 0001:001c1df0       ?CalcVolumetricPressure@CTriMesh@@UAEXPAUgeom_world_data@@ABU?$Vec3_tpl@M@@MM1AAU3@2@Z 351c2df0 f   trimesh.obj
 0001:001c3020       ?RemapForeignIdx@CTriMesh@@UAEXPAH0H@Z 351c4020 f   trimesh.obj
 0001:001c3600       ?AppendVertices@CTriMesh@@UAEXPAU?$Vec3_tpl@M@@PAHH@Z 351c4600 f   trimesh.obj
 0001:001c3790       ?GetIslandDisk@CTriMesh@@QAEMHABU?$Vec3_tpl@M@@AAU2@1AAM@Z 351c4790 f   trimesh.obj
 0001:001c4520       ?Load@CTriMesh@@UAEXAAVCMemStream@@V?$strided_pointer@$$CBU?$Vec3_tpl@M@@@@V?$strided_pointer@G@@PAD@Z 351c5520 f   trimesh.obj
 0001:001c4fc0       ?UnprojectSphere@CTriMesh@@UAEHU?$Vec3_tpl@M@@MMPAUcontact@@@Z 351c5fc0 f   trimesh.obj
 0001:001c60a0       ?SVD3x3@@YA?AU?$Vec3_tpl@M@@ABU?$Matrix33_tpl@M@@@Z 351c70a0 f   trimesh.obj
 0001:001c62f0       ?CreateTriMesh@CTriMesh@@QAEPAV1@V?$strided_pointer@$$CBU?$Vec3_tpl@M@@@@V?$strided_pointer@G@@PADPAHHHHHM@Z 351c72f0 f   trimesh.obj
 0001:001c7810       ?SplitIntoIslands@CTriMesh@@QAEPAV1@PAUplane@primitives@@HH@Z 351c8810 f   trimesh.obj
 0001:001c8d00       ?FilterMesh@CTriMesh@@QAEHMM@Z 351c9d00 f   trimesh.obj
 0001:001ca220       ?CalcPhysicalProperties@CTriMesh@@UAEHPAUphys_geometry@@@Z 351cb220 f   trimesh.obj
 0001:001ca6d0       ?PrepareForIntersectionTest@CTriMesh@@UAEHPAUgeometry_under_test@@PAVCGeometry@@0_N@Z 351cb6d0 f   trimesh.obj
 0001:001ca9b0       ?RegisterIntersection@CTriMesh@@UAEHPAUprimitive@primitives@@0PAUgeometry_under_test@@1PAUprim_inters@@@Z 351cb9b0 f   trimesh.obj
 0001:001ce2d0       ?Voxelize@CTriMesh@@QAE?AUvoxgrid@1@U?$Quat_tpl@M@@M@Z 351cf2d0 f   trimesh.obj
 0001:001cf270       ?Boxify@CTriMesh@@UAEHPAUbox@primitives@@HABUSBoxificationParams@IGeometry@@@Z 351d0270 f   trimesh.obj
 0001:001d48d0       ?Clone@CTriMesh@@QAEPAV1@PAV1@H@Z 351d58d0 f   trimesh.obj
 0001:001d4e90       ?CalculateBuoyancy@CTriMesh@@UAEMPBUplane@primitives@@PBUgeom_world_data@@AAU?$Vec3_tpl@M@@@Z 351d5e90 f   trimesh.obj
 0001:001d6440       ?GetVolume@CTriMesh@@UAEMXZ 351d7440 f   trimesh.obj
 0001:001d64c0       ?CleanupAfterIntersectionTest@CVoxelBV@@UAEXPAUgeometry_under_test@@@Z 351d74c0 f   voxelbv.obj
 0001:001d6560       ?GetBBox@CVoxelBV@@UAEXPAUbox@primitives@@@Z 351d7560 f   voxelbv.obj
 0001:001d6640       ?MarkUsedTriangle@CVoxelBV@@UAEXHPAUgeometry_under_test@@@Z 351d7640 f   voxelbv.obj
 0001:001d6690       ?GetNodeBV@CVoxelBV@@UAEXAAPAUBV@@HH@Z 351d7690 f   voxelbv.obj
 0001:001d68f0       ?project_box_on_3dgrid@@YAXPAUbox@primitives@@PAUgrid3d@2@PAUgeometry_under_test@@PAU?$Vec3_tpl@H@@@Z 351d78f0 f   voxelbv.obj
 0001:001d6fb0       ?GetNodeContents@CVoxelBV@@UAEHHPAUBV@@HHPAUgeometry_under_test@@1@Z 351d7fb0 f   voxelbv.obj
 0001:001d72f0       ?PrepareForIntersectionTest@CVoxelBV@@UAEHPAUgeometry_under_test@@PAVCGeometry@@0@Z 351d82f0 f   voxelbv.obj
 0001:001d7510       ?GetNodeBV@CVoxelBV@@UAEXABU?$Matrix33_tpl@M@@ABU?$Vec3_tpl@M@@MAAPAUBV@@HH@Z 351d8510 f   voxelbv.obj
 0001:001d7930       ?GetMemoryStatistics@CVoxelGeom@@UAEXPAVICrySizer@@@Z 351d8930 f   voxelgeom.obj
 0001:001d79d0       ?CreateVoxelGrid@CVoxelGeom@@QAEPAV1@PAUgrid3d@primitives@@@Z 351d89d0 f   voxelgeom.obj
 0001:001d8060       ?DrawToOcclusionCubemap@CVoxelGeom@@UAEHPBUgeom_world_data@@HHHPAUSOcclusionCubeMap@@@Z 351d9060 f   voxelgeom.obj
 0001:001d86a0       ?Intersect@CVoxelGeom@@UAEHPAUIGeometry@@PAUgeom_world_data@@1PAUintersection_params@@AAPAUgeom_contact@@@Z 351d96a0 f   voxelgeom.obj
 0001:001d9f40       ??0CryEvent@@QAE@XZ        351daf40 f   CryPhysics.obj
 0001:001d9f60       ??1CryEvent@@QAE@XZ        351daf60 f   CryPhysics.obj
 0001:001d9f70       ?Set@CryEvent@@QAEXXZ      351daf70 f   CryPhysics.obj
 0001:001d9f80       ?Wait@CryEvent@@QBEXXZ     351daf80 f   CryPhysics.obj
 0001:001d9f90       ?CryPureCallHandler@@YAXXZ 351daf90 f   CryPhysics.obj
 0001:001d9fa0       ?CryInvalidParameterHandler@@YAXPB_W00II@Z 351dafa0 f   CryPhysics.obj
 0001:001d9fb0       _ModuleInitISystem         351dafb0 f   CryPhysics.obj
 0001:001da060       ?cry_rand32@@YAIXZ         351db060 f   CryPhysics.obj
 0001:001da0a0       ?cry_frand@@YAMXZ          351db0a0 f   CryPhysics.obj
 0001:001da100       ?Init@_CryMemoryManagerPoolHelper@@SAXXZ 351db100 f i CryPhysics.obj
 0001:001da280       ?CryGetIMemoryManager@@YAPAUIMemoryManager@@XZ 351db280 f   CryPhysics.obj
 0001:001da2c0       ?CryInterlockedIncrement@@YAJPCH@Z 351db2c0 f   CryPhysics.obj
 0001:001da2d0       ?CryInterlockedDecrement@@YAJPCH@Z 351db2d0 f   CryPhysics.obj
 0001:001da2e0       ?CryInterlockedCompareExchange@@YAJPCJJJ@Z 351db2e0 f   CryPhysics.obj
 0001:001da300       ?CryCreateCriticalSectionInplace@@YAXPAX@Z 351db300 f   CryPhysics.obj
 0001:001da310       ?CryDeleteCriticalSectionInplace@@YAXPAX@Z 351db310 f   CryPhysics.obj
 0001:001da340       ?CryGetCurrentThreadId@@YAIXZ 351db340 f   CryPhysics.obj
 0001:001da350       _CryGetMemoryInfoForModule 351db350 f   CryPhysics.obj
 0001:001da350       _CryModuleGetMemoryInfo    351db350 f   CryPhysics.obj
 0001:001da3a0       ?OnSystemEvent@CSystemEventListner_Physics@@UAEXW4ESystemEvent@@II@Z 351db3a0 f i CryPhysics.obj
 0001:001da400       _CryModuleMalloc           351db400 f   CryPhysics.obj
 0001:001da490       _CryModuleFree             351db490 f   CryPhysics.obj
 0001:001da4f0       _CryModuleMemalign         351db4f0 f   CryPhysics.obj
 0001:001da580       ??2@YAPAXI@Z               351db580 f   CryPhysics.obj
 0001:001da5d0       ??_U@YAPAXI@Z              351db5d0 f   CryPhysics.obj
 0001:001da620       ??3@YAXPAX@Z               351db620 f   CryPhysics.obj
 0001:001da6a0       ??_V@YAXPAX@Z              351db6a0 f   CryPhysics.obj
 0001:001da720       ??_GICryUnknown@@MAEPAXI@Z 351db720 f i CryPhysics.obj
 0001:001da720       ??_GCEngineModule_CryPhysics@@MAEPAXI@Z 351db720 f i CryPhysics.obj
 0001:001da720       ??_EIPhysUtils@@UAEPAXI@Z  351db720 f i physicalworld.obj
 0001:001da720       ??_EICryUnknown@@MAEPAXI@Z 351db720 f i CryPhysics.obj
 0001:001da720       ??_GIPhysUtils@@UAEPAXI@Z  351db720 f i physicalworld.obj
 0001:001da720       ??_ECEngineModule_CryPhysics@@MAEPAXI@Z 351db720 f i CryPhysics.obj
 0001:001da750       ??_EICryFactory@@MAEPAXI@Z 351db750 f i CryPhysics.obj
 0001:001da750       ??_GICryFactory@@MAEPAXI@Z 351db750 f i CryPhysics.obj
 0001:001da780       ??0InitPhysicsGlobals@@QAE@XZ 351db780 f i CryPhysics.obj
 0001:001daca0       _CreatePhysicalWorld       351dbca0 f   CryPhysics.obj
 0001:001dadc0       ?GetFactory@CEngineModule_CryPhysics@@UBEPAUICryFactory@@XZ 351dbdc0 f i CryPhysics.obj
 0001:001dadd0       ?GetName@CEngineModule_CryPhysics@@MAEPBDXZ 351dbdd0 f i CryPhysics.obj
 0001:001dade0       ?GetCategory@CEngineModule_CryPhysics@@MAEPBDXZ 351dbde0 f i CryPhysics.obj
 0001:001dadf0       ?Initialize@CEngineModule_CryPhysics@@MAE_NAAUSSystemGlobalEnvironment@@ABUSSystemInitParams@@@Z 351dbdf0 f i CryPhysics.obj
 0001:001daee0       ??_GCSystemEventListner_Physics@@UAEPAXI@Z 351dbee0 f i CryPhysics.obj
 0001:001daee0       ??_ECSystemEventListner_Physics@@UAEPAXI@Z 351dbee0 f i CryPhysics.obj
 0001:001daee0       ??_EISystemEventListener@@UAEPAXI@Z 351dbee0 f i CryPhysics.obj
 0001:001daee0       ??_GISystemEventListener@@UAEPAXI@Z 351dbee0 f i CryPhysics.obj
 0001:001daf10       ??0CFactory@CEngineModule_CryPhysics@@AAE@XZ 351dbf10 f i CryPhysics.obj
 0001:001dafc0       ?GetClassNameA@CFactory@CEngineModule_CryPhysics@@UBEPBDXZ 351dbfc0 f i CryPhysics.obj
 0001:001dafd0       ?GetClassID@CFactory@CEngineModule_CryPhysics@@UBEABUCryGUID@@XZ 351dbfd0 f i CryPhysics.obj
 0001:001dafe0       ?ClassSupports@CFactory@CEngineModule_CryPhysics@@UBE_NABUCryGUID@@@Z 351dbfe0 f i CryPhysics.obj
 0001:001db030       ?ClassSupports@CFactory@CEngineModule_CryPhysics@@UBEXAAPBUCryGUID@@AAI@Z 351dc030 f i CryPhysics.obj
 0001:001db050       ?GetTriMesh@CBoxGeom@@UAEPAUIGeometry@@H@Z 351dc050 f i boxgeom.obj
 0001:001db050       ?RayTrace@CPhysicalEntity@@UAEHAAUSRayTraceRes@@@Z 351dc050 f i rwi.obj
 0001:001db050       ?IsConvex@CHeightfield@@UAEHM@Z 351dc050 f i waterman.obj
 0001:001db050       ?GetParams@CPhysicalStub@@UBEHPAUpe_params@@@Z 351dc050 f i physarea.obj
 0001:001db050       ?GetStatus@CPhysicalStub@@UBEHPAUpe_status@@@Z 351dc050 f i physarea.obj
 0001:001db050       ?GetContactCount@CPhysicalEntity@@UAEHH@Z 351dc050 f i livingentity.obj
 0001:001db050       ?GetForeignData@CPhysicalStub@@UBEPAXH@Z 351dc050 f i physarea.obj
 0001:001db050       ?GetTriMesh@CGeometry@@UAEPAUIGeometry@@H@Z 351dc050 f i livingentity.obj
 0001:001db050       ?CalcPhysicalProperties@CGeometry@@UAEHPAUphys_geometry@@@Z 351dc050 f i livingentity.obj
 0001:001db050       ?IsConvex@CVoxelGeom@@UAEHM@Z 351dc050 f i geoman.obj
 0001:001db050       ?QueryComposite@CEngineModule_CryPhysics@@MBEPAXPBD@Z 351dc050 f i CryPhysics.obj
 0001:001db050       ?Step@CPhysicalStub@@UAEHM@Z 351dc050 f i physarea.obj
 0001:001db050       ?get_deleter@?$sp_counted_impl_p@VCEngineModule_CryPhysics@@@detail@boost@@UAEPAXABVsp_typeinfo@23@@Z 351dc050 f i CryPhysics.obj
 0001:001db050       ?HasCollisionContactsWith@CPhysicalEntity@@UAEHPAV1@@Z 351dc050 f i livingentity.obj
 0001:001db050       ?IsAwake@CPhysicalEntity@@UBEHH@Z 351dc050 f i livingentity.obj
 0001:001db050       ?HasContactsWith@CPhysicalEntity@@UAEHPAV1@@Z 351dc050 f i livingentity.obj
 0001:001db060       ??$throw_exception@Vbad_alloc@std@@@boost@@YAXABVbad_alloc@std@@@Z 351dc060 f i CryPhysics.obj
 0001:001db090       ?dispose@?$sp_counted_impl_p@VCEngineModule_CryPhysics@@@detail@boost@@UAEXXZ 351dc090 f i CryPhysics.obj
 0001:001db0a0       ??_GCFactory@CEngineModule_CryPhysics@@UAEPAXI@Z 351dc0a0 f i CryPhysics.obj
 0001:001db0a0       ??_ECFactory@CEngineModule_CryPhysics@@UAEPAXI@Z 351dc0a0 f i CryPhysics.obj
 0001:001db0d0       ??$?0VCEngineModule_CryPhysics@@@shared_count@detail@boost@@QAE@PAVCEngineModule_CryPhysics@@@Z 351dc0d0 f i CryPhysics.obj
 0001:001db180       ??_Esp_counted_base@detail@boost@@UAEPAXI@Z 351dc180 f i CryPhysics.obj
 0001:001db180       ??_E?$sp_counted_impl_p@VCEngineModule_CryPhysics@@@detail@boost@@UAEPAXI@Z 351dc180 f i CryPhysics.obj
 0001:001db180       ??_G?$sp_counted_impl_p@VCEngineModule_CryPhysics@@@detail@boost@@UAEPAXI@Z 351dc180 f i CryPhysics.obj
 0001:001db180       ??_Gsp_counted_base@detail@boost@@UAEPAXI@Z 351dc180 f i CryPhysics.obj
 0001:001db1b0       ??_Ebad_alloc@std@@UAEPAXI@Z 351dc1b0 f i CryPhysics.obj
 0001:001db1b0       ??_Gbad_alloc@std@@UAEPAXI@Z 351dc1b0 f i CryPhysics.obj
 0001:001db1e0       ?QueryInterface@CEngineModule_CryPhysics@@MBEPAXABUCryGUID@@@Z 351dc1e0 f i CryPhysics.obj
 0001:001db240       ?CreateClassInstance@CFactory@CEngineModule_CryPhysics@@UBE?AV?$shared_ptr@UICryUnknown@@@boost@@XZ 351dc240 f i CryPhysics.obj
 0001:001db310       ?DeInitialize@?$Node_Alloc_Lock@$00$00@@SAXXZ 351dc310 f i StdAfx.obj
 0001:001db35a       __purecall                 351dc35a f   MSVCRT:MSVCR100.dll
 0001:001db360       __CIasin                   351dc360 f   MSVCRT:MSVCR100.dll
 0001:001db366       _memcpy                    351dc366 f   MSVCRT:MSVCR100.dll
 0001:001db370       __allshl                   351dc370 f   MSVCRT:llshl.obj
 0001:001db390       _memset                    351dc390 f   MSVCRT:MSVCR100.dll
 0001:001db396       __onexit                   351dc396 f   MSVCRT:atonexit.obj
 0001:001db437       _atexit                    351dc437 f   MSVCRT:atonexit.obj
 0001:001db450       __ftol2_sse                351dc450 f   MSVCRT:ftol2.obj
 0001:001db459       __ftol2_pentium4           351dc459 f   MSVCRT:ftol2.obj
 0001:001db46c       __ftol2_sse_excpt          351dc46c f   MSVCRT:ftol2.obj
 0001:001db486       __ftol2                    351dc486 f   MSVCRT:ftol2.obj
 0001:001db4fc       __CIacos                   351dc4fc f   MSVCRT:MSVCR100.dll
 0001:001db510       __allmul                   351dc510 f   MSVCRT:llmul.obj
 0001:001db550       __alloca_probe             351dc550     MSVCRT:chkstk.obj
 0001:001db550       __chkstk                   351dc550 f   MSVCRT:chkstk.obj
 0001:001db580       __aullshr                  351dc580 f   MSVCRT:ullshr.obj
 0001:001db5a0       __alldiv                   351dc5a0 f   MSVCRT:lldiv.obj
 0001:001db650       __alloca_probe_16          351dc650 f   MSVCRT:alloca16.obj
 0001:001db666       __alloca_probe_8           351dc666     MSVCRT:alloca16.obj
 0001:001db67c       ?what@exception@std@@UBEPBDXZ 351dc67c f   MSVCRT:MSVCR100.dll
 0001:001db6d0       __CRT_INIT@12              351dc6d0 f   MSVCRT:crtdll.obj
 0001:001db9f0       __DllMainCRTStartup@12     351dc9f0 f   MSVCRT:crtdll.obj
 0001:001dba14       __unlock                   351dca14 f   MSVCRT:MSVCR100.dll
 0001:001dba1a       ___dllonexit               351dca1a f   MSVCRT:MSVCR100.dll
 0001:001dba20       __lock                     351dca20 f   MSVCRT:MSVCR100.dll
 0001:001dba30       __SEH_prolog4              351dca30 f   MSVCRT:sehprolg4.obj
 0001:001dba75       __SEH_epilog4              351dca75 f   MSVCRT:sehprolg4.obj
 0001:001dba89       __except_handler4          351dca89 f   MSVCRT:chandler4gs.obj
 0001:001dbaae       ___sse2_available_init     351dcaae f   MSVCRT:cpu_disp.obj
 0001:001dbabe       ___clean_type_info_names   351dcabe f   MSVCRT:tncleanup.obj
 0001:001dbaca       __RTC_Initialize           351dcaca f   MSVCRT:_initsect_.obj
 0001:001dbaf0       __RTC_Terminate            351dcaf0 f   MSVCRT:_initsect_.obj
 0001:001dbb20       __ValidateImageBase        351dcb20 f   MSVCRT:pesect.obj
 0001:001dbb60       __FindPESection            351dcb60 f   MSVCRT:pesect.obj
 0001:001dbbb0       __IsNonwritableInCurrentImage 351dcbb0 f   MSVCRT:pesect.obj
 0001:001dbc6c       __initterm                 351dcc6c f   MSVCRT:MSVCR100.dll
 0001:001dbc72       __initterm_e               351dcc72 f   MSVCRT:MSVCR100.dll
 0001:001dbc78       __amsg_exit                351dcc78 f   MSVCRT:MSVCR100.dll
 0001:001dbc7e       ___CppXcptFilter           351dcc7e f   MSVCRT:MSVCR100.dll
 0001:001dbc84       _DllMain@12                351dcc84 f   MSVCRT:dllmain.obj
 0001:001dbca8       ___security_init_cookie    351dcca8 f   MSVCRT:gs_support.obj
 0001:001dbd43       @__security_check_cookie@4 351dcd43 f   MSVCRT:secchk.obj
 0001:001dbd52       __except_handler4_common   351dcd52 f   MSVCRT:MSVCR100.dll
 0001:001dbd58       ___clean_type_info_names_internal 351dcd58 f   MSVCRT:MSVCR100.dll
 0001:001dbd5e       ___report_gsfailure        351dcd5e f   MSVCRT:gs_report.obj
 0001:001dbe64       __crt_debugger_hook        351dce64 f   MSVCRT:MSVCR100.dll
 0001:001dc1c0       ??__Fs_dummyMemReplay@?1??CryGetIMemReplay@@YAPAUIMemReplay@@XZ@YAXXZ 351dd1c0 f i articulatedentity.obj
 0001:001dc1f0       ??__FserializeString@?1??SetSharedSerializeString@?$CSerializeWrapper@UISerialize@@@@QAEAAUSSerializeString@@ABV?$CryStringT@D@@@Z@YAXXZ 351dd1f0 f i physicalentity.obj
 0001:001dc3d0       ??__Fp@?1??CreateClassInstance@CFactory@CEngineModule_CryPhysics@@UBE?AV?$shared_ptr@UICryUnknown@@@boost@@XZ@YAXXZ 351dd3d0 f i CryPhysics.obj
 0002:00000000       __imp__QueryPerformanceCounter@4 351de000     kernel32:KERNEL32.dll
 0002:00000004       __imp__Sleep@4             351de004     kernel32:KERNEL32.dll
 0002:00000008       __imp__InterlockedCompareExchange@12 351de008     kernel32:KERNEL32.dll
 0002:0000000c       __imp__CreateEventA@16     351de00c     kernel32:KERNEL32.dll
 0002:00000010       __imp__CloseHandle@4       351de010     kernel32:KERNEL32.dll
 0002:00000014       __imp__SetEvent@4          351de014     kernel32:KERNEL32.dll
 0002:00000018       __imp__WaitForSingleObject@8 351de018     kernel32:KERNEL32.dll
 0002:0000001c       __imp__InitializeCriticalSection@4 351de01c     kernel32:KERNEL32.dll
 0002:00000020       __imp__DeleteCriticalSection@4 351de020     kernel32:KERNEL32.dll
 0002:00000024       __imp__EnterCriticalSection@4 351de024     kernel32:KERNEL32.dll
 0002:00000028       __imp__LeaveCriticalSection@4 351de028     kernel32:KERNEL32.dll
 0002:0000002c       __imp__GetCurrentThreadId@0 351de02c     kernel32:KERNEL32.dll
 0002:00000030       __imp__LoadLibraryA@4      351de030     kernel32:KERNEL32.dll
 0002:00000034       __imp__GetProcAddress@8    351de034     kernel32:KERNEL32.dll
 0002:00000038       __imp__GetModuleHandleA@4  351de038     kernel32:KERNEL32.dll
 0002:0000003c       __imp__IsDebuggerPresent@0 351de03c     kernel32:KERNEL32.dll
 0002:00000040       __imp__InterlockedIncrement@4 351de040     kernel32:KERNEL32.dll
 0002:00000044       __imp__InterlockedDecrement@4 351de044     kernel32:KERNEL32.dll
 0002:00000048       __imp__InterlockedExchangeAdd@8 351de048     kernel32:KERNEL32.dll
 0002:0000004c       __imp__UnhandledExceptionFilter@4 351de04c     kernel32:KERNEL32.dll
 0002:00000050       __imp__GetCurrentProcess@0 351de050     kernel32:KERNEL32.dll
 0002:00000054       __imp__TerminateProcess@8  351de054     kernel32:KERNEL32.dll
 0002:00000058       __imp__GetSystemTimeAsFileTime@4 351de058     kernel32:KERNEL32.dll
 0002:0000005c       __imp__GetCurrentProcessId@0 351de05c     kernel32:KERNEL32.dll
 0002:00000060       __imp__GetTickCount@0      351de060     kernel32:KERNEL32.dll
 0002:00000064       __imp__DisableThreadLibraryCalls@4 351de064     kernel32:KERNEL32.dll
 0002:00000068       __imp__IsProcessorFeaturePresent@4 351de068     kernel32:KERNEL32.dll
 0002:0000006c       __imp__InterlockedExchange@8 351de06c     kernel32:KERNEL32.dll
 0002:00000070       __imp__DecodePointer@4     351de070     kernel32:KERNEL32.dll
 0002:00000074       __imp__EncodePointer@4     351de074     kernel32:KERNEL32.dll
 0002:00000078       __imp__SetUnhandledExceptionFilter@4 351de078     kernel32:KERNEL32.dll
 0002:0000007c       \177KERNEL32_NULL_THUNK_DATA 351de07c     kernel32:KERNEL32.dll
 0002:00000080       __imp__strtoul             351de080     MSVCRT:MSVCR100.dll
 0002:00000084       __imp___set_invalid_parameter_handler 351de084     MSVCRT:MSVCR100.dll
 0002:00000088       __imp___set_purecall_handler 351de088     MSVCRT:MSVCR100.dll
 0002:0000008c       __imp__exit                351de08c     MSVCRT:MSVCR100.dll
 0002:00000090       __imp_??0exception@std@@QAE@ABQBDH@Z 351de090     MSVCRT:MSVCR100.dll
 0002:00000094       __imp_?what@exception@std@@UBEPBDXZ 351de094     MSVCRT:MSVCR100.dll
 0002:00000098       __imp_??1exception@std@@UAE@XZ 351de098     MSVCRT:MSVCR100.dll
 0002:0000009c       __imp___unlock             351de09c     MSVCRT:MSVCR100.dll
 0002:000000a0       __imp____dllonexit         351de0a0     MSVCRT:MSVCR100.dll
 0002:000000a4       __imp___lock               351de0a4     MSVCRT:MSVCR100.dll
 0002:000000a8       __imp___onexit             351de0a8     MSVCRT:MSVCR100.dll
 0002:000000ac       __imp__vsnprintf_s         351de0ac     MSVCRT:MSVCR100.dll
 0002:000000ac       __imp___vsnprintf_s        351de0ac     MSVCRT:MSVCR100.dll
 0002:000000b0       __imp__vsnprintf           351de0b0     MSVCRT:MSVCR100.dll
 0002:000000b0       __imp___vsnprintf          351de0b0     MSVCRT:MSVCR100.dll
 0002:000000b4       __imp___malloc_crt         351de0b4     MSVCRT:MSVCR100.dll
 0002:000000b8       __imp__free                351de0b8     MSVCRT:MSVCR100.dll
 0002:000000bc       __imp___encoded_null       351de0bc     MSVCRT:MSVCR100.dll
 0002:000000c0       __imp___initterm           351de0c0     MSVCRT:MSVCR100.dll
 0002:000000c4       __imp___initterm_e         351de0c4     MSVCRT:MSVCR100.dll
 0002:000000c8       __imp___amsg_exit          351de0c8     MSVCRT:MSVCR100.dll
 0002:000000cc       __imp____CppXcptFilter     351de0cc     MSVCRT:MSVCR100.dll
 0002:000000d0       __imp___except_handler4_common 351de0d0     MSVCRT:MSVCR100.dll
 0002:000000d4       __imp____clean_type_info_names_internal 351de0d4     MSVCRT:MSVCR100.dll
 0002:000000d8       __imp___crt_debugger_hook  351de0d8     MSVCRT:MSVCR100.dll
 0002:000000dc       __imp___isnan              351de0dc     MSVCRT:MSVCR100.dll
 0002:000000e0       __imp___CIacos             351de0e0     MSVCRT:MSVCR100.dll
 0002:000000e4       __imp__memmove             351de0e4     MSVCRT:MSVCR100.dll
 0002:000000e8       __imp___snprintf           351de0e8     MSVCRT:MSVCR100.dll
 0002:000000ec       __imp__memset              351de0ec     MSVCRT:MSVCR100.dll
 0002:000000f0       __imp__memcpy              351de0f0     MSVCRT:MSVCR100.dll
 0002:000000f4       __imp___CIasin             351de0f4     MSVCRT:MSVCR100.dll
 0002:000000f8       __imp___purecall           351de0f8     MSVCRT:MSVCR100.dll
 0002:000000fc       __imp___ltoa               351de0fc     MSVCRT:MSVCR100.dll
 0002:000000fc       __imp__ltoa                351de0fc     MSVCRT:MSVCR100.dll
 0002:00000100       __imp__sprintf             351de100     MSVCRT:MSVCR100.dll
 0002:00000104       \177MSVCR100_NULL_THUNK_DATA 351de104     MSVCRT:MSVCR100.dll
 0002:00000108       __imp__MessageBoxA@16      351de108     user32:USER32.dll
 0002:0000010c       \177USER32_NULL_THUNK_DATA 351de10c     user32:USER32.dll
 0002:00000110       ___xc_a                    351de110     MSVCRT:cinitexe.obj
 0002:00000150       ___xc_z                    351de150     MSVCRT:cinitexe.obj
 0002:00000154       ___xi_a                    351de154     MSVCRT:cinitexe.obj
 0002:00000160       ___xi_z                    351de160     MSVCRT:cinitexe.obj
 0002:00000198       ??_7IMemReplay@@6B@        351de198     articulatedentity.obj
 0002:00000230       __real@3f800000            351de230     articulatedentity.obj
 0002:00000234       __real@3f000000            351de234     articulatedentity.obj
 0002:00000238       __real@3fc00000            351de238     articulatedentity.obj
 0002:0000023c       __real@bf800000            351de23c     articulatedentity.obj
 0002:00000240       __real@7149f2ca            351de240     articulatedentity.obj
 0002:00000244       __real@00000000            351de244     articulatedentity.obj
 0002:00000250       __mask@@NegFloat@          351de250     articulatedentity.obj
 0002:00000260       __real@3c23d70a            351de260     articulatedentity.obj
 0002:00000264       __real@3fc90fdb            351de264     articulatedentity.obj
 0002:00000268       ??_7CDummyMemReplay@@6B@   351de268     articulatedentity.obj
 0002:00000300       __real@501502f9            351de300     articulatedentity.obj
 0002:00000304       __real@d01502f9            351de304     articulatedentity.obj
 0002:00000308       __real@3c6bedfa            351de308     articulatedentity.obj
 0002:0000030c       __real@3e4ccccd            351de30c     articulatedentity.obj
 0002:00000310       __real@3dcccccd            351de310     articulatedentity.obj
 0002:00000314       __real@3a23d70b            351de314     articulatedentity.obj
 0002:00000318       ??_7CArticulatedEntity@@6B@ 351de318     articulatedentity.obj
 0002:0000044c       __real@41200000            351de44c     articulatedentity.obj
 0002:00000450       __real@42c80000            351de450     articulatedentity.obj
 0002:00000454       __real@40000000            351de454     articulatedentity.obj
 0002:00000458       ??_C@_04OACGEDLG@qext?$AA@ 351de458     articulatedentity.obj
 0002:00000460       ??_C@_01IIACKFLH@q?$AA@    351de460     articulatedentity.obj
 0002:00000468       ??_C@_0EN@FCJJGCPA@?$CFs?3?5?$CI?$CF?450s?5?$EA?5?$CF?41f?0?$CF?41f?0?$CF?41f?$CJ?5Val@ 351de468     articulatedentity.obj
 0002:000004b8       ??_C@_02IKMLBCHJ@q0?$AA@   351de4b8     articulatedentity.obj
 0002:000004bc       ??_C@_0DN@ECLMILFI@?$CFs?3?5?$CI?$CF?450s?5?$EA?5?$CF?41f?0?$CF?41f?0?$CF?41f?$CJ?5Val@ 351de4bc     articulatedentity.obj
 0002:000004fc       ??_C@_05JHLBIJAO@pivot?$AA@ 351de4fc     articulatedentity.obj
 0002:00000502       ??_C@_00CNPNBAHC@?$AA@     351de502     articulatedentity.obj
 0002:00000504       __real@1e3ce508            351de504     articulatedentity.obj
 0002:00000508       ??_C@_05HKIHAKL@ipart?$AA@ 351de508     articulatedentity.obj
 0002:00000510       ??_C@_05BBEJFBFA@point?$AA@ 351de510     articulatedentity.obj
 0002:00000518       __real@5368d4a5            351de518     articulatedentity.obj
 0002:0000051c       ??_C@_0L@CLGAEIII@angImpulse?$AA@ 351de51c     articulatedentity.obj
 0002:00000528       __real@5a0e1bca            351de528     articulatedentity.obj
 0002:00000530       ??_C@_0EN@KMHCOBOM@?$CFs?3?5?$CI?$CF?450s?5?$EA?5?$CF?41f?0?$CF?41f?0?$CF?41f?$CJ?5Val@ 351de530     articulatedentity.obj
 0002:00000580       ??_C@_07LKMFNFAN@impulse?$AA@ 351de580     articulatedentity.obj
 0002:00000588       __real@6753c21c            351de588     articulatedentity.obj
 0002:0000058c       __real@51ba43b7            351de58c     articulatedentity.obj
 0002:00000590       __real@3c8efa35            351de590     articulatedentity.obj
 0002:00000594       __real@358637bd            351de594     articulatedentity.obj
 0002:00000598       __real@3e45798ee2308c3a    351de598     articulatedentity.obj
 0002:000005a0       __real@c00921fb54442d18    351de5a0     articulatedentity.obj
 0002:000005a8       __real@401921fb54442d18    351de5a8     articulatedentity.obj
 0002:000005b0       __real@41700000            351de5b0     articulatedentity.obj
 0002:000005b8       __real@3eb0c6f7a0b5ed8d    351de5b8     articulatedentity.obj
 0002:000005c0       ??_C@_09GMEIBLE@offsPivot?$AA@ 351de5c0     articulatedentity.obj
 0002:000005cc       ??_C@_09OMNEEBCL@numjoints?$AA@ 351de5cc     articulatedentity.obj
 0002:000005d8       ??_C@_05LAFFIJJO@quat0?$AA@ 351de5d8     articulatedentity.obj
 0002:000005e0       ??_C@_09MBCEGBCG@q0changed?$AA@ 351de5e0     articulatedentity.obj
 0002:000005ec       ??_C@_02HJEEANKG@dq?$AA@   351de5ec     articulatedentity.obj
 0002:000005f0       ??_C@_05LDAEHAKN@joint?$AA@ 351de5f0     articulatedentity.obj
 0002:000005f8       ??_C@_03BHLLPCMD@vel?$AA@  351de5f8     articulatedentity.obj
 0002:000005fc       ??_C@_03PCBNCGFH@pos?$AA@  351de5fc     articulatedentity.obj
 0002:00000600       ??_C@_05BJPFJFDJ@awake?$AA@ 351de600     articulatedentity.obj
 0002:00000608       __real@40800000            351de608     articulatedentity.obj
 0002:0000060c       __real@41c80000            351de60c     articulatedentity.obj
 0002:00000610       __real@40a00000            351de610     articulatedentity.obj
 0002:00000614       __real@40c00000            351de614     articulatedentity.obj
 0002:00000618       __real@3716feb5            351de618     articulatedentity.obj
 0002:00000620       ??_C@_0FD@NAFJCAP@CArticulatedEntity?3?3AddGeometry?3@ 351de620     articulatedentity.obj
 0002:00000674       __real@2edbe6ff            351de674     articulatedentity.obj
 0002:00000678       __real@447a0000            351de678     articulatedentity.obj
 0002:0000067c       __real@49742400            351de67c     articulatedentity.obj
 0002:00000680       __real@40400000            351de680     articulatedentity.obj
 0002:00000684       ??_C@_0CK@MJPDAFHG@CArticulatedEntity?3Action?$CIaction@ 351de684     articulatedentity.obj
 0002:000006b0       __real@3d23d70a            351de6b0     articulatedentity.obj
 0002:000006b4       __real@3f7d70a4            351de6b4     articulatedentity.obj
 0002:000006b8       __real@3e860a92            351de6b8     articulatedentity.obj
 0002:000006bc       __real@3f7f7cff            351de6bc     articulatedentity.obj
 0002:000006c0       __real@be800000            351de6c0     articulatedentity.obj
 0002:000006c4       __real@3e800000            351de6c4     articulatedentity.obj
 0002:000006c8       __real@bf000000            351de6c8     articulatedentity.obj
 0002:000006cc       __real@3d8efa35            351de6cc     articulatedentity.obj
 0002:000006d0       __real@3fcccccd            351de6d0     articulatedentity.obj
 0002:000006d4       __real@3f99999a            351de6d4     articulatedentity.obj
 0002:000006d8       __real@3727c5ac            351de6d8     articulatedentity.obj
 0002:000006dc       __real@3a83126f            351de6dc     articulatedentity.obj
 0002:000006e0       __real@38d1b717            351de6e0     articulatedentity.obj
 0002:000006e4       __real@322bcc77            351de6e4     articulatedentity.obj
 0002:000006e8       __real@3f666666            351de6e8     articulatedentity.obj
 0002:000006ec       __real@3d8f5c29            351de6ec     articulatedentity.obj
 0002:000006f0       __real@40200000            351de6f0     articulatedentity.obj
 0002:000006f8       __real@3fc45f306dc9c883    351de6f8     articulatedentity.obj
 0002:00000700       __real@3f4f5c28            351de700     articulatedentity.obj
 0002:00000704       __real@3e99999a            351de704     articulatedentity.obj
 0002:00000708       ??_C@_0BJ@NDOEJGHE@CArticulatedEntity?3?3Step?$AA@ 351de708     articulatedentity.obj
 0002:00000724       __real@58635fa9            351de724     articulatedentity.obj
 0002:00000728       __real@d8635fa9            351de728     articulatedentity.obj
 0002:0000072c       ??_C@_0CL@ECFNLKDN@CArticulatedEntity?3SetParams?$CIpar@ 351de72c     articulatedentity.obj
 0002:00000758       __real@40490fdb            351de758     articulatedentity.obj
 0002:0000075c       __real@40c90fdb            351de75c     articulatedentity.obj
 0002:00000770       ??_7CBVTree@@6B@           351de770     livingentity.obj
 0002:000007e0       ??_7IGeometry@@6B@         351de7e0     livingentity.obj
 0002:000008a0       ??_7CRayBV@@6B@            351de8a0     livingentity.obj
 0002:00000910       ??_7CLivingEntity@@6B@     351de910     livingentity.obj
 0002:00000a30       __real@404ca5dc1a63c1f8    351dea30     livingentity.obj
 0002:00000a38       ??_7CGeometry@@6B@         351dea38     livingentity.obj
 0002:00000b30       __real@43a3d5c3            351deb30     livingentity.obj
 0002:00000b34       __real@c2c80000            351deb34     livingentity.obj
 0002:00000b38       __real@3b480190            351deb38     livingentity.obj
 0002:00000b3c       __real@414c0000            351deb3c     livingentity.obj
 0002:00000b40       __real@41a00000            351deb40     livingentity.obj
 0002:00000b48       __real@404436720cee34f2    351deb48     livingentity.obj
 0002:00000b50       __real@40c45f07af68ecef    351deb50     livingentity.obj
 0002:00000b58       __real@36800000            351deb58     livingentity.obj
 0002:00000b60       __real@3f9954a49d7f2b6f    351deb60     livingentity.obj
 0002:00000b68       __real@3da0a0a1            351deb68     livingentity.obj
 0002:00000b70       __real@3f19222d989f5e57    351deb70     livingentity.obj
 0002:00000b78       ??_C@_0N@DIIBGNIK@velRequested?$AA@ 351deb78     livingentity.obj
 0002:00000b88       __real@c0800000            351deb88     livingentity.obj
 0002:00000b8c       ??_C@_0N@MHIKDJFP@sizeCollider?$AA@ 351deb8c     livingentity.obj
 0002:00000b9c       __real@461c4000            351deb9c     livingentity.obj
 0002:00000ba0       ??_C@_09EOJBHBBH@heightEye?$AA@ 351deba0     livingentity.obj
 0002:00000bac       ??_C@_0M@FLAOEHJJ@heightPivot?$AA@ 351debac     livingentity.obj
 0002:00000bb8       ??_C@_02EDDPJOD@dt?$AA@    351debb8     livingentity.obj
 0002:00000bbc       ??_C@_03DAPAKLGM@dir?$AA@  351debbc     livingentity.obj
 0002:00000bc0       ??_7CSingleBoxTree@@6B@    351debc0     livingentity.obj
 0002:00000c30       ??_7CCylinderGeom@@6B@     351dec30     livingentity.obj
 0002:00000d28       ??_7CCapsuleGeom@@6B@      351ded28     livingentity.obj
 0002:00000e20       __real@4010c152382d7365    351dee20     livingentity.obj
 0002:00000e28       ??_7CRayGeom@@6B@          351dee28     livingentity.obj
 0002:00000f20       __real@3e23d70a            351def20     livingentity.obj
 0002:00000f24       __real@41000000            351def24     livingentity.obj
 0002:00000f28       __real@3fb999999999999a    351def28     livingentity.obj
 0002:00000f30       __real@3b83126f            351def30     livingentity.obj
 0002:00000f34       __real@3fd9999a            351def34     livingentity.obj
 0002:00000f38       __real@3f8ccccd            351def38     livingentity.obj
 0002:00000f3c       __real@3f19999a            351def3c     livingentity.obj
 0002:00000f40       __real@3ff39a816dfbe7fa    351def40     livingentity.obj
 0002:00000f48       __real@3fee28c7460698c7    351def48     livingentity.obj
 0002:00000f50       __real@3ecccccd            351def50     livingentity.obj
 0002:00000f54       __real@42700000            351def54     livingentity.obj
 0002:00000f58       __real@3ccccccd            351def58     livingentity.obj
 0002:00000f5c       __real@42a00000            351def5c     livingentity.obj
 0002:00000f60       __real@aedbe6ff            351def60     livingentity.obj
 0002:00000f68       __real@3fe41b2f7ba3bcbe    351def68     livingentity.obj
 0002:00000f70       __real@c11cf5c3            351def70     livingentity.obj
 0002:00000f78       __real@3f91df46a2529d39    351def78     livingentity.obj
 0002:00000f80       ??_C@_0CL@HEHKAFBI@CLivingEntity?3SetParams?$CIplayer_d@ 351def80     livingentity.obj
 0002:00000fb0       __real@3f847ae147ae147b    351defb0     livingentity.obj
 0002:00000fb8       __real@3f8147ae            351defb8     livingentity.obj
 0002:00000fbc       __real@3b23d70b            351defbc     livingentity.obj
 0002:00000fc0       __real@40555555            351defc0     livingentity.obj
 0002:00000fc4       ??_C@_0CF@GMDAKOKI@CLivingEntity?3Action?$CIaction_impu@ 351defc4     livingentity.obj
 0002:00000fec       ??_C@_0CC@ELHODBNL@CLivingEntity?3Action?$CIaction_move@ 351defec     livingentity.obj
 0002:00001010       __real@45cccccd            351df010     livingentity.obj
 0002:00001014       __real@42480000            351df014     livingentity.obj
 0002:00001018       __real@3f866666            351df018     livingentity.obj
 0002:0000101c       __real@4f800000            351df01c     livingentity.obj
 0002:00001020       __real@3f333333            351df020     livingentity.obj
 0002:00001028       __real@3ff0000000000000    351df028     livingentity.obj
 0002:00001030       __real@4000000000000000    351df030     livingentity.obj
 0002:00001038       __real@3f7746ea            351df038     livingentity.obj
 0002:0000103c       __real@3e8483ee            351df03c     livingentity.obj
 0002:00001040       __real@3fb33333            351df040     livingentity.obj
 0002:00001048       __real@3fd0000000000000    351df048     livingentity.obj
 0002:00001050       __real@bfc00000            351df050     livingentity.obj
 0002:00001054       __real@3db22d0e            351df054     livingentity.obj
 0002:00001058       __real@3e23d70b            351df058     livingentity.obj
 0002:0000105c       __real@3f7ff2e5            351df05c     livingentity.obj
 0002:00001060       __real@3ca3d70a            351df060     livingentity.obj
 0002:00001064       __real@bf8147ae            351df064     livingentity.obj
 0002:00001068       __real@c000000000000000    351df068     livingentity.obj
 0002:00001070       __real@c0000000            351df070     livingentity.obj
 0002:00001074       __real@3f733333            351df074     livingentity.obj
 0002:00001078       __real@3fee666674000000    351df078     livingentity.obj
 0002:00001080       __real@3f400000            351df080     livingentity.obj
 0002:00001088       __real@3fd3333340000000    351df088     livingentity.obj
 0002:00001090       __real@358637be            351df090     livingentity.obj
 0002:00001094       ??_C@_0BE@PGDCIADM@CLivingEntity?3?3Step?$AA@ 351df094     livingentity.obj
 0002:000010a8       __real@00800000            351df0a8     particleentity.obj
 0002:000010b0       ??_7CParticleEntity@@6B@   351df0b0     particleentity.obj
 0002:000011cc       __real@3f4ccccd            351df1cc     particleentity.obj
 0002:000011d0       __real@3d4ccccd            351df1d0     particleentity.obj
 0002:000011d4       __real@c47a0000            351df1d4     particleentity.obj
 0002:000011d8       ??_C@_06IKLLLDHL@normal?$AA@ 351df1d8     particleentity.obj
 0002:000011e0       ??_C@_07MBJMFGGL@heading?$AA@ 351df1e0     particleentity.obj
 0002:000011e8       ??_C@_09GLPKLBIH@thickness?$AA@ 351df1e8     particleentity.obj
 0002:000011f4       ??_C@_04IAGNFIBA@size?$AA@ 351df1f4     particleentity.obj
 0002:000011fc       ??_C@_04IJEANHEE@mass?$AA@ 351df1fc     particleentity.obj
 0002:00001204       ??_C@_0P@LKCCAGNB@ParticleEntity?$AA@ 351df204     particleentity.obj
 0002:00001214       ??_C@_07OKNHCJLM@ifawake?$AA@ 351df214     particleentity.obj
 0002:0000121c       ??_C@_0CO@DMIGAK@CParticleEntity?3SetParams?$CIpe_par@ 351df21c     particleentity.obj
 0002:0000124c       __real@43c80000            351df24c     particleentity.obj
 0002:00001250       __real@3d888889            351df250     particleentity.obj
 0002:00001254       __real@3f7851ec            351df254     particleentity.obj
 0002:00001258       __real@3c23d70b            351df258     particleentity.obj
 0002:0000125c       __real@42200000            351df25c     particleentity.obj
 0002:00001260       __real@3f1a36e2eb1c432d    351df260     particleentity.obj
 0002:00001268       ??_C@_0CE@EPNDKOAE@RayWorldIntersection?$CIPhysParticl@ 351df268     particleentity.obj
 0002:0000128c       __real@bf8ccccd            351df28c     particleentity.obj
 0002:00001290       ??_C@_0BI@KOOFBDI@CParticleEntity?3?3DoStep?$AA@ 351df290     particleentity.obj
 0002:000012c0       ??_7IPhysicalEntity@@6B@   351df2c0     physarea.obj
 0002:0000132c       __real@2f800000            351df32c     physarea.obj
 0002:00001330       __real@ff7843b0            351df330     physarea.obj
 0002:00001334       __real@7f7843b0            351df334     physarea.obj
 0002:00001338       __real@3fe0000000000000    351df338     physarea.obj
 0002:00001340       __real@0000000000000000    351df340     physarea.obj
 0002:00001348       __real@3fd5555555555555    351df348     physarea.obj
 0002:00001350       __real@3bc79ca10c924223    351df350     physarea.obj
 0002:00001358       __real@3ddb7cdfd9d7bdbb    351df358     physarea.obj
 0002:00001360       ??_7CPhysicalPlaceholder@@6B@ 351df360     physarea.obj
 0002:000013d8       ??_7CPhysicalStub@@6B@     351df3d8     physarea.obj
 0002:00001450       ??_7CPhysArea@@6B@         351df450     physarea.obj
 0002:000014d8       __real@4008000000000000    351df4d8     physarea.obj
 0002:000014e0       __real@bfd0000000000000    351df4e0     physarea.obj
 0002:000014e8       __real@4020000000000000    351df4e8     physarea.obj
 0002:000014f0       __real@3fe8000000000000    351df4f0     physarea.obj
 0002:000014f8       __real@3e112e0be826d695    351df4f8     physarea.obj
 0002:00001500       __real@be112e0be826d695    351df500     physarea.obj
 0002:00001508       __real@c415af1d78b58c40    351df508     physarea.obj
 0002:00001510       __real@4415af1d78b58c40    351df510     physarea.obj
 0002:00001518       __real@3fc5555555555555    351df518     physarea.obj
 0002:00001520       __real@4010000000000000    351df520     physarea.obj
 0002:00001528       __real@4cbebc20            351df528     physarea.obj
 0002:0000152c       __real@3ffeb852            351df52c     physarea.obj
 0002:00001540       ??_7CPhysicalEntity@@6B@   351df540     physicalentity.obj
 0002:0000165c       ??_C@_05MHMEBBGO@scale?$AA@ 351df65c     physicalentity.obj
 0002:00001664       ??_C@_0BF@LALMAGNL@?5pos?3?5?$CF?41f?0?$CF?41f?0?$CF?41f?$AA@ 351df664     physicalentity.obj
 0002:00001680       ??_C@_0FA@PBHKFAEH@?$CFs?3?5?$CI?$CF?450s?5?$EA?5?$CF?41f?0?$CF?41f?0?$CF?41f?$CJ?5Val@ 351df680     physicalentity.obj
 0002:000016d0       ??_C@_0CI@IOBNLHFK@?$CIperhaps?5non?9uniform?5scaling?5was@ 351df6d0     physicalentity.obj
 0002:000016f8       ??_C@_07CEEBLDMK@BBox?$FL1?$FN?$AA@ 351df6f8     physicalentity.obj
 0002:00001700       ??_C@_07CFIDNJPN@BBox?$FL0?$FN?$AA@ 351df700     physicalentity.obj
 0002:00001708       ??_C@_0BE@NGINBJG@?5pt?3?5?$CF?41f?0?$CF?41f?0?$CF?41f?$AA@ 351df708     physicalentity.obj
 0002:0000171c       ??_C@_0DF@BCOOIFOK@?$CIperhaps?5non?9uniform?5scaling?5was@ 351df71c     physicalentity.obj
 0002:00001754       ??_C@_07HAFFKDBK@density?$AA@ 351df754     physicalentity.obj
 0002:0000175c       __real@ccbebc20            351df75c     physicalentity.obj
 0002:00001760       __real@e0ad78ec            351df760     physicalentity.obj
 0002:00001764       __real@60ad78ec            351df764     physicalentity.obj
 0002:00001768       __real@bf7ff972            351df768     physicalentity.obj
 0002:00001770       ??_7CBoxGeom@@6B@          351df770     physicalentity.obj
 0002:00001868       ??_7CSphereGeom@@6B@       351df868     physicalentity.obj
 0002:00001960       __real@3cf5c28f            351df960     physicalentity.obj
 0002:00001964       ??_C@_0BM@NPMINFME@CPhysicalEntity?3AddGeometry?$AA@ 351df964     physicalentity.obj
 0002:00001980       __real@41100000            351df980     physicalentity.obj
 0002:00001984       ??_C@_04GGBPDDBN@?$CF?41f?$AA@ 351df984     physicalentity.obj
 0002:0000198c       ??_C@_09PHALKAAM@?$CF?41f?1?$CF?41f?$AA@ 351df98c     physicalentity.obj
 0002:00001998       ??_C@_0BB@OCIOGPEL@shift?3?5?$CF?41f?1?$CF?41f?$AA@ 351df998     physicalentity.obj
 0002:000019ac       ??_C@_0BA@FIGEHIAC@pull?3?5?$CF?41f?1?$CF?41f?$AA@ 351df9ac     physicalentity.obj
 0002:000019bc       ??_C@_0BA@KIPLJKAO@push?3?5?$CF?41f?1?$CF?41f?$AA@ 351df9bc     physicalentity.obj
 0002:000019cc       ??_C@_0BA@MGOMOLHA@bend?3?5?$CF?41f?1?$CF?41f?$AA@ 351df9cc     physicalentity.obj
 0002:000019dc       ??_C@_0BB@EIMABIKF@twist?3?5?$CF?41f?1?$CF?41f?$AA@ 351df9dc     physicalentity.obj
 0002:000019f0       __real@bdcccccd            351df9f0     physicalentity.obj
 0002:000019f4       __real@be315b57            351df9f4     physicalentity.obj
 0002:000019f8       __real@3e315b57            351df9f8     physicalentity.obj
 0002:000019fc       ??_C@_06GJCCMIGE@?$CF?42fkg?$AA@ 351df9fc     physicalentity.obj
 0002:00001a04       __real@43480000            351dfa04     physicalentity.obj
 0002:00001a08       __real@43fa0000            351dfa08     physicalentity.obj
 0002:00001a0c       __real@3ba3d70a            351dfa0c     physicalentity.obj
 0002:00001a10       __real@3b03126f            351dfa10     physicalentity.obj
 0002:00001a14       __real@be428f5f            351dfa14     physicalentity.obj
 0002:00001a18       ??_C@_0BJ@KINLGGMJ@Lattice?5tension?3?5?$CFf?5?$CI?$CFs?$CJ?$AA@ 351dfa18     physicalentity.obj
 0002:00001a34       ??_C@_05MOLGPPCG@twist?$AA@ 351dfa34     physicalentity.obj
 0002:00001a3c       ??_C@_04JFAPGDHH@bend?$AA@ 351dfa3c     physicalentity.obj
 0002:00001a44       ??_C@_05CLOOKOFG@shift?$AA@ 351dfa44     physicalentity.obj
 0002:00001a4c       ??_C@_04BEGLKOGM@pull?$AA@ 351dfa4c     physicalentity.obj
 0002:00001a54       ??_C@_04GHHNIPCF@push?$AA@ 351dfa54     physicalentity.obj
 0002:00001a5c       __real@48435000            351dfa5c     physicalentity.obj
 0002:00001a60       __real@48c35000            351dfa60     physicalentity.obj
 0002:00001a64       __real@47c35000            351dfa64     physicalentity.obj
 0002:00001a68       ??_C@_0CK@CECADMJN@CPhysicalEntity?3SetParams?$CIpe_par@ 351dfa68     physicalentity.obj
 0002:00001a94       ??_C@_0CL@MNMOENND@CPhysicalEntity?3?3SetParams?$CIpe_pa@ 351dfa94     physicalentity.obj
 0002:00001ac0       ??_C@_0CJ@DICFJNIC@CPhysicalEntity?3SetParams?$CIpe_par@ 351dfac0     physicalentity.obj
 0002:00001aec       ??_C@_06CPGPAJPB@hasDfm?$AA@ 351dfaec     physicalentity.obj
 0002:00001af4       ??_C@_09BMMJDEMI@usedParts?$AA@ 351dfaf4     physicalentity.obj
 0002:00001b00       ??_C@_0O@NOMKKJCH@dampingConstr?$AA@ 351dfb00     physicalentity.obj
 0002:00001b10       ??_C@_0M@ODBAFIDM@limitConstr?$AA@ 351dfb10     physicalentity.obj
 0002:00001b1c       ??_C@_05LDEILEND@axisx?$AA@ 351dfb1c     physicalentity.obj
 0002:00001b24       ??_C@_08KGHNBEIB@szHelper?$AA@ 351dfb24     physicalentity.obj
 0002:00001b30       ??_C@_0L@GDBJIHOA@bBreakable?$AA@ 351dfb30     physicalentity.obj
 0002:00001b3c       ??_C@_0P@DEBFNDAF@maxTorqueTwist?$AA@ 351dfb3c     physicalentity.obj
 0002:00001b4c       ??_C@_0O@DJBOCDGJ@maxTorqueBend?$AA@ 351dfb4c     physicalentity.obj
 0002:00001b5c       ??_C@_0O@MBJBNLLP@maxForceShift?$AA@ 351dfb5c     physicalentity.obj
 0002:00001b6c       ??_C@_0N@LOFJHOOI@maxForcePull?$AA@ 351dfb6c     physicalentity.obj
 0002:00001b7c       ??_C@_0N@MNEPFPKB@maxForcePush?$AA@ 351dfb7c     physicalentity.obj
 0002:00001b8c       ??_C@_01EFFIKLCJ@n?$AA@    351dfb8c     physicalentity.obj
 0002:00001b90       ??_C@_02BPBMPCEP@pt?$AA@   351dfb90     physicalentity.obj
 0002:00001b94       ??_C@_06IHFONFKC@ipart1?$AA@ 351dfb94     physicalentity.obj
 0002:00001b9c       ??_C@_06JOEFOEOD@ipart0?$AA@ 351dfb9c     physicalentity.obj
 0002:00001ba4       ??_C@_02EGCJHIOB@id?$AA@   351dfba4     physicalentity.obj
 0002:00001ba8       ??_C@_07FOFEHKBC@nJoints?$AA@ 351dfba8     physicalentity.obj
 0002:00001bb0       ??_C@_09LGGKDIJE@hasJoints?$AA@ 351dfbb0     physicalentity.obj
 0002:00001bd0       ??_7IGeomManager@@6B@      351dfbd0     physicalworld.obj
 0002:00001c2c       ??_7IThreadTask@@6B@       351dfc2c     physicalworld.obj
 0002:00001c3c       ??_7SThreadTaskInfo@@6B@   351dfc3c     physicalworld.obj
 0002:00001c3c       ??_7CMultiThreadRefCount@@6B@ 351dfc3c     physicalworld.obj
 0002:00001c40       ??_7IPhysicalWorld@@6B@    351dfc40     physicalworld.obj
 0002:00001da8       __real@3fe5555555555555    351dfda8     physicalworld.obj
 0002:00001db0       __real@3ef0001000100010    351dfdb0     physicalworld.obj
 0002:00001db8       __real@477fff00            351dfdb8     physicalworld.obj
 0002:00001dc0       ??_C@_0EI@EOAKOGBE@Error?3?5?$CKmajor?$CK?5problem?5?9?5trying?5@ 351dfdc0     physicalworld.obj
 0002:00001e08       ??_C@_06LNKFDEGN@noname?$AA@ 351dfe08     physicalworld.obj
 0002:00001e10       __real@38000000            351dfe10     physicalworld.obj
 0002:00001e18       ??_7CGeomManager@@6B@      351dfe18     physicalworld.obj
 0002:00001e78       ??_7SPhysTask@@6B@         351dfe78     physicalworld.obj
 0002:00001e88       ??_7CPhysicalEntityIt@CPhysicalWorld@@6B@ 351dfe88     physicalworld.obj
 0002:00001ea4       __real@41800000            351dfea4     physicalworld.obj
 0002:00001ea8       __real@3d800000            351dfea8     physicalworld.obj
 0002:00001eac       __real@37d1b717            351dfeac     physicalworld.obj
 0002:00001eb0       ??_C@_08KIKMFGJF@Physics0?$AA@ 351dfeb0     physicalworld.obj
 0002:00001ebc       ??_C@_08LBLHGHNE@Physics1?$AA@ 351dfebc     physicalworld.obj
 0002:00001ec8       ??_C@_08JKJKDEBH@Physics2?$AA@ 351dfec8     physicalworld.obj
 0002:00001ed4       ??_C@_08IDIBAFFG@Physics3?$AA@ 351dfed4     physicalworld.obj
 0002:00001ee0       ??_C@_0BE@EHHKEKKG@?$CFd?5active?5object?$CIs?$CJ?$AA@ 351dfee0     physicalworld.obj
 0002:00001ef8       ??_C@_0EF@JNHCCPCP@?$CFs?5?$EA?5?$CF7?42f?0?$CF7?42f?0?$CF7?42f?0?5mass?5?$CF?42@ 351dfef8     physicalworld.obj
 0002:00001f40       __real@42f00000            351dff40     physicalworld.obj
 0002:00001f4c       ??_C@_0BE@LFJFAKMB@Static?5TriMesh?5Data?$AA@ 351dff4c     physicalworld.obj
 0002:00001f60       ??_C@_0BE@OKHLKODM@external?5geometries?$AA@ 351dff60     physicalworld.obj
 0002:00001f74       ??_C@_0L@NEGCPNMO@geometries?$AA@ 351dff74     physicalworld.obj
 0002:00001f80       ??_C@_05EPHILNBP@areas?$AA@ 351dff80     physicalworld.obj
 0002:00001f88       ??_C@_0BA@CPFEOAFC@hidden?5entities?$AA@ 351dff88     physicalworld.obj
 0002:00001f98       ??_C@_08PNMNOKOB@entities?$AA@ 351dff98     physicalworld.obj
 0002:00001fa4       ??_C@_0N@OILCNOIE@placeholders?$AA@ 351dffa4     physicalworld.obj
 0002:00001fb4       ??_C@_0N@KOGLEBGK@world?5queues?$AA@ 351dffb4     physicalworld.obj
 0002:00001fc4       ??_C@_0BB@CJHEBAIA@world?5structures?$AA@ 351dffc4     physicalworld.obj
 0002:00001fd8       ??_C@_0BE@KJDJFMJA@STL?5Allocator?5Waste?$AA@ 351dffd8     physicalworld.obj
 0002:00001fec       ??_C@_0BA@NFPONAAD@static?5entities?$AA@ 351dffec     physicalworld.obj
 0002:00001ffc       ??_C@_0BC@CKIFBHJ@physical?5entities?$AA@ 351dfffc     physicalworld.obj
 0002:00002010       ??_C@_0BA@DBEKKOOB@living?5entities?$AA@ 351e0010     physicalworld.obj
 0002:00002020       ??_C@_0BC@FMIIKKPA@detached?5entities?$AA@ 351e0020     physicalworld.obj
 0002:00002034       ??_C@_08CFJOODNG@triggers?$AA@ 351e0034     physicalworld.obj
 0002:00002040       ??_C@_0BB@PLIHMJIB@deleted?5entities?$AA@ 351e0040     physicalworld.obj
 0002:00002054       ??_C@_0CG@LGHEGFDG@Error?3?5queued?5RWI?5hits?5pool?5corr@ 351e0054     physicalworld.obj
 0002:0000207c       ??_C@_0BI@BBMELPMJ@PhysEventHandler?$CI?$CFd?0?$CFd?$CJ?$AA@ 351e007c     physicalworld.obj
 0002:00002094       ??_C@_0CB@IEBMEMCB@CPhysicalWorld?3?3PumpLoggedEvents@ 351e0094     physicalworld.obj
 0002:000020b8       ??_C@_0BB@EBHBFJFK@rb_primintersect?$AA@ 351e00b8     physicalworld.obj
 0002:000020cc       ??_C@_0N@DMLBCAGA@featherstone?$AA@ 351e00cc     physicalworld.obj
 0002:000020dc       ??_C@_0N@MGKFCACL@rope?5?5?5?5?5?5?5?5?$AA@ 351e00dc     physicalworld.obj
 0002:000020ec       ??_C@_0N@EIICPGEA@cloth?5?5?5?5?5?5?5?$AA@ 351e00ec     physicalworld.obj
 0002:000020fc       ??_C@_0N@PAEACHLK@solver?5?5?5?5?5?5?$AA@ 351e00fc     physicalworld.obj
 0002:0000210c       ??_C@_0BB@GEEHMKJE@rb_geomintersect?$AA@ 351e010c     physicalworld.obj
 0002:00002120       ??_C@_0BB@DHBNBKPP@World?5step?5total?$AA@ 351e0120     physicalworld.obj
 0002:00002134       ??_C@_0BA@NILGEFEO@Queued?5requests?$AA@ 351e0134     physicalworld.obj
 0002:00002144       ??_C@_0P@COOONLDP@Entities?5total?$AA@ 351e0144     physicalworld.obj
 0002:00002154       ??_C@_0BC@GKAHDKOK@Kinematic?5objects?$AA@ 351e0154     physicalworld.obj
 0002:00002168       ??_C@_0BE@LMPPICDB@Character?5skeletons?$AA@ 351e0168     physicalworld.obj
 0002:0000217c       ??_C@_0BC@DHLIMEHH@Ropes?5?$CIcharacter?$CJ?$AA@ 351e017c     physicalworld.obj
 0002:00002190       ??_C@_0BD@KBBCJMME@Ropes?5?$CIvegetation?$CJ?$AA@ 351e0190     physicalworld.obj
 0002:000021a4       ??_C@_05GKKHKKE@Cloth?$AA@ 351e01a4     physicalworld.obj
 0002:000021ac       ??_C@_0BD@HBBFNCLM@Ropes?5?$CIstandalone?$CJ?$AA@ 351e01ac     physicalworld.obj
 0002:000021c0       ??_C@_08KLCKKNPF@Ragdolls?$AA@ 351e01c0     physicalworld.obj
 0002:000021cc       ??_C@_0BH@GBMNCFJC@Physicalized?5particles?$AA@ 351e01cc     physicalworld.obj
 0002:000021e4       ??_C@_06DCPPBEOJ@Actors?$AA@ 351e01e4     physicalworld.obj
 0002:000021ec       ??_C@_0BB@INJEDGPL@Wheeled?5vehicles?$AA@ 351e01ec     physicalworld.obj
 0002:00002200       ??_C@_0N@FFLNJJI@Rigid?5bodies?$AA@ 351e0200     physicalworld.obj
 0002:00002210       __real@48127c00            351e0210     physicalworld.obj
 0002:00002214       __real@41f00000            351e0214     physicalworld.obj
 0002:00002218       __real@40900000            351e0218     physicalworld.obj
 0002:0000221c       __real@466a6000            351e021c     physicalworld.obj
 0002:00002220       __real@40e00000            351e0220     physicalworld.obj
 0002:00002224       __real@43160000            351e0224     physicalworld.obj
 0002:00002228       __real@c11ccccd            351e0228     physicalworld.obj
 0002:00002230       ??_7CPhysicalWorld@@6BCGeomManager@@@ 351e0230     physicalworld.obj
 0002:00002290       ??_7CPhysicalWorld@@6BIPhysUtils@@@ 351e0290     physicalworld.obj
 0002:000022a0       ??_7CPhysicalWorld@@6BIPhysicalWorld@@@ 351e02a0     physicalworld.obj
 0002:00002410       __real@3b800000            351e0410     physicalworld.obj
 0002:00002418       ??_C@_0FJ@OGBDLIAD@GetEntitiesInBox?3?5too?5many?5cells@ 351e0418     physicalworld.obj
 0002:00002474       ??_C@_04IBBNLEM@Game?$AA@  351e0474     physicalworld.obj
 0002:0000247c       ??_C@_0BM@NPIOPJJB@GetEntitiesAround?$CIExternal?$CJ?$AA@ 351e047c     physicalworld.obj
 0002:00002498       ??_C@_0BL@PFOGMOID@GetEntitiesAround?$CIPhysics?$CJ?$AA@ 351e0498     physicalworld.obj
 0002:000024b4       ??_C@_0CC@FMONOPEM@CPhysicalWorld?3?3GetEntitiesAroun@ 351e04b4     physicalworld.obj
 0002:000024d8       __real@4e6e6b28            351e04d8     physicalworld.obj
 0002:000024dc       ??_C@_0CG@DAIPOGMA@CPhysicalWorld?3?3CollideEntityWit@ 351e04dc     physicalworld.obj
 0002:00002504       ??_C@_0CL@DKEANCLN@CPhysicalWorld?3?3CollideEntityWit@ 351e0504     physicalworld.obj
 0002:00002530       __real@41cdcd6500000000    351e0530     physicalworld.obj
 0002:00002538       ??_C@_03GEPAOBPJ@com?$AA@  351e0538     physicalworld.obj
 0002:0000253c       ??_C@_08PGIAAJBG@simclass?$AA@ 351e053c     physicalworld.obj
 0002:00002548       ??_C@_0L@LDLJOCKM@entity_ptr?$AA@ 351e0548     physicalworld.obj
 0002:00002554       ??_C@_0BD@INDOKC@Physical?5Grid?5Pool?$AA@ 351e0554     physicalworld.obj
 0002:00002568       ??_C@_0EI@FEBOPGDO@Error?3?5too?5many?5entity?5grid?5thun@ 351e0568     physicalworld.obj
 0002:000025b0       ??_C@_0DD@GLNFKCFH@Error?3?5?$CFs?5?$EA?5?$CF?41f?0?$CF?41f?0?$CF?41f?5is?5to@ 351e05b0     physicalworld.obj
 0002:000025e4       ??_C@_06GOJKNBFM@entity?$AA@ 351e05e4     physicalworld.obj
 0002:000025ec       __real@43800000            351e05ec     physicalworld.obj
 0002:000025f0       __real@c3480000            351e05f0     physicalworld.obj
 0002:000025f4       __real@bf4ccccd            351e05f4     physicalworld.obj
 0002:000025f8       __real@34000000            351e05f8     physicalworld.obj
 0002:000025fc       ??_C@_0CC@HNDNKDHE@CPhysicalWorld?3?3SimulateExplosio@ 351e05fc     physicalworld.obj
 0002:00002620       __real@4202a05f20000000    351e0620     physicalworld.obj
 0002:00002628       ??_C@_0CL@EIIFGMOL@CPhysicalWorld?3?3PrimitiveWorldIn@ 351e0628     physicalworld.obj
 0002:00002654       __real@c1200000            351e0654     physicalworld.obj
 0002:00002658       ??_C@_0BF@HMDKKHBB@CreatePhysicalEntity?$AA@ 351e0658     physicalworld.obj
 0002:00002670       ??_C@_0CF@MPBHKPK@CPhysicalWorld?3?3CreatePhysicalEn@ 351e0670     physicalworld.obj
 0002:00002698       ??_C@_0CG@NDJJNCNB@CPhysicalWorld?3?3DestroyPhysicalE@ 351e0698     physicalworld.obj
 0002:000026c0       ??_C@_0BC@NNEDADDI@D?3?2worldgeoms?4txt?$AA@ 351e06c0     physicalworld.obj
 0002:000026d4       ??_C@_0BB@PHBCIJJB@D?3?2worldents?4txt?$AA@ 351e06d4     physicalworld.obj
 0002:000026e8       ??_C@_0BE@MNKPLEKN@PhysicsWorkerThread?$AA@ 351e06e8     physicalworld.obj
 0002:000026fc       ??_C@_0BJ@KLNIBABK@CPhysicalWorld?3?3TimeStep?$AA@ 351e06fc     physicalworld.obj
 0002:00002718       ??_C@_0P@JAKLJLMO@RB?5thread?5data?$AA@ 351e0718     rigidbody.obj
 0002:00002728       ??_C@_0BH@JPFBLAOJ@Physics?5Contact?5Solver?$AA@ 351e0728     rigidbody.obj
 0002:00002740       __real@3f8020c5            351e0740     rigidbody.obj
 0002:00002744       ??_C@_05EBOPLLCF@LCPMC?$AA@ 351e0744     rigidbody.obj
 0002:00002750       __real@4034000000000000    351e0750     rigidbody.obj
 0002:00002758       ??_C@_0N@CNCBJKKN@LCPCG?9unproj?$AA@ 351e0758     rigidbody.obj
 0002:00002768       __real@3f50624dd2f1a9fc    351e0768     rigidbody.obj
 0002:00002770       __real@4049000000000000    351e0770     rigidbody.obj
 0002:00002778       ??_C@_05CPBNFDCL@LCPCG?$AA@ 351e0778     rigidbody.obj
 0002:00002780       __real@80000000            351e0780     rigidbody.obj
 0002:00002784       __real@bd4ccccd            351e0784     rigidbody.obj
 0002:00002788       __real@bf8eb851e0000000    351e0788     rigidbody.obj
 0002:00002790       __real@bf70624de0000000    351e0790     rigidbody.obj
 0002:00002798       __real@407f400000000000    351e0798     rigidbody.obj
 0002:000027a0       __real@39b4484bfeebc2a0    351e07a0     rigidbody.obj
 0002:000027a8       ??_C@_05LNAIGO@PreCG?$AA@  351e07a8     rigidbody.obj
 0002:000027b0       ??_C@_0BE@OAMBIDAL@InvokeContactSolver?$AA@ 351e07b0     rigidbody.obj
 0002:000027c4       ??_C@_06HPGEIPLA@?$DMnull?$DO?$AA@ 351e07c4     rigidentity.obj
 0002:000027cc       ??_C@_07KAALEJHI@?$DMlocal?$DO?$AA@ 351e07cc     rigidentity.obj
 0002:000027e8       ??_C@_02DKCKIIND@?$CFs?$AA@ 351e07e8     rigidentity.obj
 0002:000027ec       __real@c3000000            351e07ec     rigidentity.obj
 0002:000027f0       __real@43000000            351e07f0     rigidentity.obj
 0002:000027f4       __real@44800000            351e07f4     rigidentity.obj
 0002:000027f8       ??_C@_0CI@IOKCCNHB@Deleting?5Reference?5Counted?5Objec@ 351e07f8     rigidentity.obj
 0002:00002820       __real@3ba0902e            351e0820     rigidentity.obj
 0002:00002828       ??_7CRigidEntity@@6B@      351e0828     rigidentity.obj
 0002:0000295c       __real@44cccb33            351e095c     rigidentity.obj
 0002:00002960       __real@4423d5c3            351e0960     rigidentity.obj
 0002:00002964       ??_C@_0P@BDPDOPPG@sequenceNumber?$AA@ 351e0964     rigidentity.obj
 0002:00002974       ??_C@_06JPLOHAIH@angvel?$AA@ 351e0974     rigidentity.obj
 0002:0000297c       ??_C@_03BHFFHIBL@rot?$AA@  351e097c     rigidentity.obj
 0002:00002980       __real@3cb851ec            351e0980     rigidentity.obj
 0002:00002984       __real@3f7ff972            351e0984     rigidentity.obj
 0002:00002988       __real@bf99999a            351e0988     rigidentity.obj
 0002:00002990       __real@bff0000000000000    351e0990     rigidentity.obj
 0002:00002998       __real@3eaaaaab            351e0998     rigidentity.obj
 0002:0000299c       __real@3f80a3d7            351e099c     rigidentity.obj
 0002:000029a0       __real@43960000            351e09a0     rigidentity.obj
 0002:000029a4       __real@3f70a3d7            351e09a4     rigidentity.obj
 0002:000029a8       __real@bf59999a            351e09a8     rigidentity.obj
 0002:000029ac       __real@3e19999a            351e09ac     rigidentity.obj
 0002:000029b0       ??_C@_0BP@EANKIJJH@CRigidEntity?3?3RegisterContacts?$AA@ 351e09b0     rigidentity.obj
 0002:000029d0       ??_C@_0O@KJLDCHNC@maxBendTorque?$AA@ 351e09d0     rigidentity.obj
 0002:000029e0       ??_C@_0N@PCBEGNKJ@breakableAng?$AA@ 351e09e0     rigidentity.obj
 0002:000029f0       ??_C@_0N@NHHOIIFK@maxPullForce?$AA@ 351e09f0     rigidentity.obj
 0002:00002a00       ??_C@_0N@NEPDBILI@breakableLin?$AA@ 351e0a00     rigidentity.obj
 0002:00002a10       ??_C@_06KGHINEPG@radius?$AA@ 351e0a10     rigidentity.obj
 0002:00002a18       ??_C@_07IANOJGAO@damping?$AA@ 351e0a18     rigidentity.obj
 0002:00002a20       ??_C@_05GECEPKB@flags?$AA@ 351e0a20     rigidentity.obj
 0002:00002a28       ??_C@_06CNGEOGNK@yzlim1?$AA@ 351e0a28     rigidentity.obj
 0002:00002a30       ??_C@_06DEHPNHJL@yzlim0?$AA@ 351e0a30     rigidentity.obj
 0002:00002a38       ??_C@_05DHNHFHMF@yzlim?$AA@ 351e0a38     rigidentity.obj
 0002:00002a40       ??_C@_05DFPCKMPE@xlim1?$AA@ 351e0a40     rigidentity.obj
 0002:00002a48       ??_C@_05CMOJJNLF@xlim0?$AA@ 351e0a48     rigidentity.obj
 0002:00002a50       ??_C@_04BGNKAOBC@xlim?$AA@ 351e0a50     rigidentity.obj
 0002:00002a58       ??_C@_07LBPEBLNH@qframe1?$AA@ 351e0a58     rigidentity.obj
 0002:00002a60       ??_C@_07NKFCNLOK@qf1used?$AA@ 351e0a60     rigidentity.obj
 0002:00002a68       ??_C@_07KIOPCKJG@qframe0?$AA@ 351e0a68     rigidentity.obj
 0002:00002a70       ??_C@_07BBAOAIEP@qf0used?$AA@ 351e0a70     rigidentity.obj
 0002:00002a78       ??_C@_07JOFJMAFF@partid1?$AA@ 351e0a78     rigidentity.obj
 0002:00002a80       ??_C@_07IHECPBBE@partid0?$AA@ 351e0a80     rigidentity.obj
 0002:00002a88       ??_C@_03CACBEHEB@pt1?$AA@  351e0a88     rigidentity.obj
 0002:00002a8c       ??_C@_03DJDKHGAA@pt0?$AA@  351e0a8c     rigidentity.obj
 0002:00002a90       ??_C@_0L@HOHHMJMM@constraint?$AA@ 351e0a90     rigidentity.obj
 0002:00002a9c       ??_C@_05IOMEMJEC@count?$AA@ 351e0a9c     rigidentity.obj
 0002:00002aa4       ??_C@_0M@JGLONDGH@constraints?$AA@ 351e0aa4     rigidentity.obj
 0002:00002ab0       ??_C@_0EL@PLDAGNFJ@Error?3?5Rigid?5Body?5?$CI?$EA?$CF?41f?0?$CF?41f?0?$CF?4@ 351e0ab0     rigidentity.obj
 0002:00002b00       __real@bfefef9db9100000    351e0b00     rigidentity.obj
 0002:00002b08       __real@3c4ccccd            351e0b08     rigidentity.obj
 0002:00002b10       ??_C@_0EN@EHOJENEE@CRigidEntity?3?3AddGeometry?3?5?$CI?$CFs?5a@ 351e0b10     rigidentity.obj
 0002:00002b60       ??_C@_0CE@MCBDAAIP@CRigidEntity?3Action?$CIaction_impul@ 351e0b60     rigidentity.obj
 0002:00002b84       __real@3d75c28f            351e0b84     rigidentity.obj
 0002:00002b88       ??_C@_0CD@BGBGOAEC@CRigidEntity?3?3RegisterContactPoi@ 351e0b88     rigidentity.obj
 0002:00002bac       __real@40600000            351e0bac     rigidentity.obj
 0002:00002bb0       ??_C@_0BP@ODPDJPC@CRigidEntity?3?3DelayedIntersect?$AA@ 351e0bb0     rigidentity.obj
 0002:00002bd0       __real@3a200140            351e0bd0     rigidentity.obj
 0002:00002bd4       __real@3ac80190            351e0bd4     rigidentity.obj
 0002:00002bd8       ??_C@_07OHHAEMPA@seq?3?5?$CFf?$AA@ 351e0bd8     rigidentity.obj
 0002:00002be0       ??_C@_07NFEGCOHC@seq?3?5?$CFd?$AA@ 351e0be0     rigidentity.obj
 0002:00002be8       __real@ba83126f            351e0be8     rigidentity.obj
 0002:00002bec       __real@3f35c28f            351e0bec     rigidentity.obj
 0002:00002bf0       __real@3d7a35dd            351e0bf0     rigidentity.obj
 0002:00002bf4       __real@3e428f5c            351e0bf4     rigidentity.obj
 0002:00002bf8       ??_C@_0BD@GCCCEIEI@CRigidEntity?3?3Step?$AA@ 351e0bf8     rigidentity.obj
 0002:00002c18       ??_7CRopeEntity@@6B@       351e0c18     ropeentity.obj
 0002:00002d34       __real@6aa56fa6            351e0d34     ropeentity.obj
 0002:00002d38       ??_C@_03HCMCBFLP@_?$CFd?$AA@ 351e0d38     ropeentity.obj
 0002:00002d3c       __real@26901d7d            351e0d3c     ropeentity.obj
 0002:00002d40       __real@bba3d70a            351e0d40     ropeentity.obj
 0002:00002d44       ??_C@_0P@BGLENKAJ@Rope?5solver?5MC?$AA@ 351e0d44     ropeentity.obj
 0002:00002d54       ??_C@_0P@HIEGDCAH@Rope?5solver?5CG?$AA@ 351e0d54     ropeentity.obj
 0002:00002d64       __real@428c0000            351e0d64     ropeentity.obj
 0002:00002d68       __real@3ad1b717            351e0d68     ropeentity.obj
 0002:00002d6c       __real@3f59999a            351e0d6c     ropeentity.obj
 0002:00002d70       __real@3f100000            351e0d70     ropeentity.obj
 0002:00002d74       __real@bf7eb852            351e0d74     ropeentity.obj
 0002:00002d78       ??_C@_04DMCMFBAM@tied?$AA@ 351e0d78     ropeentity.obj
 0002:00002d80       ??_C@_04OHHBHOGB@link?$AA@ 351e0d80     ropeentity.obj
 0002:00002d88       ??_C@_08BLGKBCOE@saveties?$AA@ 351e0d88     ropeentity.obj
 0002:00002d94       ??_C@_08JFDIBHCE@pt_tied1?$AA@ 351e0d94     ropeentity.obj
 0002:00002da0       ??_C@_08IMCDCGGF@pt_tied0?$AA@ 351e0da0     ropeentity.obj
 0002:00002dac       ??_C@_05FDOEMPCF@Verts?$AA@ 351e0dac     ropeentity.obj
 0002:00002db4       ??_C@_04OFJFANPM@nvtx?$AA@ 351e0db4     ropeentity.obj
 0002:00002dbc       ??_C@_04DBMENFI@Segs?$AA@  351e0dbc     ropeentity.obj
 0002:00002dc4       ??_C@_07DDKGOFMH@pos_end?$AA@ 351e0dc4     ropeentity.obj
 0002:00002dcc       ??_C@_09IAPMPKID@pos_start?$AA@ 351e0dcc     ropeentity.obj
 0002:00002dd8       ??_C@_08EAMLKELC@strained?$AA@ 351e0dd8     ropeentity.obj
 0002:00002de4       ??_C@_05IHMDFKMI@nsegs?$AA@ 351e0de4     ropeentity.obj
 0002:00002dec       __real@322bcc76            351e0dec     ropeentity.obj
 0002:00002df0       __real@3ea00000            351e0df0     ropeentity.obj
 0002:00002df4       __real@3ec00000            351e0df4     ropeentity.obj
 0002:00002df8       __real@3f7ae148            351e0df8     ropeentity.obj
 0002:00002dfc       __real@3d23d70b            351e0dfc     ropeentity.obj
 0002:00002e00       __real@3db851ec            351e0e00     ropeentity.obj
 0002:00002e08       __real@3f1cd5f99c38b04b    351e0e08     ropeentity.obj
 0002:00002e10       __real@3fa66666            351e0e10     ropeentity.obj
 0002:00002e14       __real@3f7860ab            351e0e14     ropeentity.obj
 0002:00002e18       ??_C@_0P@EFOJKOHM@Rope?5collision?$AA@ 351e0e18     ropeentity.obj
 0002:00002e28       __real@3da3d70a            351e0e28     ropeentity.obj
 0002:00002e2c       ??_C@_0BC@KAOKIHJG@CRopeEntity?3?3Step?$AA@ 351e0e2c     ropeentity.obj
 0002:00002e48       __real@453b8000            351e0e48     softentity.obj
 0002:00002e50       ??_7CSoftEntity@@6B@       351e0e50     softentity.obj
 0002:00002f6c       ??_C@_0CD@HHJJGFJC@CSoftEntity?3Action?$CIaction_impuls@ 351e0f6c     softentity.obj
 0002:00002f90       ??_C@_03CEPBOMNB@vtx?$AA@  351e0f90     softentity.obj
 0002:00002f94       ??_C@_07OOCOMFL@updated?$AA@ 351e0f94     softentity.obj
 0002:00002f9c       ??_C@_0BC@LKGJNKHC@CSoftEntity?3?3Step?$AA@ 351e0f9c     softentity.obj
 0002:00002fc0       ??_7CHeightfieldBV@@6B@    351e0fc0     waterman.obj
 0002:00003030       ??_7CHeightfield@@6B@      351e1030     waterman.obj
 0002:00003130       __real@bf8020c5            351e1130     waterman.obj
 0002:00003134       __real@3fc147ae            351e1134     waterman.obj
 0002:00003138       __real@bf028f5c            351e1138     waterman.obj
 0002:00003150       __real@4023193d66ed2bfb    351e1150     wheeledvehicleentity.obj
 0002:00003158       __real@44ffe000            351e1158     wheeledvehicleentity.obj
 0002:0000315c       __real@4223d1ec            351e115c     wheeledvehicleentity.obj
 0002:00003160       __real@3a001002            351e1160     wheeledvehicleentity.obj
 0002:00003164       __real@3cc80640            351e1164     wheeledvehicleentity.obj
 0002:00003168       ??_C@_07IODEONID@curGear?$AA@ 351e1168     wheeledvehicleentity.obj
 0002:00003170       ??_C@_09DGHJKKCO@handbrake?$AA@ 351e1170     wheeledvehicleentity.obj
 0002:0000317c       ??_C@_07OAMHNPGL@wengine?$AA@ 351e117c     wheeledvehicleentity.obj
 0002:00003184       ??_C@_05JADEHCLC@steer?$AA@ 351e1184     wheeledvehicleentity.obj
 0002:0000318c       ??_C@_05CANEEOEI@pedal?$AA@ 351e118c     wheeledvehicleentity.obj
 0002:00003198       __real@3fbacee9f37bebd5    351e1198     wheeledvehicleentity.obj
 0002:000031a0       __real@c01921fb54442d18    351e11a0     wheeledvehicleentity.obj
 0002:000031a8       ??_7CWheeledVehicleEntity@@6B@ 351e11a8     wheeledvehicleentity.obj
 0002:000032dc       __real@3f5db22d            351e12dc     wheeledvehicleentity.obj
 0002:000032e0       __real@457a0000            351e12e0     wheeledvehicleentity.obj
 0002:000032e4       __real@41400000            351e12e4     wheeledvehicleentity.obj
 0002:000032e8       __real@41c00000            351e12e8     wheeledvehicleentity.obj
 0002:000032ec       __real@3f490fdb            351e12ec     wheeledvehicleentity.obj
 0002:000032f0       ??_C@_0EF@EDDEFNIG@CWheeledVehicleEntity?3?3AddGeomet@ 351e12f0     wheeledvehicleentity.obj
 0002:00003338       __real@bc23d70a            351e1338     wheeledvehicleentity.obj
 0002:0000333c       ??_C@_0CP@CDDJNAEK@CWheeledVehicleEntity?3?3CheckAddi@ 351e133c     wheeledvehicleentity.obj
 0002:00003374       __real@33d6bf95            351e1374     boolean2d.obj
 0002:00003378       __real@36a7c5ac            351e1378     boolean2d.obj
 0002:00003388       ??_7bop_meshupdate_thunk@@6B@ 351e1388     boolean3d.obj
 0002:0000338c       ??_7bop_meshupdate@@6B@    351e138c     boolean3d.obj
 0002:00003390       __real@3b449ba6            351e1390     boolean3d.obj
 0002:00003394       __real@3a03126f            351e1394     boolean3d.obj
 0002:00003398       __real@3f7fbe77            351e1398     boolean3d.obj
 0002:0000339c       ??_C@_0BD@IANNIDHM@CTriMesh?3?3Subtract?$AA@ 351e139c     boolean3d.obj
 0002:000033b0       __real@3f60624de0000000    351e13b0     qhull.obj
 0002:000033b8       __real@bb03126f            351e13b8     qhull.obj
 0002:000033c0       __real@bf60624de0000000    351e13c0     qhull.obj
 0002:000033c8       __real@bf50624de0000000    351e13c8     qhull.obj
 0002:000033d0       __real@fcf0bdc2            351e13d0     qhull.obj
 0002:000033e8       __real@bf91111111111111    351e13e8     utils.obj
 0002:000033f0       __real@3f91111111111111    351e13f0     utils.obj
 0002:000033f8       __real@3fa5555555555555    351e13f8     utils.obj
 0002:00003400       __real@bfa999999999999a    351e1400     utils.obj
 0002:00003408       __real@bfb5555555555555    351e1408     utils.obj
 0002:00003410       __real@bfc5555555555555    351e1410     utils.obj
 0002:00003418       __real@3fa999999999999a    351e1418     utils.obj
 0002:00003420       __real@3fb5555555555555    351e1420     utils.obj
 0002:00003428       ??_C@_0BB@KMIBLBAG@ReadPacked?5i?$DN?$DN?$CFi?$AA@ 351e1428     utils.obj
 0002:00003440       __real@c080000000000000    351e1440     utils.obj
 0002:00003448       __real@44000000            351e1448     utils.obj
 0002:0000344c       __real@45000000            351e144c     utils.obj
 0002:00003450       __real@c0a0000000000000    351e1450     utils.obj
 0002:00003458       __real@3b000000            351e1458     utils.obj
 0002:00003460       __real@3bc79ca100000000    351e1460     utils.obj
 0002:00003468       __real@37800080            351e1468     utils.obj
 0002:00003470       __real@3fee666660000000    351e1470     utils.obj
 0002:00003478       __real@3fb45f306dc9c883    351e1478     utils.obj
 0002:00003480       __real@3fd3333333333333    351e1480     utils.obj
 0002:00003488       __real@3fe6666666666666    351e1488     utils.obj
 0002:00003490       __real@3ee4f8b588e368f1    351e1490     utils.obj
 0002:00003498       ??_C@_0DC@MJBDGDCG@Unsupported?5polygon?5size?5for?5Occ@ 351e1498     utils.obj
 0002:000034d0       __real@40d45f07af68ecef    351e14d0     utils.obj
 0002:000034d8       __real@3ff8a71a0cc42d18    351e14d8     utils.obj
 0002:000034e0       __real@be860a92            351e14e0     utils.obj
 0002:000034e8       __real@3f09222d989f5e57    351e14e8     utils.obj
 0002:000034f8       __real@3c800000            351e14f8     aabbtree.obj
 0002:000034fc       ??_C@_0L@PDPAOLJI@AABB?5trees?$AA@ 351e14fc     aabbtree.obj
 0002:00003508       __real@42800000            351e1508     aabbtree.obj
 0002:0000350c       __real@42fe0000            351e150c     aabbtree.obj
 0002:00003510       __real@c9742400            351e1510     aabbtree.obj
 0002:00003528       __real@3eb0c6f7a0000000    351e1528     capsulegeom.obj
 0002:00003530       __real@3e960418            351e1530     capsulegeom.obj
 0002:00003534       __real@3f34fdf4            351e1534     capsulegeom.obj
 0002:00003538       __real@3f2aaaab            351e1538     capsulegeom.obj
 0002:0000353c       __real@40860a92            351e153c     capsulegeom.obj
 0002:00003550       __real@3ff921fb54442d18    351e1550     cylindergeom.obj
 0002:00003558       __real@3faaaaab            351e1558     cylindergeom.obj
 0002:0000355c       __real@3e000000            351e155c     cylindergeom.obj
 0002:00003560       __real@beaaaaab            351e1560     cylindergeom.obj
 0002:00003578       ??_7CVoxelBV@@6B@          351e1578     geoman.obj
 0002:000035e4       ??_7CBreakableGrid2d@@6B@  351e15e4     geoman.obj
 0002:00003600       ??_C@_0BA@JHFFHIMH@brekable2d?5grid?$AA@ 351e1600     geoman.obj
 0002:00003610       ??_7CMemStream@@6B@        351e1610     geoman.obj
 0002:00003620       ??_7CVoxelGeom@@6B@        351e1620     geoman.obj
 0002:00003748       __real@3f60624dd2f1a9fc    351e1748     heightfieldgeom.obj
 0002:00003750       __real@3f1a36e2e0000000    351e1750     heightfieldgeom.obj
 0002:00003758       __real@3fe6a09e667f3bcd    351e1758     heightfieldgeom.obj
 0002:00003768       __real@2f52f8ac174d6123    351e1768     intersectionchecks.obj
 0002:00003770       __real@3feff7ced916872b    351e1770     intersectionchecks.obj
 0002:00003778       __real@3d17b426            351e1778     intersectionchecks.obj
 0002:0000377c       __real@3e2aaaab            351e177c     intersectionchecks.obj
 0002:00003780       __real@3fef5c2900000000    351e1780     intersectionchecks.obj
 0002:00003788       __real@bf3504f3            351e1788     intersectionchecks.obj
 0002:0000378c       __real@3f3504f3            351e178c     intersectionchecks.obj
 0002:00003790       __real@be4ccccd            351e1790     intersectionchecks.obj
 0002:00003794       ??_C@_0BB@PKNEGLNF@RB_PrimIntersect?$AA@ 351e1794     jobq.obj
 0002:000037a8       ??_C@_0N@IPMPGLJF@Featherstone?$AA@ 351e17a8     jobq.obj
 0002:000037b8       ??_C@_04FEDAIEKO@Rope?$AA@ 351e17b8     jobq.obj
 0002:000037c0       ??_C@_09HHOKDCAB@RB_Solver?$AA@ 351e17c0     jobq.obj
 0002:000037cc       ??_C@_0BB@NPOCPIBL@RB_GeomIntersect?$AA@ 351e17cc     jobq.obj
 0002:000037f0       __real@bfffd70a40000000    351e17f0     linunprojectionchecks.obj
 0002:000037f8       __real@c007eb8520000000    351e17f8     linunprojectionchecks.obj
 0002:00003800       __real@3fa99999a0000000    351e1800     linunprojectionchecks.obj
 0002:00003808       __real@3fefef9db22d0e56    351e1808     linunprojectionchecks.obj
 0002:00003810       __real@3f847ae140000000    351e1810     linunprojectionchecks.obj
 0002:00003818       __real@3f40624dd2f1a9fc    351e1818     linunprojectionchecks.obj
 0002:00003820       __real@3ff028f5c28f5c29    351e1820     linunprojectionchecks.obj
 0002:00003828       __real@3fefae147ae147ae    351e1828     linunprojectionchecks.obj
 0002:00003830       __real@3f804189            351e1830     linunprojectionchecks.obj
 0002:00003838       __real@3feff7cee0000000    351e1838     linunprojectionchecks.obj
 0002:00003840       __real@3ff00418a0000000    351e1840     linunprojectionchecks.obj
 0002:00003848       __real@3fa2f684bda12f68    351e1848     linunprojectionchecks.obj
 0002:00003850       __real@3efa36e2d7731900    351e1850     linunprojectionchecks.obj
 0002:00003858       __real@3f689374c0000000    351e1858     linunprojectionchecks.obj
 0002:00003860       __real@3f747ae140000000    351e1860     linunprojectionchecks.obj
 0002:00003868       __real@3f50624de0000000    351e1868     linunprojectionchecks.obj
 0002:00003870       __real@ffee42d130773b76    351e1870     obbtree.obj
 0002:00003878       __real@7fee42d130773b76    351e1878     obbtree.obj
 0002:00003880       ??_C@_09HCPCMEJO@OBB?5trees?$AA@ 351e1880     obbtree.obj
 0002:000038a0       __real@3feeb851eb851eb8    351e18a0     rotunprojectionchecks.obj
 0002:000038a8       __real@3ff0a3d70a3d70a4    351e18a8     rotunprojectionchecks.obj
 0002:000038b0       __real@3ff0525460aa64c3    351e18b0     rotunprojectionchecks.obj
 0002:000038b8       __real@3fef5cfaacd9e83e    351e18b8     rotunprojectionchecks.obj
 0002:000038d8       ??_C@_0CD@LFICKIIJ@PrimitiveWorldIntersection?$CIQueue@ 351e18d8     rwi.obj
 0002:000038fc       ??_C@_0BN@NCMAGHFA@RayWorldIntersection?$CIQueued?$CJ?$AA@ 351e18fc     rwi.obj
 0002:0000391c       ??_C@_0CF@KIKHOLPD@CPhysicalWorld?3?3RayWorldIntersec@ 351e191c     rwi.obj
 0002:00003944       ??_C@_0BA@CEOHFAK@SingleBox?5trees?$AA@ 351e1944     singleboxtree.obj
 0002:00003968       __real@41490fdb            351e1968     spheregeom.obj
 0002:0000396c       __real@bf7fbe77            351e196c     spheregeom.obj
 0002:00003970       __real@3fe6a09e667f3bcc    351e1970     spheregeom.obj
 0002:00003978       __real@3f828f5c            351e1978     spheregeom.obj
 0002:00003984       ??_7IPhysicalEntityIt@@6B@ 351e1984     physicalworld.obj
 0002:00003984       ??_7ITetrLattice@@6B@      351e1984     tetrlattice.obj
 0002:00003984       ??_7IBreakableGrid2d@@6B@  351e1984     geoman.obj
 0002:000039a0       ??_7CTetrLattice@@6B@      351e19a0     tetrlattice.obj
 0002:000039bc       ??_C@_0BN@LFEFBEHO@CTetrLattice?3?3CheckStructure?$AA@ 351e19bc     tetrlattice.obj
 0002:000039dc       __real@3f004189            351e19dc     tetrlattice.obj
 0002:000039f0       ??_7COBBTree@@6B@          351e19f0     trimesh.obj
 0002:00003a60       ??_7CAABBTree@@6B@         351e1a60     trimesh.obj
 0002:00003ad0       ??_7CTriMesh@@6B@          351e1ad0     trimesh.obj
 0002:00003bd0       ??_C@_0O@EBEONEPM@auxilary?5data?$AA@ 351e1bd0     trimesh.obj
 0002:00003be0       ??_C@_0BB@NABIJMGH@wasted?5mesh?5data?$AA@ 351e1be0     trimesh.obj
 0002:00003bf4       ??_C@_09HDIEJGOE@mesh?5data?$AA@ 351e1bf4     trimesh.obj
 0002:00003c00       ??_C@_0BI@PKAJMKLJ@CTriMesh?3?3RebuildBVTree?$AA@ 351e1c00     trimesh.obj
 0002:00003c18       __real@39d1b717            351e1c18     trimesh.obj
 0002:00003c1c       __real@40029cbc            351e1c1c     trimesh.obj
 0002:00003c20       __real@3efae147            351e1c20     trimesh.obj
 0002:00003c24       __real@3951b717            351e1c24     trimesh.obj
 0002:00003c28       __real@40001062            351e1c28     trimesh.obj
 0002:00003c48       ??_C@_0M@KMODIPJI@voxel?5grids?$AA@ 351e1c48     voxelgeom.obj
 0002:00003c54       ??_7ISystemEventListener@@6B@ 351e1c54     CryPhysics.obj
 0002:00003c5c       ??_C@_0BD@PJOKHJBB@Pure?5function?5call?$AA@ 351e1c5c     CryPhysics.obj
 0002:00003c70       ??_C@_0CL@LKHBOBAH@Invalid?5parameter?5detected?5in?5CR@ 351e1c70     CryPhysics.obj
 0002:00003c9c       ??_C@_0DJ@DLJMMMP@Could?5not?5access?5CrySystem?4dll?5?$CI@ 351e1c9c     CryPhysics.obj
 0002:00003cd8       ??_C@_0P@NHEMOHAI@Memory?5Manager?$AA@ 351e1cd8     CryPhysics.obj
 0002:00003ce8       ??_C@_0O@FFDHMLKN@CrySystem?4dll?$AA@ 351e1ce8     CryPhysics.obj
 0002:00003cf8       ??_C@_0BO@JDKBDPNB@CryGetIMemoryManagerInterface?$AA@ 351e1cf8     CryPhysics.obj
 0002:00003d18       ??_C@_0BB@PNKHDABP@CrySystemCrtFree?$AA@ 351e1d18     CryPhysics.obj
 0002:00003d2c       ??_C@_0BB@MFMFBMDO@CrySystemCrtSize?$AA@ 351e1d2c     CryPhysics.obj
 0002:00003d40       ??_C@_0BD@BBIFHONI@CrySystemCrtMalloc?$AA@ 351e1d40     CryPhysics.obj
 0002:00003d54       ??_C@_0O@LCCIKADF@CryGetMemSize?$AA@ 351e1d54     CryPhysics.obj
 0002:00003d64       ??_C@_07CKAGCLEE@CryFree?$AA@ 351e1d64     CryPhysics.obj
 0002:00003d6c       ??_C@_0L@FICCDMFO@CryRealloc?$AA@ 351e1d6c     CryPhysics.obj
 0002:00003d78       ??_C@_09MCKPOEAK@CryMalloc?$AA@ 351e1d78     CryPhysics.obj
 0002:00003d84       ??_C@_0BO@HAMEIFMK@Critical?5Section?5hanging?5lock?$AA@ 351e1d84     CryPhysics.obj
 0002:00003da4       ??_7IPhysUtils@@6B@        351e1da4     physicalworld.obj
 0002:00003da4       ??_7ICryUnknown@@6B@       351e1da4     CryPhysics.obj
 0002:00003db8       ?iid@?1??IID@ICryUnknown@@CAABUCryGUID@@XZ@4U3@B 351e1db8     CryPhysics.obj
 0002:00003dc8       ?iid@?1??IID@IEngineModule@@CAABUCryGUID@@XZ@4U3@B 351e1dc8     CryPhysics.obj
 0002:00003dd8       ??_7ICryFactory@@6B@       351e1dd8     CryPhysics.obj
 0002:00003df0       ??_7CSystemEventListner_Physics@@6B@ 351e1df0     CryPhysics.obj
 0002:00003df8       __real@3ac90fdb            351e1df8     CryPhysics.obj
 0002:00003dfc       ??_C@_0L@CODMBEB@CryPhysics?$AA@ 351e1dfc     CryPhysics.obj
 0002:00003e08       ??_7CEngineModule_CryPhysics@@6B@ 351e1e08     CryPhysics.obj
 0002:00003e24       ??_C@_09BHIABECK@CryEngine?$AA@ 351e1e24     CryPhysics.obj
 0002:00003e30       ??_7CFactory@CEngineModule_CryPhysics@@6B@ 351e1e30     CryPhysics.obj
 0002:00003e48       ??_7bad_alloc@std@@6B@     351e1e48     CryPhysics.obj
 0002:00003e50       ??_C@_0P@GHFPNOJB@bad?5allocation?$AA@ 351e1e50     CryPhysics.obj
 0002:00003e60       ??_7sp_counted_base@detail@boost@@6B@ 351e1e60     CryPhysics.obj
 0002:00003e70       ??_C@_0BI@KMAEJCIO@EngineModule_CryPhysics?$AA@ 351e1e70     CryPhysics.obj
 0002:00003e88       ?cid@?1??GetClassID@CFactory@CEngineModule_CryPhysics@@UBEABUCryGUID@@XZ@4U4@B 351e1e88     CryPhysics.obj
 0002:00003e98       ??_7?$sp_counted_impl_p@VCEngineModule_CryPhysics@@@detail@boost@@6B@ 351e1e98     CryPhysics.obj
 0002:00003ea8       ??_C@_0BN@FOKPCDPC@Boost?5threw?5an?5exception?3?5?$CFs?$AA@ 351e1ea8     CryPhysics.obj
 0002:00003ed8       __pRawDllMain              351e1ed8     MSVCRT:crtdll.obj
 0002:00003ed8       __pDefaultRawDllMain       351e1ed8     MSVCRT:crtdll.obj
 0002:00003ee8       __load_config_used         351e1ee8     MSVCRT:loadcfg.obj
 0002:00003f90       ___safe_se_handler_table   351e1f90     <linker-defined>
 0002:00003f94       ___rtc_iaa                 351e1f94     MSVCRT:_initsect_.obj
 0002:00003f98       ___rtc_izz                 351e1f98     MSVCRT:_initsect_.obj
 0002:00003f9c       ___rtc_taa                 351e1f9c     MSVCRT:_initsect_.obj
 0002:00003fa0       ___rtc_tzz                 351e1fa0     MSVCRT:_initsect_.obj
 0002:0000400c       __IMPORT_DESCRIPTOR_KERNEL32 351e200c     kernel32:KERNEL32.dll
 0002:00004020       __IMPORT_DESCRIPTOR_USER32 351e2020     user32:USER32.dll
 0002:00004034       __IMPORT_DESCRIPTOR_MSVCR100 351e2034     MSVCRT:MSVCR100.dll
 0002:00004048       __NULL_IMPORT_DESCRIPTOR   351e2048     kernel32:KERNEL32.dll
 0003:00000000       ?fVec3_One@?$Vec3Constants@M@@2U?$Vec3_tpl@M@@B 351e3000     articulatedentity.obj
 0003:0000003c       ?g_stub@@3VCPhysicalStub@@A 351e303c     physarea.obj
 0003:00000058       ?sEmptyStringBuffer@?1??_emptyHeader@?$CryStringT@D@@KAPAUStrHeader@2@XZ@4PAU32@A 351e3058     physicalentity.obj
 0003:00000088       ?g_physThreadId@@3HA       351e3088     physicalworld.obj
 0003:0000008c       ?__cursubstep@@3HA         351e308c     physicalworld.obj
 0003:00000160       ?fVec3_Zero@?$Vec3Constants@M@@2U?$Vec3_tpl@M@@B 351e3160     rigidentity.obj
 0003:0000016c       ?fVec2_Zero@?$Vec2Constants@M@@2U?$Vec2_tpl@M@@A 351e316c     rigidentity.obj
 0003:00000174       ?fVec2_OneX@?$Vec2Constants@M@@2U?$Vec2_tpl@M@@A 351e3174     rigidentity.obj
 0003:0000017c       ?fVec2_OneY@?$Vec2Constants@M@@2U?$Vec2_tpl@M@@A 351e317c     rigidentity.obj
 0003:00000184       ?fVec2_One@?$Vec2Constants@M@@2U?$Vec2_tpl@M@@A 351e3184     rigidentity.obj
 0003:000001d4       ?g_bSaferBooleans@@3HA     351e31d4     boolean3d.obj
 0003:000001f0       ?mtx_pool_size@?$matrix_tpl@M@@2HA 351e31f0     matrixnm.obj
 0003:000001f4       ?vecn_pool_size@?$vectorn_tpl@M@@2HA 351e31f4     matrixnm.obj
 0003:000001f8       ?mtx_pool_size@?$matrix_tpl@N@@2HA 351e31f8     matrixnm.obj
 0003:000003a0       ?defgwd@@3Ugeom_world_data@@A 351e33a0     geometry.obj
 0003:00000400       ?defip@@3Uintersection_params@@A 351e3400     geometry.obj
 0003:00000498       ?table@CIntersectionChecker@@2PAY07P6AHPBUprimitive@primitives@@0PAUprim_inters@@@ZA 351e3498     intersectionchecks.obj
 0003:00000598       ?default_function@CIntersectionChecker@@2P6AHPBUprimitive@primitives@@0PAUprim_inters@@@ZA 351e3598     intersectionchecks.obj
 0003:000005b4       ?g_jobName@@3PAPADA        351e35b4     jobq.obj
 0003:000005d0       ?table@CUnprojectionChecker@@2PAY177P6AHPAUunprojection_mode@@PBUprimitive@primitives@@H1HPAUcontact@@PAUgeom_contact_area@@@ZA 351e35d0     linunprojectionchecks.obj
 0003:00000800       ?table@COverlapChecker@@2PAY07P6AHPBUprimitive@primitives@@0PAV1@@ZA 351e3800     overlapchecks.obj
 0003:00000900       ?default_function@COverlapChecker@@2P6AHPBUprimitive@primitives@@0PAV1@@ZA 351e3900     overlapchecks.obj
 0003:00000a30       ?g_Overlapper@@3VCOverlapChecker@@A 351e3a30     trimesh.obj
 0003:00000a98       ?m_seed@CLCGRndGen@@0_KA   351e3a98     CryPhysics.obj
 0003:00000ae0       ___native_dllmain_reason   351e3ae0     MSVCRT:natstart.obj
 0003:00000ae4       ___native_vcclrit_reason   351e3ae4     MSVCRT:natstart.obj
 0003:00000ae8       ___security_cookie         351e3ae8     MSVCRT:gs_cookie.obj
 0003:00000aec       ___security_cookie_complement 351e3aec     MSVCRT:gs_cookie.obj
 0003:00000af0       ?__ae_step@@3HA            351e3af0     articulatedentity.obj
 0003:00000af4       ?__maxdiff@@3MA            351e3af4     articulatedentity.obj
 0003:00000af8       ?s_pMemReplay@?1??CryGetIMemReplay@@YAPAUIMemReplay@@XZ@4PAU2@A 351e3af8     articulatedentity.obj
 0003:00000afc       ?s_dummyMemReplay@?1??CryGetIMemReplay@@YAPAUIMemReplay@@XZ@4UCDummyMemReplay@@A 351e3afc     articulatedentity.obj
 0003:00000b00       ??_B?1??CryGetIMemReplay@@YAPAUIMemReplay@@XZ@51 351e3b00     articulatedentity.obj
 0003:00001200       ?g_pCurParticle@CParticleEntity@@2PAPAV1@A 351e4200     particleentity.obj
 0003:00001a6c       ?s_EmptyElems@?1??set_null@?$SmallDynStorage@MHUStandardAlloc@NAlloc@@@NArray@@IAEXXZ@4PAMA 351e4a6c     physarea.obj
 0003:00001a70       ?s_EmptyHeader@?1??set_null@?$SmallDynStorage@MHUStandardAlloc@NAlloc@@@NArray@@IAEXXZ@4UEmptyHeader@23@A 351e4a70     physarea.obj
 0003:00001a78       ??_B?1??set_null@?$SmallDynStorage@MHUStandardAlloc@NAlloc@@@NArray@@IAEXXZ@51 351e4a78     physarea.obj
 0003:00001a7c       ?s_EmptyElems@?1??set_null@?$SmallDynStorage@UGeomQuery@@HUStandardAlloc@NAlloc@@@NArray@@IAEXXZ@4PAUGeomQuery@@A 351e4a7c     physarea.obj
 0003:00001a80       ?s_EmptyHeader@?1??set_null@?$SmallDynStorage@UGeomQuery@@HUStandardAlloc@NAlloc@@@NArray@@IAEXXZ@4UEmptyHeader@23@A 351e4a80     physarea.obj
 0003:00001a88       ??_B?1??set_null@?$SmallDynStorage@UGeomQuery@@HUStandardAlloc@NAlloc@@@NArray@@IAEXXZ@51 351e4a88     physarea.obj
 0003:00001a90       ?g_parts@CPhysicalEntity@@2PAUSPartHelper@@A 351e4a90     physicalentity.obj
 0003:00001a94       ?g_joints@CPhysicalEntity@@2PAUSStructuralJointHelper@@A 351e4a94     physicalentity.obj
 0003:00001a98       ?g_jointsDbg@CPhysicalEntity@@2PAUSStructuralJointDebugHelper@@A 351e4a98     physicalentity.obj
 0003:00001a9c       ?g_jointidx@CPhysicalEntity@@2PAHA 351e4a9c     physicalentity.obj
 0003:00001aa0       ?g_nPartsAlloc@CPhysicalEntity@@2HA 351e4aa0     physicalentity.obj
 0003:00001aa4       ?g_nJointsAlloc@CPhysicalEntity@@2HA 351e4aa4     physicalentity.obj
 0003:00001aa8       ?g_pSliceMesh@@3PAVCTriMesh@@A 351e4aa8     physicalentity.obj
 0003:00001ab0       ?g_StaticRigidBodies@@3PAVRigidBody@@A 351e4ab0     physicalentity.obj
 0003:00001b80       ?g_StaticPhysicalEntity@@3VCPhysicalEntity@@A 351e4b80     physicalentity.obj
 0003:00001c78       ?m_defpart@CPhysicalEntity@@2Ugeom@@A 351e4c78     physicalentity.obj
 0003:00001ce4       ?s_used_memory@?1??_usedMemory@?$CryStringT@D@@SAIH@Z@4IA 351e4ce4     physicalentity.obj
 0003:00003c2c       ?serializeString@?1??SetSharedSerializeString@?$CSerializeWrapper@UISerialize@@@@QAEAAUSSerializeString@@ABV?$CryStringT@D@@@Z@4U3@A 351e6c2c     physicalentity.obj
 0003:00003c30       ??_B?1??SetSharedSerializeString@?$CSerializeWrapper@UISerialize@@@@QAEAAUSSerializeString@@ABV?$CryStringT@D@@@Z@51 351e6c30     physicalentity.obj
 0003:00003c38       ?g_nPhysWorlds@@3HA        351e6c38     physicalworld.obj
 0003:00003c40       ?g_pPhysWorlds@@3PAPAVCPhysicalWorld@@A 351e6c40     physicalworld.obj
 0003:00003d40       ?g_dummyBuf@@3PAHA         351e6d40     physicalworld.obj
 0003:00003d80       ?g_timeFiber@@3_JC         351e6d80     physicalworld.obj
 0003:00003d88       ?__curstep@@3HA            351e6d88     physicalworld.obj
 0003:0000c71c       ?g_RBdata@@3PAPAURBdata@@A 351ef71c     rigidbody.obj
 0003:0000c720       ?__solver_step@@3HA        351ef720     rigidbody.obj
 0003:0000d868       ?g_REdata@@3PAUREdata@@A   351f0868     rigidentity.obj
 0003:0000e478       ?__bstop@@3HA              351f1478     rigidentity.obj
 0003:0000e494       ?s_used_memory@?1??_usedMemory@?$CryStackStringT@D$0CAA@@@SAII@Z@4IA 351f1494     rigidentity.obj
 0003:0000f378       ?str@?1??numbered_tag@@YAPBDPBDI@Z@4PADA 351f2378     ropeentity.obj
 0003:00010278       ?g_lockProcessedAux@CPhysicalEntity@@2HC 351f3278     softentity.obj
 0003:00012820       ?g_BoolHash@@3PAIA         351f5820     boolean2d.obj
 0003:0001a820       ?g_BoolGrid@@3PAHA         351fd820     boolean2d.obj
 0003:0001e820       ?g_BoolIdBuf@@3PAHA        35201820     boolean2d.obj
 0003:00022828       ?g_BoolPtBuf@@3PAU?$Vec2_tpl@M@@A 35205828     boolean2d.obj
 0003:0002a828       ?g_BoolInters@@3PAUinters2d@@A 3520d828     boolean2d.obj
 0003:0002b828       ?g_nTriangulationErrors@@3HA 3520e828     boolean3d.obj
 0003:0002bba8       ?mtx_pool@?$matrix_tpl@M@@2PAMA 3520eba8     matrixnm.obj
 0003:0002c3a8       ?vecn_pool@?$vectorn_tpl@M@@2PAMA 3520f3a8     matrixnm.obj
 0003:0002c7a8       ?mtx_pool@?$matrix_tpl@N@@2PANA 3520f7a8     matrixnm.obj
 0003:0002d7a8       ?g_bHasSSE@@3HA            352107a8     matrixnm.obj
 0003:0002d7ac       ?mtx_pool_pos@?$matrix_tpl@M@@2HA 352107ac     matrixnm.obj
 0003:0002d7b0       ?vecn_pool_pos@?$vectorn_tpl@M@@2HA 352107b0     matrixnm.obj
 0003:0002d7b4       ?mtx_pool_pos@?$matrix_tpl@N@@2HA 352107b4     matrixnm.obj
 0003:0002d7b8       ?__qhullcalled@@3HA        352107b8     qhull.obj
 0003:00040bb0       ?g_pLockIntersect@@3PCHC   35223bb0     geometry.obj
 0003:00040bb8       ?g_idata@@3PAUintersData@@A 35223bb8     geometry.obj
 0003:0009fec9       ?g_Intersector@@3VCIntersectionChecker@@A 35282ec9     intersectionchecks.obj
 0003:0009fecc       ?g_pHFbuf@@3PAPAVCHeightfield@@A 35282ecc     jobq.obj
 0003:0009ff18       ?g_Unprojector@@3VCUnprojectionChecker@@A 35282f18     linunprojectionchecks.obj
 0003:0009ff50       ?dummyAreaPt@@3PAU?$Vec3_tpl@M@@A 35282f50     linunprojectionchecks.obj
 0003:000a0018       ?gSpuQuery3DengineForHeights@@3IA 35283018     rwi.obj
 0003:000a0030       ?g_RWIContacts@@3PAUgeom_contact@@A 35283030     rwi.obj
 0003:000a21a8       ?g_Faces@CTetrLattice@@2PAUSCGFace@@A 352851a8     tetrlattice.obj
 0003:000a21ac       ?g_Tets@CTetrLattice@@2PAUSCGTetr@@A 352851ac     tetrlattice.obj
 0003:000a21b0       ?g_nFacesAlloc@CTetrLattice@@2HA 352851b0     tetrlattice.obj
 0003:000a21b4       ?g_nTetsAlloc@CTetrLattice@@2HA 352851b4     tetrlattice.obj
 0003:000a2530       ?__gtrimesh@@3HA           35285530     trimesh.obj
 0003:000a28c0       ?g_subrefBuf@@3PAUsubref@@A 352858c0     CryPhysics.obj
 0003:000a2a28       ?g_sintab@@3PAMA           35285a28     CryPhysics.obj
 0003:000a3a2c       ?numAllocations@_CryMemoryManagerPoolHelper@@2HC 35286a2c     CryPhysics.obj
 0003:000a3a30       ?requestedMemory@_CryMemoryManagerPoolHelper@@2JC 35286a30     CryPhysics.obj
 0003:000a3a34       ?freedMemory@_CryMemoryManagerPoolHelper@@2JC 35286a34     CryPhysics.obj
 0003:000a3a38       ?allocatedMemory@_CryMemoryManagerPoolHelper@@2JC 35286a38     CryPhysics.obj
 0003:000a3a3c       ?g_subrefGeomParams@@3PAPAUsubref@@A 35286a3c     CryPhysics.obj
 0003:000a3a48       ?g_subrefAction@@3PAPAUsubref@@A 35286a48     CryPhysics.obj
 0003:000a3a90       ?g_subrefParams@@3PAPAUsubref@@A 35286a90     CryPhysics.obj
 0003:000a3afc       ?g_szGeomParams@@3PAHA     35286afc     CryPhysics.obj
 0003:000a3b08       ?g_szAction@@3PAHA         35286b08     CryPhysics.obj
 0003:000a3b50       ?g_szParams@@3PAHA         35286b50     CryPhysics.obj
 0003:000a3bbc       ?gEnv@@3PAUSSystemGlobalEnvironment@@A 35286bbc     CryPhysics.obj
 0003:000a3bc0       ?m_pFirst@Test@CryUnitTest@@2PAU12@A 35286bc0     CryPhysics.obj
 0003:000a3bc4       ?m_pLast@Test@CryUnitTest@@2PAU12@A 35286bc4     CryPhysics.obj
 0003:000a3bc8       ?g_pHeadToRegFactories@@3PAUSRegFactoryNode@@A 35286bc8     CryPhysics.obj
 0003:000a3bcc       ?g_bProfilerEnabled@@3_NA  35286bcc     CryPhysics.obj
 0003:000a3bd0       ?g_iTraceAllocations@@3HA  35286bd0     CryPhysics.obj
 0003:000a3bd4       ?_CryMalloc@_CryMemoryManagerPoolHelper@@2P6APAXIAAII@ZA 35286bd4     CryPhysics.obj
 0003:000a3bd8       ?_CryGetMemSize@_CryMemoryManagerPoolHelper@@2P6AIPAXI@ZA 35286bd8     CryPhysics.obj
 0003:000a3bdc       ?_CryRealloc@_CryMemoryManagerPoolHelper@@2P6APAXPAXIAAI1I@ZA 35286bdc     CryPhysics.obj
 0003:000a3be0       ?_CryFree@_CryMemoryManagerPoolHelper@@2P6AIPAXI@ZA 35286be0     CryPhysics.obj
 0003:000a3be4       ?_CryCrtMalloc@_CryMemoryManagerPoolHelper@@2P6APAXI@ZA 35286be4     CryPhysics.obj
 0003:000a3be8       ?_CryCrtRealloc@_CryMemoryManagerPoolHelper@@2P6APAXPAXI@ZA 35286be8     CryPhysics.obj
 0003:000a3bec       ?_CryCrtFree@_CryMemoryManagerPoolHelper@@2P6AIPAX@ZA 35286bec     CryPhysics.obj
 0003:000a3bf0       ?_CryCrtSize@_CryMemoryManagerPoolHelper@@2P6AIPAX@ZA 35286bf0     CryPhysics.obj
 0003:000a3bf4       ?_CryGetIMemoryManagerInterface@_CryMemoryManagerPoolHelper@@2P6AXPAPAX@ZA 35286bf4     CryPhysics.obj
 0003:000a3bf8       ?m_bInitialized@_CryMemoryManagerPoolHelper@@2HA 35286bf8     CryPhysics.obj
 0003:000a3bfc       ?g_random_generator@@3VCLCGRndGen@@A 35286bfc     CryPhysics.obj
 0003:000a3bfd       ?Now@@3VInitPhysicsGlobals@@A 35286bfd     CryPhysics.obj
 0003:000a3c00       ?s_factory@CFactory@CEngineModule_CryPhysics@@0V12@A 35286c00     CryPhysics.obj
 0003:000a3c30       ?s_used_memory@?1??_usedMemory@?$CryStringT@_W@@SAIH@Z@4IA 35286c30     CryPhysics.obj
 0003:000a3c38       ?supportedIIDs@?1???0CFactory@CEngineModule_CryPhysics@@AAE@XZ@4PAUCryGUID@@A 35286c38     CryPhysics.obj
 0003:000a3c58       ?p@?1??CreateClassInstance@CFactory@CEngineModule_CryPhysics@@UBE?AV?$shared_ptr@UICryUnknown@@@boost@@XZ@4V?$shared_ptr@VCEngineModule_CryPhysics@@@5@A 35286c58     CryPhysics.obj
 0003:000a3c60       ??_B?1??CreateClassInstance@CFactory@CEngineModule_CryPhysics@@UBE?AV?$shared_ptr@UICryUnknown@@@boost@@XZ@51 35286c60     CryPhysics.obj
 0003:000a3c68       ?g_globalSections@?$Node_Alloc_Lock@$00$00@@2PAUInternalCriticalSectionDummy@@A 35286c68     StdAfx.obj
 0003:000a5ce8       ?m_bInitialized@?$Node_Alloc_Lock@$00$00@@2_NA 35288ce8     StdAfx.obj
 0003:000a5cf0       ?__type_info_root_node@@3U__type_info_node@@A 35288cf0     MSVCRT:tncleanup.obj
 0003:000a601c       ___native_startup_state    3528901c     <common>
 0003:000a6020       ___native_startup_lock     35289020     <common>
 0003:000a6024       ___sse2_available          35289024     <common>
 0003:000a6028       ___dyn_tls_init_callback   35289028     <common>
 0003:000a602c       ___onexitend               3528902c     <common>
 0003:000a6030       ___onexitbegin             35289030     <common>
 0004:00000000       ?m_Self@CrySimpleThreadSelf@@1PAV1@A 3528a000     CryPhysics.obj

 entry point at        0001:001db9f0

 Static symbols

 0001:000454c0       ?qsort@@YAXPAMPAHHH@Z      350464c0 f   physarea.obj
 0001:00045f10       ?SignalEventAreaChange@@YAXPAVCPhysicalWorld@@PAVCPhysArea@@@Z 35046f10 f   physarea.obj
 0001:0007d530       ?qsort@@YAXPAPAVCPhysicalEntity@@PAMPAHHH@Z 3507e530 f   physicalworld.obj
 0001:00083500       ?qsort@@YAXPAPAVCPhysicalEntity@@ABU?$Vec3_tpl@M@@1HH@Z 35084500 f   physicalworld.obj
 0001:00083b00       ?CreateTriMesh@@YAXAAVCTriMesh@@PAUtriangle@primitives@@@Z 35084b00 f   physicalworld.obj
 0001:00098f50       ??$qsort@PAUentity_contact@@@@YAXPAPAUentity_contact@@HHH@Z 35099f50 f   rigidbody.obj
 0001:00099010       ??$qsort@PAVRigidBody@@@@YAXPAPAVRigidBody@@HHH@Z 3509a010 f   rigidbody.obj
 0001:00099100       ??$qsort@PAUentity_contact_unproj@@@@YAXPAPAUentity_contact_unproj@@HHH@Z 3509a100 f   rigidbody.obj
 0001:000ae490       ?qsort@@YAXPAUedgeitem@@HH@Z 350af490 f   rigidentity.obj
 0001:0011fcf0       ?qsort@@YAXPAHPAPAXHH@Z    35120cf0 f   qhull.obj
 0001:001b70f0       ?ExpandGlobalLoadState@@YAXH@Z 351b80f0 f   trimesh.obj
 0001:001db682       _pre_c_init                351dc682 f   MSVCRT:crtdll.obj
 0001:001db8da       ___DllMainCRTStartup       351dc8da f   MSVCRT:crtdll.obj
 0001:001dbe70       ??__Eg_stub@@YAXXZ         351dce70 f   physarea.obj
 0001:001dbe80       ??__Eg_StaticRigidBodies@@YAXXZ 351dce80 f   physicalentity.obj
 0001:001dbe90       ??__Eg_StaticPhysicalEntity@@YAXXZ 351dce90 f   physicalentity.obj
 0001:001dbeb0       ??__ECryUserInvalidID@@YAXXZ 351dceb0 f   rigidentity.obj
 0001:001dbec0       ??__ECrySessionInvalidID@@YAXXZ 351dcec0 f   rigidentity.obj
 0001:001dbed0       ??__Eg_idata@@YAXXZ        351dced0 f   geometry.obj
 0001:001dc0c0       ??__Enow@@YAXXZ            351dd0c0 f   geometry.obj
 0001:001dc0d0       ??__EinitHeightfieldGlobals@@YAXXZ 351dd0d0 f   heightfieldbv.obj
 0001:001dc0f0       ??__EinitTriMeshGlobals@@YAXXZ 351dd0f0 f   trimesh.obj
 0001:001dc100       ??__EinitVoxgridGlobals@@YAXXZ 351dd100 f   voxelbv.obj
 0001:001dc120       ??__Eg_random_generator@@YAXXZ 351dd120 f   CryPhysics.obj
 0001:001dc140       ??__Eg_system_event_listener_physics@@YAXXZ 351dd140 f   CryPhysics.obj
 0001:001dc150       ??__ENow@@YAXXZ            351dd150 f   CryPhysics.obj
 0001:001dc160       ??__E?s_factory@CFactory@CEngineModule_CryPhysics@@0V12@A@@YAXXZ 351dd160 f   CryPhysics.obj
 0001:001dc180       ??__EautoInitializer@@YAXXZ 351dd180 f   StdAfx.obj
 0001:001dc1d0       ??__Fg_stub@@YAXXZ         351dd1d0 f   physarea.obj
 0001:001dc1e0       ??__Fg_StaticPhysicalEntity@@YAXXZ 351dd1e0 f   physicalentity.obj
 0001:001dc220       ??__Fg_entSoft@?1??SetStateFromTypedSnapshot@CPhysicalEntity@@UAEHV?$CSerializeWrapper@UISerialize@@@@HH@Z@YAXXZ 351dd220 f   physicalworld.obj
 0001:001dc230       ??__Fg_entRope@?1??SetStateFromTypedSnapshot@CPhysicalEntity@@UAEHV?$CSerializeWrapper@UISerialize@@@@HH@Z@YAXXZ 351dd230 f   physicalworld.obj
 0001:001dc240       ??__Fg_entArticulated@?1??SetStateFromTypedSnapshot@CPhysicalEntity@@UAEHV?$CSerializeWrapper@UISerialize@@@@HH@Z@YAXXZ 351dd240 f   physicalworld.obj
 0001:001dc250       ??__Fg_entParticle@?1??SetStateFromTypedSnapshot@CPhysicalEntity@@UAEHV?$CSerializeWrapper@UISerialize@@@@HH@Z@YAXXZ 351dd250 f   physicalworld.obj
 0001:001dc260       ??__Fg_entLiving@?1??SetStateFromTypedSnapshot@CPhysicalEntity@@UAEHV?$CSerializeWrapper@UISerialize@@@@HH@Z@YAXXZ 351dd260 f   physicalworld.obj
 0001:001dc270       ??__Fg_entRigid@?1??SetStateFromTypedSnapshot@CPhysicalEntity@@UAEHV?$CSerializeWrapper@UISerialize@@@@HH@Z@YAXXZ 351dd270 f   physicalworld.obj
 0001:001dc280       ??__Fg_entStatic@?1??SetStateFromTypedSnapshot@CPhysicalEntity@@UAEHV?$CSerializeWrapper@UISerialize@@@@HH@Z@YAXXZ 351dd280 f   physicalworld.obj
 0001:001dc290       ??__Fg_entSoft@?1??SerializeGarbageTypedSnapshot@CPhysicalWorld@@UAEXV?$CSerializeWrapper@UISerialize@@@@HH@Z@YAXXZ 351dd290 f   physicalworld.obj
 0001:001dc2a0       ??__Fg_entRope@?1??SerializeGarbageTypedSnapshot@CPhysicalWorld@@UAEXV?$CSerializeWrapper@UISerialize@@@@HH@Z@YAXXZ 351dd2a0 f   physicalworld.obj
 0001:001dc2b0       ??__Fg_entArticulated@?1??SerializeGarbageTypedSnapshot@CPhysicalWorld@@UAEXV?$CSerializeWrapper@UISerialize@@@@HH@Z@YAXXZ 351dd2b0 f   physicalworld.obj
 0001:001dc2c0       ??__Fg_entParticle@?1??SerializeGarbageTypedSnapshot@CPhysicalWorld@@UAEXV?$CSerializeWrapper@UISerialize@@@@HH@Z@YAXXZ 351dd2c0 f   physicalworld.obj
 0001:001dc2d0       ??__Fg_entLiving@?1??SerializeGarbageTypedSnapshot@CPhysicalWorld@@UAEXV?$CSerializeWrapper@UISerialize@@@@HH@Z@YAXXZ 351dd2d0 f   physicalworld.obj
 0001:001dc2e0       ??__Fg_entWheeled@?1??SerializeGarbageTypedSnapshot@CPhysicalWorld@@UAEXV?$CSerializeWrapper@UISerialize@@@@HH@Z@YAXXZ 351dd2e0 f   physicalworld.obj
 0001:001dc2f0       ??__Fg_entRigid@?1??SerializeGarbageTypedSnapshot@CPhysicalWorld@@UAEXV?$CSerializeWrapper@UISerialize@@@@HH@Z@YAXXZ 351dd2f0 f   physicalworld.obj
 0001:001dc300       ??__Fg_entStatic@?1??SerializeGarbageTypedSnapshot@CPhysicalWorld@@UAEXV?$CSerializeWrapper@UISerialize@@@@HH@Z@YAXXZ 351dd300 f   physicalworld.obj
 0001:001dc310       ??__Fg_entWheeled@?1??SetStateFromTypedSnapshot@CPhysicalEntity@@UAEHV?$CSerializeWrapper@UISerialize@@@@HH@Z@YAXXZ 351dd310 f   physicalworld.obj
 0001:001dc320       ??__FCrySessionInvalidID@@YAXXZ 351dd320 f   rigidentity.obj
 0001:001dc360       ??__FCryUserInvalidID@@YAXXZ 351dd360 f   rigidentity.obj
 0001:001dc3a0       ??__Fg_system_event_listener_physics@@YAXXZ 351dd3a0 f   CryPhysics.obj
 0001:001dc3b0       ??__F?s_factory@CFactory@CEngineModule_CryPhysics@@0V12@A@@YAXXZ 351dd3b0 f   CryPhysics.obj
 0001:001dc410       ??__FautoInitializer@@YAXXZ 351dd410 f   StdAfx.obj
